:020000040800F2
:100000000000052049230008752100087721000819
:10001000792100087B2100087D21000800000000F4
:10002000000000000000000000000000D1AB00084C
:100030007F2100080000000071AC0008992300082F
:1000400099230008992300089923000899230008A0
:100050009923000899230008992300089923000890
:100060009923000899230008992300089923000880
:100070009923000899230008992300089923000870
:100080009923000899230008992300089923000860
:100090009923000899230008992300089923000850
:1000A0009923000899230008992300089923000840
:1000B0009923000899230008992300089923000830
:1000C0009923000899230008992300089923000820
:1000D0009923000899230008992300089923000810
:1000E0009923000899230008992300089923000800
:1000F00099230008992300089923000899230008F0
:1001000099230008992300089923000899230008DF
:1001100099230008992300088121000899230008E9
:1001200099230008992300089923000899230008BF
:1001300099230008992300089923000899230008AF
:100140009923000899230008992300088D210008AD
:10015000992300089923000899230008992300088F
:10016000992300089923000899230008992300087F
:100170009923000899230008992300080000000033
:10018000992300089923000899230008992300085F
:10019000992300089923000899230008992300084F
:1001A0009921000899230008A52100089923000837
:1001B000992300089923000899230008992300082F
:0801C0009923000899230008AF
:1001D00010B5054C237833B9044B13B10448AFF381
:1001E00000800123237010BD501200200000000089
:1001F00074EA050808B5034B1BB103490348AFF384
:10020000008008BD000000005412002074EA0508B8
:1002100001F0FF01102A2BDB10F0070F08D010F8B7
:10022000013B013A8B422DD010F0070F42B3F6D1BB
:10023000F0B441EA012141EA014122F007047FF0D4
:1002400000070023F0E80256083C85EA010586EA2B
:10025000010685FA47F5A3FA87F586FA47F6A5FA67
:1002600087F68EB9EED1F0BC01F0FF0102F0070273
:1002700032B110F8013B013A83EA010313B1F8D11E
:100280000020704701387047002D06BF35460338FF
:10029000073815F0010F07D1013015F4807F02BF38
:1002A000013015F4C03F0130F0BC0138704700BF89
:1002B00010F8012B11F8013B012A28BF9A42F7D010
:1002C000D01A7047034613F8012B002AFBD1181AE5
:1002D0000138704781F0004102E000BF83F0004325
:1002E00030B54FEA41044FEA430594EA050F08BFD1
:1002F00090EA020F1FBF54EA000C55EA020C7FEA95
:10030000645C7FEA655C00F0E2804FEA5454D4EB11
:100310005555B8BF6D420CDD2C4480EA020281EADB
:10032000030382EA000083EA010180EA020281EA13
:100330000303362D88BF30BD11F0004F4FEA013165
:100340004FF4801C4CEA113102D0404261EB410174
:1003500013F0004F4FEA03334CEA133302D05242FA
:1003600063EB430394EA050F00F0A780A4F10104B6
:10037000D5F1200E0DDB02FA0EFC22FA05F28018F0
:1003800041F1000103FA0EF2801843FA05F35941D6
:100390000EE0A5F120050EF1200E012A03FA0EFC55
:1003A00028BF4CF0020C43FA05F3C01851EBE3717F
:1003B00001F0004507D54FF0000EDCF1000C7EEB9C
:1003C00000006EEB0101B1F5801F1BD3B1F5001FDA
:1003D0000CD349085FEA30004FEA3C0C04F10104F9
:1003E0004FEA445212F5800F80F09A80BCF1004F22
:1003F00008BF5FEA500C50F1000041EB045141EAA4
:10040000050130BD5FEA4C0C404141EB0101013C6C
:1004100028BFB1F5801FE9D291F0000F04BF01465B
:100420000020B1FA81F308BF2033A3F10B03B3F12D
:1004300020020CDA0C3208DD02F1140CC2F10C02BD
:1004400001FA0CF021FA02F10CE002F11402D8BF1B
:10045000C2F1200C01FA02F120FA0CFCDCBF41EAE7
:100460000C019040E41AA2BF01EB0451294330BDB6
:100470006FEA04041F3C1CDA0C340EDC04F1140493
:10048000C4F1200220FA04F001FA02F340EA03006A
:1004900021FA04F345EA030130BDC4F10C04C4F1B0
:1004A000200220FA02F001FA04F340EA0300294690
:1004B00030BD21FA04F0294630BD94F0000F83F4DA
:1004C000801306BF81F480110134013D4EE77FEABD
:1004D000645C18BF7FEA655C29D094EA050F08BF09
:1004E00090EA020F05D054EA000C04BF19461046EA
:1004F00030BD91EA030F1EBF0021002030BD5FEA2E
:10050000545C05D14000494128BF41F0004130BD55
:1005100014F580043CBF01F5801130BD01F00045A9
:1005200045F0FE4141F470014FF0000030BD7FEA1C
:10053000645C1ABF194610467FEA655C1CBF0B4617
:10054000024650EA013406BF52EA033591EA030F2E
:1005500041F4002130BD00BF90F0000F04BF002126
:10056000704730B54FF4806404F132044FF0000559
:100570004FF0000150E700BF90F0000F04BF0021D2
:10058000704730B54FF4806404F1320410F0004538
:1005900048BF40424FF000013EE700BF42004FEA33
:1005A000E2014FEA31014FEA02701FBF12F07F43B0
:1005B00093F07F4F81F06051704732F07F4208BF67
:1005C000704793F07F4F04BF41F40021704730B56E
:1005D0004FF4607401F0004521F000411CE700BFBA
:1005E00050EA010208BF704730B54FF000050AE03D
:1005F00050EA010208BF704730B511F0004502D53E
:10060000404261EB41014FF4806404F132045FEA3F
:10061000915C3FF4D8AE4FF003025FEADC0C18BFE8
:1006200003325FEADC0C18BF033202EBDC02C2F1DA
:10063000200300FA03FC20FA02F001FA03FE40EA6C
:100640000E0021FA02F11444BDE600BF70B54FF070
:10065000FF0C4CF4E06C1CEA11541DBF1CEA13554E
:1006600094EA0C0F95EA0C0F00F0DEF82C4481EAB6
:10067000030621EA4C5123EA4C5350EA013518BFD6
:1006800052EA033541F4801143F4801338D0A0FBC3
:1006900002CE4FF00005E1FB02E506F00042E0FB70
:1006A00003E54FF00006E1FB03569CF0000F18BF76
:1006B0004EF0010EA4F1FF04B6F5007F64F540741E
:1006C00004D25FEA4E0E6D4146EB060642EAC621B1
:1006D00041EA55514FEAC52040EA5E504FEACE2E1E
:1006E000B4F1FD0C88BFBCF5E06F1ED8BEF1004F21
:1006F00008BF5FEA500E50F1000041EB045170BD9D
:1007000006F0004646EA010140EA020081EA0301E0
:10071000B4EB5C04C2BFD4EB0C0541EA045170BDDC
:1007200041F480114FF0000E013C00F3AB8014F156
:10073000360FDEBF002001F0004170BDC4F100049F
:10074000203C35DA0C341BDC04F11404C4F1200520
:1007500000FA05F320FA04F001FA05F240EA02007B
:1007600001F0004221F0004110EBD37021FA04F6B1
:1007700042EB06015EEA430E08BF20EAD37070BD6B
:10078000C4F10C04C4F1200500FA04F320FA05F0CA
:1007900001FA04F240EA020001F0004110EBD370CC
:1007A00041F100015EEA430E08BF20EAD37070BD3C
:1007B000C4F1200500FA05F24EEA020E20FA04F315
:1007C00001FA05F243EA020321FA04F001F00041C4
:1007D00021FA04F220EA020000EBD3705EEA430E35
:1007E00008BF20EAD37070BD94F0000F0FD101F064
:1007F0000046400041EB010111F4801F08BF013C9D
:10080000F7D041EA060195F0000F18BF704703F0DA
:100810000046520043EB030313F4801F08BF013D61
:10082000F7D043EA0603704794EA0C0F0CEA13551D
:1008300018BF95EA0C0F0CD050EA410618BF52EAD7
:100840004306D1D181EA030101F000414FF00000DD
:1008500070BD50EA410606BF1046194652EA4306EB
:1008600019D094EA0C0F02D150EA013613D195EA5F
:100870000C0F05D152EA03361CBF104619460AD1A7
:1008800081EA030101F0004141F0FE4141F47001B1
:100890004FF0000070BD41F0FE4141F4780170BDA1
:1008A00070B54FF0FF0C4CF4E06C1CEA11541DBF06
:1008B0001CEA135594EA0C0F95EA0C0F00F0A7F808
:1008C000A4EB050481EA030E52EA03354FEA013135
:1008D00000F088804FEA03334FF0805545EA131348
:1008E00043EA12634FEA022245EA111545EA106510
:1008F0004FEA00260EF000419D4208BF964244F1A7
:10090000FD0404F5407402D25B084FEA3202B61AC5
:1009100065EB03055B084FEA32024FF480104FF499
:10092000002CB6EB020E75EB030E22BFB61A75460D
:1009300040EA0C005B084FEA3202B6EB020E75EBA0
:10094000030E22BFB61A754640EA5C005B084FEA08
:100950003202B6EB020E75EB030E22BFB61A7546D5
:1009600040EA9C005B084FEA3202B6EB020E75EBE0
:10097000030E22BFB61A754640EADC0055EA060EA1
:1009800018D04FEA051545EA16754FEA06164FEAE4
:10099000C30343EA52734FEAC2025FEA1C1CC0D190
:1009A00011F4801F0BD141EA00014FF000004FF01D
:1009B000004CB6E711F4801F04BF01430020B4F1DE
:1009C000FD0C88BFBCF5E06F3FF6AFAEB5EB030C96
:1009D00004BFB6EB020C5FEA500C50F1000041EB93
:1009E000045170BD0EF0004E4EEA113114EB5C0460
:1009F000C2BFD4EB0C0541EA045170BD41F4801133
:100A00004FF0000E013C90E645EA060E8DE60CEA3A
:100A1000135594EA0C0F08BF95EA0C0F3FF43BAF57
:100A200094EA0C0F0AD150EA01347FF434AF95EA0E
:100A30000C0F7FF425AF104619462CE795EA0C0FF2
:100A400006D152EA03353FF4FDAE1046194622E7BF
:100A500050EA410618BF52EA43067FF4C5AE50EA99
:100A600041047FF40DAF52EA43057FF4EBAE12E789
:100A70004FF0FF3C06E000BF4FF0010C02E000BF6A
:100A80004FF0010C4DF804CD4FEA410C7FEA6C5C4D
:100A90004FEA430C18BF7FEA6C5C1BD001B050EAF0
:100AA000410C0CBF52EA430C91EA030F02BF90EADB
:100AB000020F0020704710F1000F91EA030F58BF9A
:100AC000994208BF90422CBFD8176FEAE37040F0FC
:100AD000010070474FEA410C7FEA6C5C02D150EA9A
:100AE000013C07D14FEA430C7FEA6C5CD6D152EA55
:100AF000033CD3D05DF8040B704700BF844610461A
:100B000062468C461946634600E000BF01B5FFF718
:100B1000B7FF002848BF10F1000F01BD4DF808EDE8
:100B2000FFF7F4FF0CBF012000205DF808FB00BFB9
:100B30004DF808EDFFF7EAFF34BF012000205DF813
:100B400008FB00BF4DF808EDFFF7E0FF94BF012060
:100B500000205DF808FB00BF4DF808EDFFF7CEFF61
:100B600094BF012000205DF808FB00BF4DF808EDA0
:100B7000FFF7C4FF34BF012000205DF808FB00BF71
:100B80004FEA410C7FEA6C5C02D150EA013C0AD189
:100B90004FEA430C7FEA6C5C02D152EA033C02D17B
:100BA0004FF0000070474FF0010070474FEA4102DC
:100BB00012F5001215D211D56FF47873B3EB6252AF
:100BC00012D94FEAC12343F0004343EA505311F0D6
:100BD000004F23FA02F018BF404270474FF0000068
:100BE000704750EA013005D111F0004008BF6FF0A6
:100BF000004070474FF00000704700BF4A0011D21C
:100C000012F5001211D20DD56FF47873B3EB625266
:100C10000ED44FEAC12343F0004343EA505323FA72
:100C200002F070474FF00000704750EA013002D1E7
:100C30004FF0FF3070474FF0000070474FEA41021D
:100C4000B2F1E04324BFB3F5001CDCF1FE5C0DD92A
:100C500001F0004C4FEAC0024CEA5070B2F1004F74
:100C600040EB830008BF20F00100704711F0804F77
:100C700021D113F13872BCBF01F00040704741F43C
:100C800080114FEA5252C2F11802C2F1200C10FA40
:100C90000CF320FA02F018BF40F001004FEAC12324
:100CA0004FEAD32303FA0CFC40EA0C0023FA02F3C8
:100CB0004FEA4303CCE77FEA625307D150EA01339E
:100CC0001EBF4FF0FE4040F44000704701F000406E
:100CD00040F0FE4040F40000704700BF80F000404C
:100CE00002E000BF81F0004142001FBF5FEA410304
:100CF00092EA030F7FEA226C7FEA236C6AD04FEA04
:100D00001262D2EB1363C1BFD21841404840414048
:100D1000B8BF5B42192B88BF704710F0004F40F4FA
:100D2000000020F07F4018BF404211F0004F41F416
:100D3000000121F07F4118BF494292EA030F3FD0E2
:100D4000A2F1010241FA03FC10EB0C00C3F12003F5
:100D500001FA03F100F0004302D5494260EB400084
:100D6000B0F5000F13D3B0F1807F06D340084FEAEF
:100D7000310102F10102FE2A51D2B1F1004F40EBE4
:100D8000C25008BF20F0010040EA0300704749004C
:100D900040EB0000013A28BFB0F5000FEDD2B0FAE9
:100DA00080FCACF1080CB2EB0C0200FA0CF0AABF0C
:100DB00000EBC25052421843BCBFD04018437047AA
:100DC00092F0000F81F4000106BF80F400000132B0
:100DD000013BB5E74FEA41037FEA226C18BF7FEA87
:100DE000236C21D092EA030F04D092F0000F08BFC9
:100DF0000846704790EA010F1CBF0020704712F0B0
:100E00007F4F04D1400028BF40F00040704712F1EE
:100E100000723CBF00F50000704700F0004343F053
:100E2000FE4040F4000070477FEA226216BF084689
:100E30007FEA23630146420206BF5FEA412390EA4C
:100E4000010F40F4800070474FF0000304E000BF42
:100E500010F0004348BF40425FEA000C08BF7047F3
:100E600043F0964301464FF000001CE050EA0102B7
:100E700008BF70474FF000030AE000BF50EA0102CC
:100E800008BF704711F0004302D5404261EB4101B9
:100E90005FEA010C02BF84460146002043F0B643DE
:100EA00008BFA3F18053A3F50003BCFA8CF2083A03
:100EB000A3EBC25310DB01FA02FC634400FA02FC0C
:100EC000C2F12002BCF1004F20FA02F243EB020013
:100ED00008BF20F00100704702F1200201FA02FC75
:100EE000C2F1200250EA4C0021FA02F243EB020068
:100EF00008BF20EADC7070477BB972B90029BEBF19
:100F000000204FF0004106E008BF00281CBF6FF032
:100F100000414FF0FF3000F029BAADF1080C6DE947
:100F200004CE002909DB002B1ADB00F0B7F8DDF84E
:100F300004E0DDE9022304B07047404261EB410167
:100F4000002B1BDB00F0AAF8DDF804E0DDE902234A
:100F500004B0404261EB4101524263EB43037047EE
:100F6000524263EB430300F099F8DDF804E0DDE959
:100F7000022304B0404261EB41017047524263EBEF
:100F8000430300F08BF8DDF804E0DDE9022304B050
:100F9000524263EB4303704753B94AB9002908BF73
:100FA00000281CBF4FF0FF314FF0FF3000F0DEB9DA
:100FB000ADF1080C6DE904CE00F070F8DDF804E046
:100FC000DDE9022304B0704707EE900AF5EEC07A1F
:100FD000F1EE10FA01D400F023B8F1EE677A08B50B
:100FE00017EE900A00F01CF8404261EB410108BD89
:100FF00038B50022002304460D46FFF799FD28B9B5
:1010000020462946BDE8384000F02AB8204605F1C0
:10101000004100F025F8404261EB410138BD00BFBE
:10102000D0B5FFF7BBFA0C4B002206460F46FFF780
:101030000DFBFFF7E3FD0446FFF78EFA074B002296
:10104000FFF704FB02460B4630463946FFF746F9E8
:10105000FFF7D4FD2146D0BD0000F03D0000F04177
:10106000D0B50C4B002206460F46FFF7EFFAFFF70C
:10107000C5FD0446FFF770FA074B0022FFF7E6FABA
:1010800002460B4630463946FFF728F9FFF7B6FD12
:101090002146D0BD0000F03D0000F0412DE9F047B1
:1010A000089D04468E46002B4DD18A42944669D94C
:1010B000B2FA82F252B101FA02F3C2F1200120FA2F
:1010C00001F10CFA02FC41EA030E94404FEA1C487D
:1010D000210CBEFBF8F61FFA8CF708FB16E341EA79
:1010E000034306FB07F199420AD91CEB030306F1FF
:1010F000FF3080F01F81994240F21C81023E634420
:101100005B1AA4B2B3FBF8F008FB103344EA0344C3
:1011100000FB07F7A7420AD91CEB040400F1FF33D8
:1011200080F00A81A74240F207816444023840EA15
:101130000640E41B00261DB1D4400023C5E900434E
:101140003146BDE8F0878B4209D9002D00F0EF80D1
:101150000026C5E9000130463146BDE8F087B3FA04
:1011600083F6002E4AD18B4202D3824200F2F980EC
:10117000841A61EB030301209E46002DE0D0C5E9EF
:10118000004EDDE702B9FFDEB2FA82F2002A40F03B
:101190009280A1EB0C014FEA1C471FFA8CFE01263E
:1011A000200CB1FBF7F307FB131140EA01410EFBE2
:1011B00003F0884208D91CEB010103F1FF3802D289
:1011C000884200F2CB804346091AA4B2B1FBF7F083
:1011D00007FB101144EA01440EFB00FEA64508D9A6
:1011E0001CEB040400F1FF3102D2A64500F2BB80E3
:1011F0000846A4EB0E0440EA03409CE7C6F1200732
:10120000B34022FA07FC4CEA030C20FA07F401FA77
:1012100006F31C43F9404FEA1C4900FA06F3B1FB00
:10122000F9F8200C1FFA8CFE09FB181140EA014165
:1012300008FB0EF0884202FA06F20BD91CEB010102
:1012400008F1FF3A80F08880884240F28580A8F15A
:1012500002086144091AA4B2B1FBF9F009FB1011AC
:1012600044EA014100FB0EFE8E4508D91CEB01014A
:1012700000F1FF346CD28E456AD90238614440EAED
:101280000840A0FB0294A1EB0E01A142C846A6466D
:1012900056D353D05DB1B3EB080261EB0E0101FAF6
:1012A00007F722FA06F3F1401F43C5E90071002653
:1012B0003146BDE8F087C2F12003D8400CFA02FCA9
:1012C00021FA03F3914001434FEA1C471FFA8CFEB9
:1012D000B3FBF7F007FB10360B0C43EA064300FBA9
:1012E0000EF69E4204FA02F408D91CEB030300F147
:1012F000FF382FD29E422DD9023863449B1B89B2FE
:10130000B3FBF7F607FB163341EA034106FB0EF386
:101310008B4208D91CEB010106F1FF3816D28B4233
:1013200014D9023E6144C91A46EA004638E72E46FF
:10133000284605E70646E3E61846F8E64B45A9D2F7
:10134000B9EB020864EB0C0E0138A3E74646EAE766
:10135000204694E74046D1E7D0467BE7023B614414
:1013600032E7304609E76444023842E7704700BF7D
:1013700008B50848084B036000238380C0E90533A3
:101380000123036201F0D2FE18B1BDE8084000F06D
:1013900099BD08BD6C12002000300240026882B086
:1013A000084B9A420BD1D3F8302803F5006342F47E
:1013B00080521A631B6B03F480530193019B02B0AC
:1013C000704700BF0030024008B50D4800230D4AA9
:1013D000C0E90A33C0E90C33C0E90023C0E9023395
:1013E00002F043F808B100F06DFD0121044802F05D
:1013F000AFF918B1BDE8084000F064BD08BD00BFFA
:101400009012002000B002400E4B07B502689A42CD
:1014100015D1A3F5F04305215A201A6B42F40002BE
:101420001A6300221B6B03F400030193019B01F07C
:101430003DFE5A2003B05DF804EB01F069BE03B035
:101440005DF804FB00B0024016480023164A042150
:101450004FF0400C00B5C0E9002310224FF4006E9D
:1014600089B08360C36183620223C0E903124FF431
:10147000C0720793C0E905C24FF48052C0E908E288
:101480000722CDE90312CDE9013203226944CDE9F7
:10149000052305F049F808B100F014FD09B05DF826
:1014A00004FB00BFD4120020400100A0F0B50023CF
:1014B00087B00393294B1E68002E4DD101220227CD
:1014C00003250C241A6001A9254B26489A6B42F08B
:1014D00001029A639B6B03F001030093009B4FF69C
:1014E0008373CDE90454CDE9013702F079F948F26C
:1014F000331301A91C480594CDE90137CDE90365F3
:1015000002F06EF94CF2037301A918480594CDE975
:101510000137CDE9036502F063F94FF63F0301A9F6
:1015200013480594CDE90137CDE9036502F058F978
:10153000282301A90F480594CDE90137CDE90365BA
:1015400002F04EF9082301A90B480594CDE90137B3
:10155000CDE9036502F044F907B0F0BDD0120020D8
:10156000003802400010024000180240000C024007
:1015700000140240001C02400008024008B535F08B
:1015800055FB34F097FB34F0C5FBFCE708B5044A83
:101590000021044807F01CFC034B186008BD00BF85
:1015A00038EB05087D150008081300202DE9F04FE1
:1015B00091B014220021DFF840A30BA8C74F55F0CB
:1015C000CBF9C74B504620211A6B0024C54E02258B
:1015D00042F01002DFF824934FF0030BDFF8208372
:1015E0001A631A6B02F010020092009A1A6B42F012
:1015F00040021A631A6B02F040020192019A1A6BC0
:1016000042F002021A631A6B02F002020292029A7C
:101610001A6B42F008021A631A6B02F00802039276
:10162000039A1A6B42F004021A631A6B02F0040266
:101630000492049A1A6B42F001021A631A6B02F0C8
:1016400001020592059A1A6B42F400721A631A6B32
:1016500002F400720692069A1A6B42F480721A63C0
:101660001A6B02F480720792079A1A6B42F4806236
:101670001A631A6B02F480620892089A1A6B42F09D
:1016800020021A631A6B02F020020992099A1A6B5F
:1016900042F080021A6301221B6B03F080030A935D
:1016A0000A9B02F029FA384600220C2102F024FAA3
:1016B000012208218C4802F01FFA384601224FF41B
:1016C000805102F019FA304600224FF4005102F026
:1016D00013FA48460022C82102F00EFA834A082372
:1016E0000BA910460D94CDE90B3402F079F84FF4B4
:1016F000D0430BA948460D94CDE90B350B23CDE91A
:101700000EB302F06DF843F623430BA97848CDE9F8
:101710000B350A23CDE90D4B0F9302F061F810232E
:101720000BA973480F95CDE90B35CDE90D4402F0B7
:1017300057F880230BA95046CDE90B350823CDE996
:101740000D440F9302F04CF84FF400410123404642
:101750000F93CDE90B150BA9CDE90D4402F040F82C
:10176000624A60210D2310460F93CDE90B150BA99A
:10177000CDE90D4402F034F880230BA95C48CDE993
:101780000B350723CDE90D440F9302F029F84FF4F0
:1017900080530BA957480D94CDE90B3402F020F883
:1017A0004FF4901240230BA950460D94CDE90B3213
:1017B00002F016F8F0230BA93846CDE90B350A23C1
:1017C000CDE90D440F9302F00BF84FF480630BA9A1
:1017D0004846CDE90B350A23CDE90D440F9301F0BE
:1017E000FFFF202201230BA95046CDE90B23CDE9B1
:1017F0000D4401F0F5FF08230BA95046CDE90B3548
:101800000D23CDE90D440F9301F0EAFF012341F2CE
:101810000C013846CDE90B130BA9CDE90D4401F0BD
:10182000DFFF4FF400530BA90D94CDE90B3403F106
:10183000804303F5F433184601F0D2FF012308205A
:101840000BA9CDE90B032848CDE90D4401F0C8FFF1
:101850004FF400730BA94846CDE90B350D23CDE9B4
:101860000D440F9301F0BCFF10230BA950460D94BB
:101870004FF0050ACDE90B3401F0B2FF48F2040144
:1018800030460D94CDE90B140BA901F0A9FF0BA96B
:101890003846CDF83CA0CDE90B55CDE90D4401F01B
:1018A0009FFF4FF4005C01230BA93046CDE90BC329
:1018B000CDE90D4401F094FF4FF4BC410D233046B7
:1018C000CDE90B150BA90F93CDE90D4401F088FF6D
:1018D00001230BA938460F9514E000BF00200240F9
:1018E00000380240001C0240002802400010024064
:1018F0000004024000240240000C02400018024094
:1019000000000240CDE90B35CDE90D4401F068FF40
:101910004FF400730BA94046CDE90B350723CDE901
:101920000D440F9301F05CFF4FF400534FF49012FD
:101930000BA938460D940427CDE90B3201F050FF76
:101940000823C0220BA90F93494B1846CDE90B255C
:10195000CDE90D4B01F044FF10230BA93046CDE932
:101960000B350A23CDE90D4B0F9301F039FF01230D
:10197000C8220BA94846CDE90B23CDE90D4401F05F
:101980002FFF4FF4F8620BA93A480D94CDE90B2BC9
:1019900001F026FF0A230BA90F93354B1846CDE91A
:1019A0000BA5CDE90D4B01F01BFF0B2332220BA938
:1019B0000F932F4B1846CDE90B25CDE90D4B01F0C8
:1019C0000FFF0BA948460D94CDE90B7401F008FFF9
:1019D00086230BA94046CDE90B350B23CDE90D4BF2
:1019E0000F9301F0FDFE01230BA940460D94CDE9B4
:1019F0000B3B01F0F5FE50230BA94046CDE90B351A
:101A00000D23CDE90D440F9301F0EAFE4FF4C07EA3
:101A100012230BA930460F97CDE90BE30123CDE943
:101A20000D3B01F0DDFE28230BA94046CDE90B3527
:101A30000A23CDE90D4B0F9301F0D2FE40230BA9F1
:101A40003046CDE90B350923CDE90D440F9301F064
:101A5000C7FE4FF440430BA90748CDF83CA0CDE9A1
:101A60000B35CDE90D4401F0BBFE11B0BDE8F08FA0
:101A700000080240001402400004024008B5124869
:101A8000124A134BC0E9002300230122C0E90433AA
:101A9000C0E90232C0E90633036202F04EF908B130
:101AA00000F010FA0021084802F06DFB08B100F0C8
:101AB00009FA0021044802F08CFB18B1BDE8084087
:101AC00000F000BA08BD00BF0C1300200054004015
:101AD000FFEAC00010B5A8B004461422002102A8F5
:101AE00054F03AFF8422002107A854F035FF226801
:101AF000174B9A422AD14FF4804307A8079303F06B
:101B000029FE08B100F0DEF9124C4FF440720121B9
:101B10001148236B43F002032363236B03F002039A
:101B20000093009B1223CDE902230023CDE9041387
:101B3000042302A9069301F053FE236C43F400131F
:101B40002364236C03F400130193019B28B010BDA0
:101B5000005400400038024000040240026808B50A
:101B60000A4B9A4210D10A4A4FF480710948136C0B
:101B700023F40013136401F017FF4FF400710548BC
:101B8000BDE8084001F010BF08BD00BF0054004090
:101B9000003802400004024010B58EB0342200210B
:101BA000002401A854F0D8FE2448254B4FF0280CFF
:101BB0004FF0350E40F2152240F235218486046143
:101BC00080F83640C0E900340923C0E905C30B237F
:101BD000C0E907E340F21B13C0E9092340F21D13DB
:101BE000C0E90244C0E90B1302F09EFB08B100F00B
:101BF00069F94FF4887302214FF4C0604FF4F0721A
:101C000001940C93ADF834408DF83640CDE90431A1
:101C1000FF21CDE906140721CDE908014FF040412D
:101C20000648CDE90A12CDE9022401A9002202F0FA
:101C300046FC08B100F046F90EB010BD601300205C
:101C40000068014070B58CB004461422002107A83A
:101C500054F082FE22683E4B9A4276D103F55043FF
:101C600002250E2607A95A6C00243A4842F08062E9
:101C70005A645A6C02F080620192019A1A6B42F027
:101C800010021A631A6B02F010020292029A1A6B87
:101C900042F400721A631A6B02F400720392039A00
:101CA0001A6B42F480621A631A6B02F48062049227
:101CB000049A1A6B42F040021A631A6B02F0400257
:101CC0000592059A1A6B42F480721A631B6B03F437
:101CD00080730693069B1023CDE907350B9601F020
:101CE0007FFD4EF6FF7307A91B480B96CDE907351C
:101CF000CDE9094401F074FDF72307A917480B96B5
:101D0000CDE90735CDE9094401F06AFD4FF4805370
:101D100007A91348CDE907350923CDE909440B93F9
:101D200001F05EFD4FF4464307A90E480B96CDE93E
:101D30000735CDE9094401F053FD5820224605211D
:101D400001F0B4F9582001F0E3F90CB070BD00BF08
:101D500000680140001002400024024000280240B8
:101D6000001802400020024000220023C0E90023A6
:101D7000002383601846704710B594B030220021CC
:101D8000022408A854F0E8FD1422002103A854F00E
:101D9000E3FD03F063F9214B012119201A6C42F095
:101DA00080521A641B6C03F080530193019B1C4BFF
:101DB0001A6842F440421A601B68129403F44043CC
:101DC0000293029B4FF48033CDE908134FF4800354
:101DD000CDE90E434FF4C873CDE91003092308A8D9
:101DE000139303F0F7F908B172B6FEE703F03EF97A
:101DF00008B172B6FEE70F234FF4A05205900621FA
:101E000003A8CDE903344FF48053CDE9062303F052
:101E1000CDFB08B172B6FEE714B010BD0038024029
:101E20000070004000B5A3B08022002102A854F049
:101E300093FD0E4B05204FF0010E01934FF4C0733C
:101E400006930223CDE90730032301A809934FF439
:101E50000033CDE90BE34FF00063209303F07AFCED
:101E600008B172B6FEE723B05DF804FB0800A000DD
:101E700008B501F0D9F8FFF77FFFFFF7D3FFFFF7B1
:101E800095FBFFF775FAFFF79FFAFFF7DDFAFFF70B
:101E9000F5FDFFF781FE00F017F800F0A3F800F061
:101EA000E9F905F051FFFFF771FB06F05DFFFEE772
:101EB0000268034B9A4201D101F0C2B8704700BFDB
:101EC0000010004072B6FEE708B50D4801230D4A28
:101ED00004214FF0180CC0E900231023C0E90213BD
:101EE0004FF48063C0E904C30023C0E906330362F2
:101EF00003F01CF918B1BDE80840FFF7E3BF08BDC7
:101F000008140020001000A0142200212DE9F04147
:101F10008AB004460DEB020054F01EFD22682C4BE3
:101F20009A4251D12B4B0225032409269A6B4FF07C
:101F3000040805A9284842F0020200279A639A6B18
:101F400002F002020192019A1A6B42F010021A6327
:101F50001A6B02F010020292029A1A6B42F002020D
:101F60001A631A6B02F002020392039A1A6B42F090
:101F700008021A631B6B03F008030493049BCDE96A
:101F80000585CDE9084601F02BFC402305A913483F
:101F9000CDE905350A23CDE90774099301F020FC4A
:101FA00005A90E480996CDE90585CDE9077401F02C
:101FB00017FC4FF4605305A909480996CDE905358A
:101FC000CDE9077401F00CFC0AB0BDE8F08100BF58
:101FD000001000A00038024000100240000402403F
:101FE000000C0240054B002205499A61C3E900122A
:101FF000C3E90222C3E90422704700BF5414002041
:10200000002C014070B588B004461422002103A8BA
:1020100054F0A2FC22681E4B9A4236D103F5863357
:102020000C24022603255A6C0DEB0401194842F4D6
:1020300000625A645A6C02F400620092009A1A6BB1
:1020400042F004021A631A6B02F004020192019A30
:102050001A6B42F008021A631B6B03F00803029329
:10206000029B4FF4F853CDE90654CDE9033601F055
:10207000B7FB04230DEB040107480794CDE90336B1
:102080000023CDE9053501F0ABFB08B070BD00BF02
:10209000002C014000080240000C02400D4B82B0B1
:1020A0000F216FF001001A6C42F080521A641A6C12
:1020B00002F080520092009A5A6C42F480425A64B4
:1020C00000225B6C03F480430193019B02B000F09B
:1020D000EDBF00BF00380240214B1A6C42F01002E5
:1020E00070B51A6488B01B6C054601A903A803F0FB
:1020F00010030293029B03F00FFB069B4BBB03F004
:10210000FBFA184E184B336040F2E733F360174B7D
:10211000B0FBF3F3013B3046736000233361B360DF
:10212000B36104F0B1FB044680B9304604F054FAC0
:10213000044658B9362000F0EBFF0F2D0DD822468B
:102140002946362000F0B2FF094B1D60204608B03A
:1021500070BD03F0D1FA4000D3E70124F6E700BFD9
:1021600000380240D81400200010004040420F0008
:1021700040000020FEE7FEE7FEE7FEE7FEE77047CF
:10218000014804F06BBA00BFD8140020014802F0E7
:10219000C7BB00BF6C8B0220014802F033B900BFFF
:1021A00060130020014801F048BA00BF90120020DF
:1021B0000120704708B553F07BFD162303604FF0F4
:1021C000FF3008BD08B553F073FD16230360FEE72A
:1021D00070B50D4614460E46731B9C4201DC20462A
:1021E00070BDAFF3008006F8010BF5E770B50D4642
:1021F00014460E46731B9C4201DC204670BD16F847
:10220000010BAFF30080F5E74FF0FF3070474FF45C
:10221000005300204B60704701207047002070473A
:102220000B4A0346116810B509B90A4911601068D4
:1022300009490A4C0344091B8B4206D953F038FD67
:102240000C2303604FF0FF3010BD1360FCE700BFAC
:1022500028150020E8A60220000005200004000048
:10226000034AD2F8883043F47003C2F888307047CC
:1022700000ED00E01022002100B589B00DEB020056
:1022800054F06AFB00231548154A03938360C0E9A4
:1022900000234FF6FF72CDE90133C0E90323C0E903
:1022A000053304F0F1FA08B1FFF70CFE4FF4805348
:1022B00004A90A48049304F021FB08B1FFF702FEC9
:1022C000002301A905480393CDE9013304F0B2FBD3
:1022D00008B1FFF7F7FD09B05DF804FB2C150020ED
:1022E0000000014010B588B004461422002103A864
:1022F00054F032FB2268124B9A421ED103F59C33F4
:1023000003A910485A6C42F001025A645A6C02F058
:1023100001020192019A1A6B42F001021A634FF412
:1023200080721B6B03F001030293029B0223CDE931
:1023300003230123079301F053FA08B010BD00BF37
:102340000000014000000240DFF834D00D480E4983
:102350000E4A002302E0D458C4500433C4188C42FF
:10236000F9D30B4A0B4C002301E013600432A24264
:10237000FBD3FFF775FF54F009F9FFF779FD7047BC
:1023800000000520000000204C120020DC5E070841
:1023900050120020E8A60220FEE770470020704798
:1023A00010B5054CC82000F021FA23781BB900F0C5
:1023B000F3F90123237010BD7A15002013B5002412
:1023C0000221C0B28DF8074000F0FAF98DF807003D
:1023D0009DF8073003F00F038DF807309DF80730A4
:1023E000052B01D98DF807409DF80720034B9DF878
:1023F00007005A7000229A7002B010BD7A150020B2
:102400002DE9F74F2F4D164600230F46AC786A781A
:102410008DF80730A2424DD9092C4ED804EB440365
:102420005B00DBB2191D03F1030B03F1060A053350
:10243000C9B25FFA8BFB5FFA8AFA5FFA83F8C4B21B
:10244000DFF88490204600F0BBF98DF807009DF876
:10245000073059462046A9F8003000F0B1F98DF850
:10246000070051469DF807302046B9F800201B02AE
:1024700003F4706313433B80A9F8003000F0A0F927
:102480008DF8070041469DF807302046A9F8003036
:1024900000F096F98DF807009DF80730B9F8002094
:1024A0001B0203F470631343A9F800303380AB7848
:1024B0000133AB7003B0BDE8F08F98469A469B4657
:1024C0001946BCE77A150020781500200122A421C6
:1024D000C0B200F063B90022A421C0B200F05EB91E
:1024E000FFF7F9BF7047000037B500230F4C0546D2
:1024F0008DF8073023781BB900F04EF901232370C3
:102500000324EDB2013CA821284600F059F914F04B
:10251000FF048DF807009DF80730DBB203D19DF86A
:10252000070003B030BD512BECD1F8E77A1500203D
:10253000002313B50C46C0B201218DF8073000F01E
:102540003FF98DF807009DF80730236002B010BDF9
:102550002DE9F3411D461D4B002416465B788DF88E
:1025600007408B422CD909292DD801EB41014C00A1
:10257000E4B2E11CE71D0834C9B2FFB2E4B25FFA6D
:1025800080F8404600F01CF98DF807009DF80730F0
:102590003946089A40469B09136000F011F98DF8FE
:1025A00007009DF8073021464046336000F008F9E7
:1025B0008DF807009DF80720120902F004022A6036
:1025C00002B0BDE8F08127462146D8E77A15002001
:1025D00070B58AB0054601F0D3FD002840F0968022
:1025E0004B4B00264B4C9D426E610CBF4A4A4B4AF6
:1025F0009D422A604A4AC5E901264FF00102C5E919
:102600000766C5E90326236B43D143F0800380208E
:102610004FF0020C05A92363236B079603F0800398
:102620000193019B1223CDE9050304233D48CDE925
:1026300008C301F0D5F84FF4807305A93948059314
:1026400001F0CEF8236C32460F21482043F40003FA
:102650002364236C03F400030293029B236A43F474
:1026600000032362236A23F40003236200F01EFDAB
:10267000482000F04DFD492032460F2100F016FDA4
:10268000492000F045FD28460AB0BDE8704001F041
:1026900054BB43F002034FF48072022122482363AB
:1026A000236B079603F002030393039B1223CDE9E8
:1026B00005230423CDE9081305A901F091F84FF48F
:1026C000007305A91848059301F08AF8236C324677
:1026D0000F211F2043F400132364236C03F4001321
:1026E0000493049B236A43F400132362236A23F4B4
:1026F0000013236200F0DAFC1F2000F009FD202007
:1027000032460F2100F0D2FC2020BAE70AB070BD9B
:102710008015002000380240005C0040005400405A
:1027200032279140001C02400004024030B54FF4B3
:102730007A7485B005460294BDF824400194089C43
:10274000009401F065FB044628B1284601F046FBE1
:102750002846FFF73DFF204605B030BD30B54FF4A9
:102760007A7485B005460294BDF824400194089C13
:10277000009401F027FC044628B1284601F02EFB06
:102780002846FFF725FF204605B030BD0148FFF77A
:102790001FBF00BF80150020FFF7F8BF1FB58DF8E1
:1027A0000F200DF10F02012300920A46014601930A
:1027B0000248FFF7BBFF05B05DF804FB8015002061
:1027C0001FB500230A460DF10F018DF80F300123CC
:1027D0000091014601930448FFF7C0FF9DF80F00E8
:1027E00005B05DF804FB00BF8015002000F03ABC86
:1027F0002DE9F3471A4C98464FF440330E461746DE
:10280000342163608146174B2046DDF82CA01A68FE
:10281000154B01FB02339D6C0A9B022DE36018BF30
:102820000025124BA560236000F01FFEA0B94946A9
:10283000204600F08DFF78B93B463246514620468F
:10284000CDF8008000F03DFE30B90A21204602B0EC
:10285000BDE8F04700F06EBE02B0BDE8F08700BFF3
:10286000F0150020D41500203016002000B00240E2
:10287000034B34211A68034B01FB0233186E704777
:10288000D415002030160020034B34211A68034B66
:1028900001FB0233586E7047D4150020301600201B
:1028A00070B500258EB00E4604460195FFF7E0FF97
:1028B000CDE90205FFF7E8FFFF234FF4C0620A9657
:1028C000ADF834508DF83650CDE906350723CDE903
:1028D0000405CDE90823FFF7CBFF0B90FFF7D4FFEA
:1028E000224601A90C90084801F0E9FD0C22074B93
:1028F0004FF0FF3154431A195160054991604FF070
:102900007F421A510EB070BD30160020D81500203D
:1029100034000020014B1860704700BFD415002020
:10292000034B0C211A68034B01FB0233986070477C
:10293000D4150020D815002030B50C4B85B00446C6
:102940001D68FFF795FF0390FFF79EFF08490346B8
:1029500034200194039A00FB0511002000902846C2
:10296000C96DFFF745FF05B030BD00BFD41500208D
:10297000301600204B4B4C485A6C42F08062F0B548
:102980005A648FB05A6C02240E2509A902F08062A5
:102990004FF48057454E0092009A1A6B42F40002A1
:1029A0001A631A6B02F400020192019A1A6B42F048
:1029B00010021A631A6B02F010020292029A1A6B4A
:1029C00042F040021A631A6B02F040020392039A2B
:1029D0001A6B42F480721A631A6B02F480720492CA
:1029E000049A1A6B42F400721A631A6B02F40072B2
:1029F0000592059A1A6B42F480621A631A6B02F40C
:102A000080620692069A1A6B42F480721A631A6BFD
:102A100002F480720792079A1A6B42F480621A637A
:102A20001B6B0D9503F480630893089B1023CDE97D
:102A300009340023CDE90B3400F0D2FE092309A9A3
:102A40001B480D93CDE9097400F0CAFE4FF46643AC
:102A500009A930460D95CDE9093400F0C1FE4EF6C6
:102A6000FF7309A913480D95CDE9093400F0B8FEAC
:102A7000F72309A90D950125CDE909340E4C20460F
:102A800000F0AEFE09A9304609970A9500F0A8FEAD
:102A9000082309A92046CDE9093500F0A1FE0FB0B1
:102AA000F0BD00BF0038024000100240002002408C
:102AB0000018024000240240002802400548082374
:102AC0000360C02343610523C3614FF48033C362B5
:102AD00002F040BED816002010B52822224C09234F
:102AE000352140F21B1040F21D1CC4E905230B23C5
:102AF000C4E9071340F215230021C4E9093040F26C
:102B000035232046C4E90B3CFFF7D8FF4FF4F07E95
:102B10004FF488732046C4E918E30023A38684F8A1
:102B20003630C4E90133C4E90333104B236001F0AC
:102B300011FD014610B92046FFF71CFF0A4801F0BD
:102B4000F3FB01224FF48051094800F0D5FF012228
:102B50000821084800F0D0FF00F016F90648FFF7FA
:102B6000DFFE002010BD00BF3016002000680140CD
:102B70000020024000280240340000202DE9F743E5
:102B8000214C0126214D4FF0000810272146814697
:102B90004FF6FF722846CDF80480C4E90067C4E907
:102BA000026803F0E1FC304600F05CFA02232146A3
:102BB0004FF6FF722846C4E90037C4E9026803F003
:102BC000D3FC032321464FF6FF722846C4E90037A1
:102BD0000823C4E9023803F0C7FC4FF40873214608
:102BE0004FF6FF72019304232846A660C4E900371C
:102BF000019BE36003F0B8FC4946284603B0BDE8FA
:102C0000F04303F0D0BC00BF5C170020E8170020A1
:102C1000544B9A6B42F0010270B59A638EB09A6B76
:102C2000064609A9504802F00102504C00250192C5
:102C3000019A1A6B42F480021A631A6B02F4800242
:102C40000292029A1A6B42F004021A631A6B02F0A3
:102C500004020392039A1A6B42F008021A631A6B79
:102C600002F008020492049A1A6B42F010021A63EE
:102C70001A6B02F010020592059A1A6B42F02002BC
:102C80001A631A6B02F020020692069A1A6B42F03F
:102C900040021A631A6B02F040020792079A1A6BFD
:102CA00042F080021A6301221B6B03F08003089339
:102CB000089B0223CDE90A320C930C230D930823C1
:102CC000099300F08DFD4CF2037309A9284809937C
:102CD00000F086FD4FF6837309A92648099300F09A
:102CE0007FFD4FF63F0309A92348099300F078FDC3
:102CF00048F2331309A92148099300F071FD2823F4
:102D000009A91F48099300F06BFD80234FF400715F
:102D10004FF4805025633463E561A663C4E9015331
:102D20004FF48063C4E903134FF48043C4E90503FF
:102D30004FF400332046C4E908350323C4E90A35BB
:102D4000104B236000F0E6FA204600F063FA2A46B2
:102D50000F21382000F0AAF9382000F0D9F90EB080
:102D600070BD00BF003802400008024088170020F4
:102D7000000C024000100240001402400018024003
:102D8000001C02401064024038B5194C0721194B51
:102D90000422194D4FF4006023600223E260AB610E
:102DA000C5E90031C5E90221C5E9043310224023F9
:102DB0000021C4E904234FF48073A162C4E9063101
:102DC0004FF48053C4E908032046C4E90111FFF71A
:102DD0001FFF29462046094C03F0A6FB003818BF08
:102DE0000120207040F20360FFF7C8FE207838BD54
:102DF000E8170020400100A06C1700203C000020D4
:102E00000D4B10B5188070200C4B0D4C19802368A9
:102E1000984763687020984751280BD1094B702060
:102E200008221C60084B1870084B1A70E36898471A
:102E3000002010BD0320FCE74E1800205018002091
:102E40000C000020481800201C1800204C180020FE
:102E5000154B37B50024054601A918780194FFF7F2
:102E600067FB0198182819D008D8102811D0142809
:102E700012D058B10124204603B030BD40280FD0F5
:102E800049280FD01C28F5D1042303E00446A8628A
:102E9000F1E70123AB62EEE70223FBE70323F9E747
:102EA0000523F7E70623F5E71C1800202DE9F04F6E
:102EB000002395B004460793CDE90533534B1A68B8
:102EC000534B1269187890472070B0B108AB04F1E9
:102ED0001605A71CDFF8489102930DF12C0A002378
:102EE000DFF840B10EAE0DF1440803932378039A46
:102EF000934205D82046FFF7ABFF15B0BDE8F08F31
:102F0000424B4246424831461B6800785B6998470D
:102F1000404B1B78012B48D1328802990A80B8F8BF
:102F20000020AAF800201B0706D53388029AAAF8C9
:102F30000030B8F800301380029BD9F8002033F835
:102F400002CB3AF8021B9445DBF80000029393B2DF
:102F500082B28CBFACEB0303A3EB0C0381429BB2A8
:102F60008CBF8A1A521A92B21344052B284B187838
:102F7000C4BFC9F800C0CBF80010702823D1A7F84F
:102F800000C0798107AB05AA0399009306ABFFF750
:102F9000DFFA059B05F8013B069B6B72079B032B31
:102FA00022D8DFE803F01F2D2F31990741BF328867
:102FB0000299C2F580520A805A07B4D5B8F80020A9
:102FC000C2F58052ADE7144BD9F800201B8853435B
:102FD000DBF800201B0B3B80104B1B8853431B0B63
:102FE0007B81CFE701232B71039B023709F1040991
:102FF0000BF1040B0133023608F10208039375E765
:103000000223F0E70323EEE70023ECE74818002053
:103010001C1800204C1800204E18002050180020CA
:10302000201800203418002008B5032000F02CF8E8
:103030000020FFF751F8FFF731F8002008BD00002D
:10304000034A044B11681B780B441360704700BFA0
:10305000541800203D000020014B1868704700BF45
:103060005418002038B50446FFF7F6FF0546631CE8
:103070001EBF044B1B78E418FFF7EEFF431BA3426F
:10308000FAD338BD3D00002007490302CA6803F4A3
:10309000E06322F4E0621204120C134343F0BF63B6
:1030A00043F40033CB60704700ED00E0164B30B5C1
:1030B000DC68C4F30224C4F10705231D042D28BFD6
:1030C0000425062B4FF0FF338CBF033C002403FA8A
:1030D00005F5002803FA04F321EA050122EA0302B8
:1030E00001FA04F141EA02034FEA0313DBB206DB03
:1030F00000F1604000F5614080F8003330BD00F021
:103100000F00024A1354F9E700ED00E014ED00E06F
:10311000002808DB4209012300F01F0003FA00F039
:10312000014B43F82200704700E100E010B504466F
:1031300008B9012010BD437F03F0FF0213B90277E5
:10314000FEF72CF9022363772379E3B92368134A46
:103150005A619A6822F018029A6062792368D2B99B
:103160004FF0FF321A6100209A68616922F0600214
:103170000A43A1699A609A6822F080020A439A6021
:1031800001236377D6E7D4E90212204600F008F85D
:103190000028E2D0CDE72269E4E700BFB71DC104F3
:1031A0001F2310B5013B1CD321FA03F4E407F9D522
:1031B000102A12D004D83AB1082A10D001200BE00E
:1031C000182AFBD1062BF9D800684161836823F0E7
:1031D00018031A438260002010BD072BF3E70F2B62
:1031E000F1E7002AEAD1EFE7036802461820D9B2D6
:1031F0001039B1FBF0F010B5054C5F29205CD065AB
:1032000023F47F7020F0030088BF0430906510BD68
:103210002C06060870B50446FFF71EFF0546002C75
:1032200073D00223226884F83530002384F83430C8
:10323000136823F00103136021680B68D8072FD4AB
:103240000B68334DA0691D40D4E901231343E268A4
:1032500013432269134362691343E269034313432F
:10326000226A1343626A042A43EA050302BFD4E9CF
:103270000B5635432B43042A0B604B6923F007039D
:1032800043EA020333D1A26AE56A13437DB390B9DE
:10329000012A21D032F0020229D1EA0127D51EE00D
:1032A000FFF7DAFE401B0528C6D9202303206365FB
:1032B00084F8350070BDB0F5005F14D1032A16D82C
:1032C00001A050F822F000BFDF3200089B32000856
:1032D000DF320008D9320008B5F1C07F07D14023A2
:1032E00001206365E4E7022AF9D9032AD5D04B61AE
:1032F0002046FFF779FFE26D3F2393408360002073
:103300000123606584F83530D4E70120D2E700BF9F
:103310003F8010F038B5054620B390F83530022BC9
:10332000DCB21DD0036800241A6822F001021A6082
:1033300021221C605C609C60DC601C615A61FFF7AC
:1033400053FFEA6D3F23934083606C6585F83440FA
:1033500085F83540C5E90F44C5E91144C5E9134472
:10336000204638BD0124FBE770B590F83440866DE7
:10337000012C34D00124002580F8344090F83540E9
:10338000012C4FF0020428D180F8354004684565CF
:10339000256825F48025256063608368402B19D15A
:1033A000A260E160C26D3F239340B360236843F0A5
:1033B00016032360636943F080036361036C1BB1F0
:1033C000236843F0080323602368002043F00103CF
:1033D000236070BDA160E260E4E780F83450022011
:1033E000F7E7406D704770B50468049D666C45EA68
:1033F000034306F04046334363644368E263B3F536
:10340000403F30D186681EB1012E03D121F07F41AB
:10341000A16370BD022E01F47F0301F47F45C8B2A1
:1034200007D1DB0CA90ADB0243EA411343EAD001CE
:10343000EEE7032E01F07F420AD1D90CED0A890292
:10344000D30F41EA451141EAD00141EAC331DFE738
:10345000190D2D0B0902130F41EA051141EA101154
:1034600041EA0331D4E7E160D3E710B5044630B355
:1034700090F8393003F0FF021BB980F83820FDF7CF
:10348000C3FF226802236168002084F83930136882
:1034900023F440330B43A1681360536B23F00703FD
:1034A0000B43E1685363136C23F47F5323F03F0312
:1034B0000B4313640123E06384F8393010BD01200D
:1034C000FCE773B590F838500446012D4FF0020523
:1034D0000FD080F839500126069D80F8386000959D
:1034E000FFF781FF2268002013683343136002B0A6
:1034F00070BD2846FBE773B516461A4690F838307B
:1035000004460225012B13D0012380F8395080F89E
:10351000383003685E61079B0093069BFFF763FFEB
:1035200022680020136843F00103136002B070BDED
:103530002846FBE7002373B50193044603680D4654
:103540001B68DB0717D42268D369526A13439E06AF
:1035500006D5FFF781FD064623685A68D20643D593
:103560002368122200209A60012384F8380084F82E
:10357000393002B070BDFFF76FFD064623685A6808
:103580009207E0D45A680192019A12F0210F17D0E5
:10359000019A950603D5E26B42F00202E263019ABA
:1035A000D00703D5E26B42F00102E26321229A6068
:1035B0000423012084F83930002384F83830D8E718
:1035C000691CDCD0FFF748FD801BA84201D8002D04
:1035D000D4D1E36B032043F02003E363002384F89A
:1035E000390084F83830C4E75A680192019A12F021
:1035F000290F16D0019A160703D5E26B42F0040298
:10360000E263019A950603D5E26B42F00202E2639F
:10361000019AD00703D5E26B42F00102E26329224E
:10362000C5E7691C99D0FFF717FD801BA842D0D8C9
:10363000002D91D1CDE770477047036870B55E6883
:1036400004461D68F20714D5E90512D51A6822F45C
:1036500080721A60C26B42F00102C26301229A605A
:10366000042380F83930002380F83830436903B1EF
:103670009847B20616D5AB0414D523681A6822F40D
:1036800000521A6020229A60E36B43F00203E36366
:10369000042384F83930002384F8383063690BB18F
:1036A00020469847300716D5290514D523681A688F
:1036B00022F400621A6008229A60E36B43F004036C
:1036C000E363042384F83930002384F838306369D5
:1036D0000BB12046984772070BD56B0509D52368B7
:1036E00020461A6822F480621A6004229A60FFF76A
:1036F000A2FFB00714D5A90512D523681A6822F4D1
:1037000000721A6002229A60E36BE363012384F87B
:103710003930002384F8383023690BB120469847AC
:10372000F20613D5EB0411D5236820461A6822F45B
:1037300080521A6010229A60E36BE363012384F8DD
:103740003930002384F83830FFF776FF70BD000071
:10375000F0B590F83830012B4FF002032BD080F8F1
:103760003930012200EB01131C4F80F838200E0184
:103770005D6AD3E9074244EA0242093C012C96BF44
:1037800005F07F4342EA05621A430368A9B9596A02
:10379000012C01EA070142EA01025A6282699A6138
:1037A00003D8426A22F07F429A62012380F83930BE
:1037B000002380F838301846F0BDD969012C01EAA1
:1037C000070142EA0102DA6100EB060292691A611E
:1037D000EBD825F07F451D62E7E700BFF0FFFC0056
:1037E0002DE9F74F0023DFF8BC916C4A01240D68E6
:1037F0009C4004EA050CAC4340F0B6804D684FEAAB
:103800004308032605F0030406FA08F6671EF6438C
:10381000012F34D8876807EA060ECF6807FA08F741
:1038200047EA0E078760476827EA0C0EC5F30017C2
:103830009F4047EA0E074760C768022C07EA060E5A
:103840008F6807FA08F747EA0E07C76019D14FEAF1
:10385000D30A03F0070B4FF00F0E00EB8A0A4FEA72
:103860008B0BDAF820700EFA0BFE27EA0E0E0F69AA
:1038700007FA0BF747EA0E07CAF8207001E0032C9D
:10388000DAD1076804FA08F415F4403F06EA07069F
:1038900046EA0406066067D0D9F8444023F00306E0
:1038A00003F003074FF00F0E44F4804406F1804606
:1038B000BF00C9F8444006F59C36D9F8444004F4EA
:1038C00080440194019C0EFA07F4D6F8088028EA97
:1038D000040E334CA0424ED004F58064A0424CD07C
:1038E00004F58064A0424AD004F58064A04248D028
:1038F00004F58064A04246D004F58064A04244D020
:1039000004F58064A04242D004F58064A04240D017
:1039100004F58064A0423ED004F58064A0420CBF50
:1039200009240A24BC40EF0244EA0E04B4606FEAA2
:103930000C06946854BF34404CEA0404AF0294600F
:10394000D46854BF34404CEA0404AF03D4605468D4
:1039500054BF34404CEA0404ED035460146854BF6F
:1039600034404CEA040414600133102B7FF43EAF62
:1039700003B0BDE8F08F0024D4E70124D2E702248D
:10398000D0E70324CEE70424CCE70524CAE70624C5
:10399000C8E70724C6E70824C4E700BF003C01408D
:1039A00000000240003802402DE9F04F00224A4C4E
:1039B000DFF82C91DFF82CA1DFF82CB1012303FAFA
:1039C00002FE3EEA01030EEA01076ED122F0030572
:1039D00002F0030C0F26414B05F180454FEA8C0C99
:1039E000984205F59C3506FA0CF6D5F8088006EAEB
:1039F00008085FD003F5806398425DD003F58063CB
:103A000098425BD003F58063984259D003F58063F8
:103A1000984257D0484557D0504557D0584557D071
:103A200003F58053984255D003F5806398420CBF4C
:103A300009230A2303FA0CF3434513D1236823EA2D
:103A400007032360636823EA07036360E36823EAEC
:103A50000703E360A36823EA0703A360AB6823EAD4
:103A60000603AB6003265300056802F0070C06FA54
:103A700003F30F274FEA8C0C25EA030507FA0CF72E
:103A8000056022FA06F500EB85052E6A26EA07078F
:103A90002F62C56825EA0305C560456825EA0E055D
:103AA0004560856825EA030383600132102A85D1C9
:103AB000BDE8F08F0023BDE70123BBE70223B9E790
:103AC0000323B7E70423B5E70523B3E70623B1E7EC
:103AD0000723AFE70823ADE7003C014000000240A8
:103AE0000014024000180240001C02400369194201
:103AF00014BF0120002070470AB18161704709049A
:103B0000FBE703689A69910701D500229A629A69D6
:103B1000D20703D49A6942F001029A61704700000B
:103B200030B5039DC1F3090104682B43606843EA83
:103B30000243054A0B4342EA555223F0004320EA70
:103B400002000343636030BDFF63FF0303682DE998
:103B5000F0419C6905460F46164614F0100470D0DB
:103B600000241022A046DA612B689A69920662D47A
:103B7000B8F1000F36D044F0040401202B689A6994
:103B8000D60505D54FF4807144F001040120D961B8
:103B9000510505D54FF4806144F008040120D96136
:103BA000920550D54FF4007244F00204DA612846C1
:103BB000FFF7A7FF2A680120536823F0FF7323F45F
:103BC0008B3323F4FF7323F0010353606B6C1C43AE
:103BD00020236C6485F84130002385F8423085F855
:103BE000403032E07A1CC0D0FFF736FA801BB84272
:103BF00001D8002FB8D12B68596895F842209869F0
:103C0000D2B200040AD5480408D4202A06D05A6843
:103C100042F480425A60FFF71FFA06462B689B6900
:103C20009906A1D4FFF718FA801B1928F6D9202489
:103C30004FF0010898E7B8F1000F9CD12022DA611B
:103C400099E720469AE70028B1D1BDE8F08170B528
:103C500004460D46164623689B699B0701D5002044
:103C600070BD324629462046FFF770FFA0B96A1C96
:103C7000F1D0FFF7F1F9801BA84201D8002DEAD15D
:103C8000636C43F020036364202384F841300023F5
:103C900084F8423084F840300120E1E72DE9F0411A
:103CA000069F0446884616461D462268936938EAF0
:103CB00003030CBF01230023B34201D0002015E011
:103CC0006B1CF3D0FFF7C8F9C01BA84201D8002D28
:103CD000EBD1636C012043F020036364202384F85C
:103CE0004130002384F8423084F84030BDE8F08150
:103CF00070B504460D46164623689B699B0601D5A0
:103D0000002070BD324629462046FFF71FFF90B9BC
:103D1000FFF7A2F9801BA84201D8002DECD1636CFB
:103D200043F020036364202384F84130002384F8A7
:103D3000423084F840300120E3E710B50446002803
:103D40004AD090F8413003F0FF021BB980F84020C0
:103D5000FDF7C0FE242384F8413023681A6822F05E
:103D600001021A60626822F070621A619A6822F495
:103D700000429A60D4E90221012924D142F4004290
:103D80009A605A68002042F0007242F400425A6081
:103D9000DA6822F40042DA60D4E904210A43A16916
:103DA00042EA0122DA60D4E907210A431A601A685C
:103DB00042F001021A602023606484F841302063DD
:103DC00084F8420010BD42F4044202299A60D8D11E
:103DD0004FF400625A60D4E70120F3E710B50446BF
:103DE00098B10268242380F84130136823F001035E
:103DF0001360FDF7B3FE0020606484F8400084F88F
:103E00004100206384F8420010BD0120FCE700005F
:103E10002DE9F74F994690F8413004460F46202B84
:103E20001646BDF834A0DDF8388040F0C6800C9B03
:103E300013B1BAF1000F06D14FF40073636401208F
:103E400003B0BDE8F08F90F84030012B00F0B58052
:103E50004FF0010B80F840B0FFF7FEF8192305463C
:103E600000905A464FF400412046FFF717FF002804
:103E7000E5D121235FFA89F23946606384F8413045
:103E8000402384F842300C9B6064204663624C4BB4
:103E9000A4F82AA000934FF08073FFF741FE2A4652
:103EA00041462046FFF7D3FE18BBB9F1010F236846
:103EB00015D1F6B20022802120469E62434600952D
:103EC000FFF7ECFEA8B9638D9BB2FF2B15D8628D6E
:103ED0004FF00073009092B22285D2B212E0320A03
:103EE000414620469A622A46FFF7B1FE08B9236888
:103EF000DFE7002384F84030A1E7FF224FF0807312
:103F00000090228539462046FFF70AFE2A464146A0
:103F10002046FFF79CFE002891D1636A226813F8BF
:103F2000011B91626362638D228D013B013A9BB25A
:103F300092B26385638D22859BB2B3B1AAB9434621
:103F4000802120460095FFF7A9FE00287FF477AF77
:103F5000638D9BB2FF2B28D9FF224FF08073009016
:103F6000228539462046FFF7DBFD638D9BB2002B8F
:103F7000CCD12A4641462046FFF7BAFE00287FF4FE
:103F80005EAF23682021D9615A6822F0FF7222F4C3
:103F90008B3222F4FF7222F001025A6084F8411041
:103FA00084F8400084F842004AE7628D4FF00073C5
:103FB000009092B22285D2B2D3E7022040E700BF40
:103FC000002000802DE9F74F994690F841300446D3
:103FD0000F46202B1646BDF834A0DDF8388040F09F
:103FE000C9800C9B13B1BAF1000F06D14FF40073D6
:103FF0006364012003B0BDE8F08F90F84030012BDE
:1040000000F0B8804FF0010B80F840B0FFF724F8C3
:104010001923054600905A464FF400412046FFF709
:104020003DFE0028E5D122235FFA89F2394660631C
:1040300084F84130402384F842300C9B6064636212
:104040004D4BA4F82AA0009303462046FFF768FDD5
:104050002A4641462046FFF7FAFD20BBB9F1010F81
:10406000236816D1F6B20022402120469E624346C4
:104070000095FFF713FEB0B9638D9BB2FF2B3F4B4A
:1040800015D8628D00934FF0007392B22285D2B2A0
:1040900012E0320A414620469A622A46FFF7D7FDCF
:1040A00008B92368DEE7002384F84030A1E7FF2247
:1040B00000934FF08073228539462046FFF730FD8C
:1040C00043460022042120460095FFF7E7FD002823
:1040D0008FD123685A6A636A1A70636A228D01332A
:1040E000013A6362638D92B2013B22859BB2638584
:1040F000638D9BB2B3B1AAB9434680212046009597
:10410000FFF7CCFD00287FF474AF638D9BB2FF2BCB
:1041100028D9FF224FF0807300902285394620462F
:10412000FFF7FEFC638D9BB2002BC9D12A464146A6
:104130002046FFF7DDFD00287FF45BAF23682021D8
:10414000D9615A6822F0FF7222F48B3222F4FF7296
:1041500022F001025A6084F8411084F8400084F88B
:10416000420047E7628D4FF00073009092B22285C3
:10417000D2B2D3E702203DE7002000800024008077
:1041800090F84100704710B590F84130202BDCB218
:104190001DD190F84030012B19D0242380F84130F4
:1041A00003681A6822F001021A601A6822F4805229
:1041B0001A601A68114319601A6842F001021A6005
:1041C000002380F8414080F84030184610BD02209E
:1041D000FCE710B590F84130202BDCB21CD190F8F0
:1041E0004030012B18D0242380F8413003681A682E
:1041F00022F001021A601A6822F4706242EA012178
:1042000019601A6842F001021A60002380F84140E8
:1042100080F84030184610BD0220FCE7D20100684B
:10422000D1F800C0843283182DE9F043C6680CF140
:1042300001075D684FF0000E4C68C6F30B4605F4AD
:104240007045D1F8189026445D60C568C5F30B45EC
:104250003D4445EA0645CE685D60C568C5F30A057C
:104260002E449D6805F470459D608D68C7680135D2
:10427000C7F30A073D4445EA06450E699D601D697E
:1042800025F007051D611E619D6991F8327091F856
:104290003180C3F818E091F8305045EA096545EAE5
:1042A000082545EA07459D615D6925F0FF055D61CB
:1042B0004D695D61DD6925F4E06525F00705DD6187
:1042C000D1E907573D43DD619D6A4D6AC3F828E097
:1042D0009D621EB3012E23D0B51E022D22D9072EBA
:1042E0000CBF02250125DE6AA4EB0C0406F0E026D3
:1042F0006C43DE6203348E6AC96A6E4344EA064444
:10430000DC621C6B24F4FF6424F007041C63196353
:10431000835843F001038350BDE8F0830425E2E7AE
:104320000325E0E70225DEE738B50446002863D020
:1043300090F8A13003F0FF021BB980F8A020FDF730
:1043400081FC022384F8A13023689A6922F070422C
:104350009A619969D4E901200243E0680243206927
:10436000024360690A4325499A619A680A409A6043
:104370009A6842EA0042A0690243E0699A60DA68FA
:104380000A40DA60DA6842EA0042206A0243606A60
:10439000DA601A690A401A611A6942EA0042A06AA0
:1043A00002431A615A6911405961E16A5A6942EA45
:1043B0000142216B0A435A61D96A94F8360001F030
:1043C0007F4194F83550D962D96A94F834200A4371
:1043D00042EA052242EA00420020DA625A6B42F0C9
:1043E00006025A639A6942F001029A610123C4F8F5
:1043F000A40084F8A13038BD0120FCE700F800F0EB
:1044000070477047036870B59E6B04465D6B72071A
:1044100014D5690712D55A6B22F004025A6304229C
:10442000DA63D0F8A43043F00103C0F8A4300023CD
:1044300080F8A12080F8A030FFF7E2FFB20716D580
:10444000AB0714D5236820465A6B22F002025A6348
:104450000222DA63D4F8A4301343C4F8A43004234E
:1044600084F8A130002384F8A030FFF7C9FFF007DB
:1044700010D5E9070ED5236820465A6B22F00102B9
:104480005A630122DA63002384F8A12084F8A03063
:1044900030F032FE320711D52B070FD523682046A6
:1044A0005A6B22F008025A630822DA63012384F867
:1044B000A130002384F8A030FFF7A3FF70BD2DE9E1
:1044C000F04190F8A03006460F469446012B4FF07D
:1044D00002001FD034244FF001080D4686F8A100D9
:1044E00004FB026486F8A08038340FCD0FC40FCDD2
:1044F0000FC40FCD0FC42B68304662463946236087
:10450000FFF78CFE33680020C3F8248086F8A18072
:1045100086F8A000BDE8F08190F8A030012B4FF0A4
:10452000020312D080F8A13003685A6B22F0010216
:104530005A63074A11645A6B42F001025A6301231D
:1045400080F8A130002380F8A0301846704700BFE3
:104550000068014090F8A1007047F0B504468BB0A8
:1045600060B390F8BD34056803F0FF021BB980F812
:10457000BC2432F03FFC03236E46271D84F8BD3473
:10458000EB6B254613F4807355F8100B08BF2361BD
:1045900002F03AFF0FCD0FC60FCD0FC695E803000E
:1045A000254686E8030097E80E0055F8100B02F048
:1045B00079FE064620B1022384F8BD34012552E07D
:1045C0000146206802F026FF3046D4F804C02426B5
:1045D0004FF0010E0146C2B2013094451BD80023B2
:1045E00024261946D8B20133844522D86E460FCD11
:1045F0000FC60FCD0FC695E8030086E8030097E8C5
:104600000E00206802F086FF01230546F0B1022269
:1046100084F8BD24D2E706FB024383F83DE083F82B
:104620003C20A3F8442083F840105965C3E91211D7
:10463000D1E706FB004282F87D1282F87C0282F804
:104640008012C2F89412C2E9A211CBE784F83800B4
:1046500084F8BD34636A012B02D1204600F0EAFCE5
:10466000206803F0F9FA28460BB0F0BD10B590F8B9
:10467000BC340446012B0CD0012380F8BC34006804
:1046800002F0BCFE206803F0D9FA002084F8BC04D4
:1046900010BD0220FCE710B590F8BC240446012AA6
:1046A0000BD0012280F8381080F8BC24006803F099
:1046B000B5FA002084F8BC0410BD0220FCE770B5F8
:1046C00001F00F0611F0800F05464FF0240006EBB5
:1046D000C6044FEA84041FD004F13C0100FB0650DD
:1046E0000124294480F83D40CA604A780E700B715D
:1046F00002B10E81022B04BF00234B7195F8BC342C
:10470000012B12D00123286885F8BC3402F0C3FFC6
:10471000002085F8BC0470BD04F51F7100FB065035
:104720000024294480F87D42DEE70220F3E710B53B
:10473000044601F00F0011F0800F4FF0240200EB4F
:10474000C0034FEA830316D003F13C0102FB004291
:104750000123214482F83D30087094F8BC34012BC9
:1047600012D00123206884F8BC3402F0D3FF00206B
:1047700084F8BC0410BD03F51F7102FB0042002346
:10478000214482F87D32E7E70220F3E738B501F0F3
:104790000F05242404FB050104FB050401F51F712A
:1047A000C4F894320023C4F88C22C4F89C3284F8F4
:1047B0007D3284F87C5203690068012B08BFC4F87D
:1047C0009022DAB21DB902F0FBFF002038BD03F0E1
:1047D000C7F8FAE701F00F01242303FB0100D0F82A
:1047E0009C02704738B501F00F05242404FB050135
:1047F00004FB05043C3163650023E264E3650123A7
:1048000084F83C5084F83D3003690068012B08BFF0
:104810002265DAB21DB902F0D3FF002038BD03F0E3
:104820009FF8FAE738B501F00F05436804469D424A
:104830002CD811F0800F4FF024001ED000FB054152
:10484000012300FB05423C3182F83D3001230D700D
:104850008B7094F8BC249A421AD0206884F8BC3437
:1048600003F088F92DB904F2C442217C206803F0DA
:1048700045FA002084F8BC0438BD00FB01431A4609
:1048800003F51F71002382F87D32DFE70120F3E793
:104890000220F1E738B501F00F02436804469A425E
:1048A0002AD802EBC20311F0800F4FF024004FEA28
:1048B000830318D003F13C0100FB02400123214493
:1048C00080F83D3000250A708D7094F8BC34012BBF
:1048D00014D00123206884F8BC3403F076F928460C
:1048E00084F8BC5438BD03F51F7100FB024000235F
:1048F000214480F87D32E5E70120F3E70220F1E76B
:1049000001F00F030A0603EBC3034FEA83034CBF16
:1049100003F13C0103F51F710144006802F0CABFB6
:104920002DE9F04F066889B00446304603F0D1F90E
:104930000390002840F06F81206803F09BF9002865
:1049400000F06981D6F8083806F500652068C3F3E1
:104950000D23C4F8FC3403F08DF9810704D52268D7
:10496000536903F002035361206803F083F9C20620
:104970002CD52268936923F010039361D6F8208028
:10498000C8F3434308F00F07022B40F0478147F676
:10499000F07318EA030F14D02423C8F30A19304621
:1049A00003FB07474A46D7F88C1203F0C3F8D7F841
:1049B0008C324B44C7F88C32D7F89C324B44C7F842
:1049C0009C322268936943F010039361206803F0DE
:1049D00051F9030300F13481206803F04BF94703D8
:1049E0000CD5274606F5106A4FF00009206803F041
:1049F0004DF90490049B002B40F0EA81206803F0FD
:104A000039F9002813DA6B6823F001036B6094F81E
:104A1000F434012B40F085820021204684F8F41400
:104A200032F0CCFA2268536903F0004353612068E6
:104A300003F020F900050AD5AB68D90702D5204656
:104A400032F04AFA2268536903F400635361206824
:104A500003F010F9020114D523685A6902F00062CC
:104A60005A6194F8F424002A40F05F820121204624
:104A700084F8F4145B6DC3F38303C4F8F83432F0A4
:104A80009DFA206803F0F6F8C30433D56B68102153
:104A9000206823F001036B6002F0EAFC06F5106366
:104AA0004FF67F3162680398824200F24782EB69D9
:104AB00043F00113EB61236B002B00F05982D5F812
:104AC000843043F00B03C5F884306B6C43F00B0368
:104AD0006B64D6F8003804F2C442217C23F4FE63F0
:104AE0002068C6F8003803F009F92268536903F416
:104AF00080535361206803F0BDF8870416D5206801
:104B000003F0EBF8206802F0BBFD2768E06000F0DE
:104B1000EDFD227B0146384602F000FC204632F0D3
:104B2000C8F92268536903F400535361206803F005
:104B3000A1F8000707D5204632F0B7F9226853697B
:104B400003F008035361206803F094F8010600F1B4
:104B50001A82206803F08EF8C2020CD5A04606F532
:104B6000126901276368BB4200F2268222685369FA
:104B700003F480135361206803F07CF883022DD581
:104B8000D4F804E0234606F5326001218E4520D991
:104B900093F8A4C20268BCF1010F40F02382002AFE
:104BA00080F22082D4F8FC7402F4803207F001070E
:104BB000BA4240F0178283F8A3C2B26942F0800281
:104BC000B2617269170600F10D826B6843F40073DD
:104BD0006B602268536903F400135361206803F08B
:104BE00049F8410007D5204632F09AF92268536906
:104BF00003F080435361206803F03CF842070AD574
:104C000023685D686B0702D5204632F08DF9226873
:104C100053682B43536009B0BDE8F08F062B7FF437
:104C2000D0AE082204F2C4413046C8F30A1802F09C
:104C300081FF242303FB0747D7F89C324344BEE699
:104C400006F53068A2460027206803F017F80490A4
:104C5000049B002B3FF4C0AE049BD80776D55FFAC7
:104C600087FB2068594603F019F810F0010F8146C0
:104C70001CD0012320682169C8F8083000F5306392
:104C80000129D0F840C003EB47139A6840F08B80AD
:104C9000110707D5A7498C4508D9100406D54FF44C
:104CA000004202E091065AD520229A6019F0080FBE
:104CB00021D008239F48C8F8083023681A6C03F5F0
:104CC0003063824203EB4713996804D9090402D583
:104CD0004FF4004199602046059232F0CFF8954B91
:104CE000059A9A4207D92169012904D104F2C442E4
:104CF000206803F003F819F0100F02D01023C8F851
:104D0000083019F0020F14D073691A0603D56B68C6
:104D100043F480636B609AF87F32012B06D1002345
:104D2000594620468AF87F3232F0F2F80223C8F85A
:104D3000083019F0200F02D02023C8F8083019F4E9
:104D4000005F03D04FF40053C8F80830049B0137CC
:104D500008F120080AF1240A5B08049378E712F0AE
:104D6000280FA3D173498C4501D9120497D41A692D
:104D7000DAF89832C2F312029B1ACAF89C326FB961
:104D8000D4F894222AB904F2C442012102F0B6FFF9
:104D900004E0D4F88C221344C4F88C3259462046DF
:104DA00032F072F882E764498C4507D111043FF56F
:104DB00076AF9006F2D520229A60EFE7002FEDD172
:104DC000D4F89432002BE9D104F2C4423946DDE72D
:104DD000049BDB0740F19C805FFA89FB2068594601
:104DE00002F065FF10F0010F804620D0012109F08C
:104DF0000F026B6B01FA02F223EA02036B630B46AC
:104E0000CAF80810216999420DD1D7E91223134439
:104E1000FB64B9F1000F06D1636D23B904F2C442FB
:104E2000206802F06BFF5946204632F036F818F041
:104E3000080F02D00823CAF8083018F0100F02D06B
:104E40001023CAF8083018F0400F02D04023CAF8E7
:104E5000083018F0020F12D04946304602F008FB25
:104E600097F83F30012B07D14FF0000359462046F9
:104E700087F83F3032F050F80223CAF8083018F0B3
:104E8000800F45D0FA6D7B6D9A4241D89B1ABA6C5F
:104E900021689342059128BF134603339B0806936C
:104EA00001F5106303EB49130793079B0698996973
:104EB000FA6D89B27B6D814228D39A420CD3059B4F
:104EC00009F00F010120D3F8342800FA01F122EA99
:104ED0000102C3F834281BE0A3EB0208BB6C5A465E
:104EE0000598984528BF984608F103039B08069348
:104EF000237C00931FFA88F3F96C02F01DFDFB6C14
:104F00004344FB64FB6D4344FB65CEE79A42D6D233
:104F1000049B09F1010924370AF1200A5B08049374
:104F200068E5204631F0F0FF7CE5204631F0D4FF03
:104F3000A7E500BF0A30544F0A31544F996020331F
:104F400053F8202C22F4001243F8202CC3F8E81167
:104F5000D3F8E02122F40012C3F8E021D3F8E021D5
:104F600042F00062C3F8E021039A0132039299E50E
:104F70006B6943F4005343F02B036B612B6943F0DF
:104F80000B032B61A5E5B369012704F27F284FF0DD
:104F9000240923F08003B3616368BB427FF6D9AD77
:104FA00009FB07F318F80330012B03D1F9B22046AF
:104FB000FFF7A6FC0137EFE798F86430D9F8002036
:104FC000012B09D1002A07DA67F07F01204688F813
:104FD0006330C9B2FFF794FC013708F1240809F1E6
:104FE0002009BFE5013124332030CFE500681204E9
:104FF00070B5446A19B922438262002070BD836A89
:105000004D1E04EB134400235E1CDBB29D4205D809
:105010003F31224300EB81004260EEE7403300EB7A
:1050200083035B6804EB13443346EDE70368002019
:105030005962704702680021012380F8F414C0F817
:1050400000350846936943F000639361536D43F064
:10505000805343F00303536570470000024A13680E
:1050600043F480731360704700700040194B37B5EC
:105070001A6C194C42F080521A641B6C03F0805376
:105080000193019B236843F480332360FDF7E4FF21
:1050900005466368DA030CD523680F4D43F40033EB
:1050A0002360FDF7D9FF04466B689B030AD50020F7
:1050B00006E0FDF7D1FF401BB0F57A7FE9D9032068
:1050C00003B030BDFDF7C8FF001BB0F57A7FEBD908
:1050D000F5E700BF00380240007000402DE9F041C4
:1050E000DDF8188004460E4615461F462268936870
:1050F000334214BF01230023AB4201D1002012E050
:10510000B8F1FF3FF3D0FDF7A7FFC01B404502D821
:10511000B8F1000FEAD10423012084F84130636C18
:1051200043F001036364BDE8F081000030B504463C
:1051300085B0FDF791FF0346002C47D094F841203D
:1051400002F0FF014AB90390204684F84010FCF7B2
:10515000DBFE41F28832039BA2642068A1680268EA
:10516000013922F4F85242EA01222021026020464D
:10517000A26C00920022FFF7B1FF10BB2268E56924
:10518000E36811682B43256A21F07F412B43656852
:1051900021F0D00143EA05630B4313605568D4E95D
:1051A00005310B43216943EA0143094929400B4377
:1051B0005360136843F0010313600123606484F8B3
:1051C0004130002384F8403005B030BD0120FBE7BA
:1051D000FEF8E0FF2DE9F341044640B30368DB0726
:1051E00010D423689F0764D42368190700F1AA80AC
:1051F00023685A0700F1CB80A269002A40F034816D
:1052000000202BE0964B9A6802F00C02042A07D08B
:105210009A6802F00C02082A0BD15A68560208D587
:105220008F4B1B689D03DCD56368002BD9D101200F
:1052300014E06268B2F5803F13D11A6842F48032FC
:105240001A60FDF709FF864E054633689803C8D4F7
:10525000FDF702FF401B6428F7D9032002B0BDE828
:10526000F0817F4D2B6892B923F480332B602B683B
:1052700023F480232B60FDF7EFFE06462B6899038D
:10528000AFD5FDF7E9FE801B6428F7D9E5E7B2F555
:10529000A02F07D143F480232B602B6843F4803385
:1052A0002B60CEE723F480332B602B6823F480231C
:1052B000F6E76B4B9A6812F00C0F07D09A6802F071
:1052C0000C02082A11D15A6852020ED4644A13689B
:1052D0009B0702D5E368012BA9D11368216923F04C
:1052E000F80343EAC10313607EE7E268C2B11A68BB
:1052F0005B4D42F001021A60FDF7AEFE06462B68D8
:105300009F0707D52B68226923F0F80343EAC203FD
:105310002B6069E7FDF7A0FE801B0228EFD99CE710
:105320001A684F4E22F001021A60FDF795FE0546FD
:10533000336898077FF558AFFDF78EFE401B0228B3
:10534000F6D98AE76369464D83B16B6F43F0010379
:105350006B67FDF781FE06466B6F9B073FF548AF15
:10536000FDF77AFE801B0228F6D976E76B6F23F0F3
:1053700001036B67FDF770FE06466B6F9F077FF5B5
:1053800037AFFDF769FE801B0228F6D965E7344B7D
:105390001A6CD00027D41A6C012742F080521A648C
:1053A0001B6C03F080530193019B2E4D2B68D90594
:1053B0001BD5A3682A4D012B27D12B6F43F0010386
:1053C0002B6741F28838FDF747FE254E0546336FBF
:1053D0009B073FD5002F3FF40FAF214A136C23F0FA
:1053E0008053136408E70027DFE72B6843F48073DA
:1053F0002B60FDF731FE06462B68DA05D9D4FDF7A0
:105400002BFE801B6428F7D927E7ABB92B6F41F23D
:10541000883823F001032B672B6F23F004032B67DD
:10542000FDF71AFE06462B6F9807D3D5FDF714FE3D
:10543000801B4045F7D910E7052B2B6F03D143F0B4
:1054400004032B67B9E723F001032B672B6F23F0CD
:105450000403B5E7FDF700FE401B4045B7D9FCE665
:105460000038024000700040384DAB6803F00C0378
:10547000082B41D02B68022A23F080732B602ED199
:10548000FDF7EAFD06462B68990122D4A36A5B0862
:105490005A1ED4E907310B4343EA0243626A43EAE6
:1054A0008213E26A43EA026343F000536B602B68A5
:1054B00043F080732B60FDF7CFFD244D04462B682D
:1054C0009A013FF59DAEFDF7C7FD001B0228F6D9F6
:1054D000C3E6FDF7C1FD801B0228D4D9BDE6FDF768
:1054E000BBFD04462B689B017FF58AAEFDF7B4FD3A
:1054F000001B0228F6D9B0E6012A6B683FF497AE8C
:1055000003F48002E1698A427FF491AE03F03F0226
:10551000216A8A427FF48BAE47F6C072616A1A40F4
:10552000B2EB811F7FF483AEA26A03F440315208CC
:10553000013AB1EB024F7FF47AAE03F07063E26A96
:10554000B3EB026F3FF45CAE71E600BF003802407F
:10555000134908B58B6803F00C03042B1BD0082BF0
:105560001BD14A684B68496802F03F0213F480037C
:10557000C1F388111ABF0B4800230B48A1FB00019F
:10558000FBF70AFD064B5B68C3F3014301335B0085
:10559000B0FBF3F008BD0348FCE70348FAE700BF9F
:1055A0000038024040787D010024F4002DE9F041EC
:1055B0000D46044610B90120BDE8F081464A136843
:1055C00003F00F038B4228D32268970730D4D0070B
:1055D00044D4414A136803F00F03AB4267D82268F2
:1055E000510770D4130707D53C4A2169936823F407
:1055F000604343EAC1039360FFF7AAFF374B384A81
:105600009B68C3F30313D35CD840364B1860364B0A
:105610001868FCF761FD0020CEE7136823F00F0344
:105620000B431360136803F00F038B42C3D1CBE726
:1056300012F0040F294B03D0996841F4E0519960AE
:10564000160703D5996841F4604199602349A06821
:105650008B6823F0F00303438B60B8E761681F4B4E
:1056600001291A681BD112F4003FA4D09A6841F2B4
:1056700088381A4F22F003020A439A60FDF7ECFCC7
:105680000646BB68626803F00C03B3EB820FA0D040
:10569000FDF7E2FC801B4045F3D903208CE702298B
:1056A00002D112F0007FE0E712F0020FDDE713688D
:1056B00023F00F032B431360136803F00F03AB4277
:1056C0007FF479AF8BE70549E0688B6823F4E053FA
:1056D00003438B6086E700BF003C02400038024075
:1056E0005CEB05080800002040000020014B186812
:1056F000704700BF08000020044B054A9B68C3F3B5
:105700008223D35C034A1068D840704700380240B7
:105710006CEB0508080000200F2303600B4B9A6810
:1057200002F0030242609A6802F0F00282609A6816
:1057300002F4E052C2609B68DB0803F4E0530361AB
:10574000034B1B6803F00F030B60704700380240E7
:10575000003C024003682DE9F74313F001060446BC
:105760000BD0AA4A916821F400019160466B9168C0
:105770003143B6FA86F67609916013F4002512D00B
:10578000A249E56BD1F88C20B5F5801F22F44012B8
:1057900008BF012642EA050216BFB5FA85F50025C5
:1057A0006D09C1F88C20D80210D59848216CD0F82A
:1057B0008C20B1F5800F22F4400242EA0102C0F8C9
:1057C0008C2000F08481002908BF012513F0807F20
:1057D00018BF0126990631D58C4B8D4F1A6C42F0BB
:1057E00080521A641B6C03F080530193019B3B6849
:1057F00043F480733B60FDF72FFC80463B68DA057D
:1058000040F16781814F3B6F13F4407340F06C812E
:10581000236B03F44072B2F5407F7C4A40F08A81EA
:10582000916823F0704021F4F81120F44070014396
:105830009160C3F30B03116F0B4313672368D90601
:105840000CD5724AD2F88C1021F08071C2F88C10FD
:10585000D2F88C10A06B0143C2F88C105A0408D502
:105860006A49606ED1F8902022F440320243C1F8B8
:1058700090201F0408D56549A06ED1F8902022F42D
:1058800040220243C1F89020D80308D55F49E06E5A
:10589000D1F8902022F440120243C1F890209903DD
:1058A00008D55A49206FD1F8902022F440020243D3
:1058B000C1F890205A0608D55449606CD1F8902060
:1058C00022F003020243C1F890201F0608D54F4979
:1058D000A06CD1F8902022F00C020243C1F8902075
:1058E000D80508D54949E06CD1F8902022F0300263
:1058F0000243C1F89020990508D54449206DD1F89C
:10590000902022F0C0020243C1F890205A0508D529
:105910003E49606DD1F8902022F440720243C1F8F4
:1059200090201F0508D53949A06DD1F8902022F4A8
:1059300040620243C1F89020D80408D53349E06D95
:10594000D1F8902022F440520243C1F890209904EB
:1059500008D52E49206ED1F8902022F4404202430F
:10596000C1F890205A0208D52849A06FD1F890209C
:1059700022F080620243C1F890209F020CD5234898
:10598000E16FD0F89020B1F1006F22F0006208BF03
:1059900001250A43C0F8902013F0080F18BF012515
:1059A000580308D51949606FD1F8902022F0407251
:1059B0000243C1F89020190209D51449D4F8800097
:1059C000D1F8902022F080520243C1F89020012E9D
:1059D00000F0B4809A0100F1B180012D75D10B4D1A
:1059E0002B6823F080532B60FDF736FB06462B68AF
:1059F0009F0000F127812268160301D5E36B4BB1AC
:105A0000D00222D5236C03BB04E000BF0038024063
:105A100000700040D5F88830D5F8881003F4403382
:105A200001F0E0410B43616943EA8113A16943EA54
:105A30000163C5F88830D5F88C30A16A23F4F85397
:105A4000013943EA0123C5F88C30910215D5E36F83
:105A5000B3F1006F11D18249D1F88830D1F88800B4
:105A600003F0706300F0E0400343606943EA801391
:105A7000206A43EA0043C1F88830120719D5784AF2
:105A8000D2F88810D2F8883001F0706103F4403306
:105A90000B43616943EA8113E16943EA0173C2F888
:105AA0008830D2F88C30E16A23F440330B43C2F8DB
:105AB0008C306B4C236843F080532360FDF7CCFAA5
:105AC000054623689B0040F1C480002009E00126C0
:105AD0007CE6FDF7C1FAA0EB080064287FF68EAEE5
:105AE000032003B0BDE8F083226B02F440729342BE
:105AF0003FF48EAE3B6F3A6F23F4407342F4803232
:105B00003A673A6F22F480323A673B673B6FDB07B4
:105B10007FF57EAEFDF7A0FA41F2883980463B6FF3
:105B200098073FF575AEFDF797FAA0EB08004845DA
:105B3000F5D9D5E7916821F4F81179E6484E336834
:105B400023F080633360FDF787FA074633681B0153
:105B500072D42268D70712D5636B83B9D6F8843024
:105B6000D6F8841003F4403301F070610B43616890
:105B700043EA8113A16843EA0173C6F8843016032F
:105B800003D5E36BB3F5801F05D0D0021ED5236C7F
:105B9000B3F5800F1AD13249D1F88430D1F884009E
:105BA00003F4403300F0E0400343606843EA8013AD
:105BB000E06843EA0063C1F88430D1F88C00636A7E
:105BC00020F01F00013B0343C1F88C30D10111D5F7
:105BD0002349D1F88430D1F8840003F0706300F0D9
:105BE000E0400343606843EA8013206943EA0043CE
:105BF000C1F8843092010DD5236962681B0443EA21
:105C00008213E26843EA0263A26843EA0273144A19
:105C1000C2F88430124E336843F080633360FDF77E
:105C20001BFA074633681B013FF5D7AEFDF714FAA0
:105C3000C01B6428F6D953E7FDF70EFAC01B642891
:105C400084D94DE7FDF708FA801B64287FF6CFAEB4
:105C500046E7FDF701FA401B64287FF632AF3FE7C5
:105C600000380240836B1A68D36B43F48073D363AC
:105C70007047F0B5054689B00E46FDF7EDF90023F3
:105C8000074608212868CDE9003301F0B3F804463F
:105C9000D8B9296D2868090401F056F90446A0B95D
:105CA0004FF0FF320823302106902868CDE9022307
:105CB0000223CDE90413012302A9079300F0D1FFC9
:105CC000286801F071F9044690B1204609B0F0BD92
:105CD000426B930212D500F0A3FF08AB03EB8403E1
:105CE000013443F8200CFDF7B7F9C01B013023D075
:105CF0002868426B12F02A0FEAD002E0426B91044E
:105D0000F1D4426B120702D508248463DDE7426BAD
:105D1000930701D50224F8E7446B14F0200401D066
:105D20002024F2E7019B40F23A521BBA82633360AF
:105D3000009B1BBA7360C8E74FF00044C5E7000042
:105D40002DE9F041044686B015461F4641B9836BE4
:105D5000012643F000638363304606B0BDE8F0815E
:105D600090F83430012BDEB270D100233A448363C3
:105D7000C06D824204D9A36B43F00073A363EBE7C9
:105D8000D4F800C00322206C4FEA472884F834205E
:105D9000CCF82C30DCF83C2042F49572CCF83C2056
:105DA0002C4A8360C2632C4AC0E91323026813683B
:105DB00023F0C00313600A464FEA98030CF18001F8
:105DC000FDF7D2FA226860B1D36B23F49573D363E5
:105DD000224B9363A36B43F08043A36384F8346046
:105DE000BAE7D36A9021002043F00803D362636CC2
:105DF000012B4FF0FF33CDE900384FF0020318BFFD
:105E00006D02CDE9021301236946CDE90403104672
:105E100000F027FF012F12D982232946206823632F
:105E200001F018F8A0B123680C4A9A63A36B1843D9
:105E30000123A06384F83430002323638CE781239B
:105E400029462068236300F0EDFFEBE7022683E795
:105E5000064681E77B5F0008C9640008FF05400033
:105E60002DE9F041044686B01E46884641B9836B51
:105E7000012743F000638363384606B0BDE8F08134
:105E800090F83430012BDFB26ED100219319816379
:105E9000C06D834204D9A36B43F00073A363EBE7A7
:105EA00020680323314D84F83430C162C36B43F062
:105EB0001A03C363E36BDD632D4DC3E91351636CB8
:105EC000012B18BF5202012E12D9A02311462363C1
:105ED00000F0F0FF0546226880B1264B9363012352
:105EE000A06B0543A56384F8343000232363C3E724
:105EF00090231146236300F0C5FFEBE7D36A7602D7
:105F0000E06B803243F00803016842F8543C4023C0
:105F100083600B6823F0C00343F040030B60B308B9
:105F20004146FDF721FA78B12368DA6B22F01A02B4
:105F3000DA63104A9A63A36B43F08043A36301239F
:105F400084F83430256397E74FF0FF3369462068C3
:105F50002F460495CDE900369023CDE90235012383
:105F6000059300F07EFE87E7022785E7655C000861
:105F7000C9640008FF054000704710B5846B236BAF
:105F8000822B09D1206800F0ADFF28B1A36B184324
:105F9000A0632046FFF7F0FF23682046DA6A22F06C
:105FA0000802DA6240F23A529A63012384F83430EC
:105FB0000023236301F002FF10BD0000436E9A0F1F
:105FC0000A70C3F383624A70C3F301628A70C3F339
:105FD0000742CA70C3F30722DBB20A714B71836EAA
:105FE0001A0DCA80C3F303420A72C3F3C0324A7265
:105FF000C3F380328A72C3F34032CA72C3F30032F1
:106000000A7300224A73426C10B5002A6CD140F624
:10601000FC74C26E04EA830343EA92730B61C2F319
:10602000C2630B75C2F302634B75C2F342538B75A7
:10603000C2F38243C2F3C232CB750A760B690A7E81
:10604000013302F00702023203FA02F242650B7AD0
:1060500003F00F040123A34083655B0A5343C36528
:106060004FF400730366C36EC3F380324A76C3F302
:10607000C61203F07F038A76CB76036F0020DA0F17
:106080000A77C3F341724A77C3F382628A77C3F314
:106090008352CA77C3F3405281F82020C3F30042F1
:1060A00081F8210081F82220C3F3C03281F8232037
:1060B000C3F3803281F82420C3F3403281F82520D5
:1060C000C3F3003281F82620C3F3812281F8272010
:1060D000C3F30122C3F3460381F8282081F8293055
:1060E000012381F82A3010BD012A0FD11B04B0F81A
:1060F0006E2003F47C1313430B610B6901339B0285
:106100004365C3654FF400738365ABE70368054AD5
:106110009A63836B43F080538363012380F83430A8
:106120001846E0E7FF0540002DE9F041002398B054
:1061300004460B93CDE90933CDE9073376230C935D
:106140000AAB93E8070007AB8DE8070020680ECB89
:1061500000F04AFD0546002840F0E38020684368CF
:1061600023F48073436000F05EFD226802205368D0
:1061700043F480735360FCF775FF2068069500F0C8
:1061800083FD054640B9206801F04EF870B12068E3
:10619000A56400F079FD98B1012584F83450A36B13
:1061A0000343A363284618B0BDE8F0810123A3642C
:1061B0000021206800F0C8FE28B14FF08050EBE7C6
:1061C000A36C012BF4D000264FF6FE77DFF85C813C
:1061D00014E03146206800F0B7FE0028DCD14146CB
:1061E000206800F083FF0028E7D13146206800F0E6
:1061F00035FD069B0546C60F01330693069BBB4241
:1062000001D8002EE5D0069BBB420CD8C5F38075A3
:10621000012320686564ADF8163000F008FD28B948
:106220004FF08060B8E74FF08070B5E7636C032BE8
:1062300043D0206800F00EFF0028ADD10146206851
:1062400000F00CFD04216067206800F007FD0821C4
:10625000A067206800F002FD0C21E067206800F0D4
:10626000FDFC636CC4F88000032B26D00DF11601F1
:10627000206800F097FF00288ED1636C2068032B04
:106280001BD0BDF816102165090400F0F8FE0028A7
:1062900082D10146206800F0E1FC0421606620689C
:1062A00000F0DCFC0821A066206800F0D7FC0C217F
:1062B000E066206800F0D2FC20670421206800F02E
:1062C000CDFC0DA9000DE0642046FFF777FE0546E2
:1062D00000287FF472AF226D03462068120400F09C
:1062E0001BFE00287FF458AF04F1100393E8070069
:1062F000231D8DE8070020680ECB00F075FC4FF4DD
:106300000071206800F076FD00283FF44BAF236851
:106310000125054A9A63A36B1843A06384F834509F
:1063200040E701253EE700BFFF054000000010C127
:1063300010B5044608B9012010BD90F8343003F0C0
:10634000FF0213B90277FBF75DFE0323204684F8B2
:106350003430FFF7E9FE0028EDD10123A06320636C
:1063600084F83430E8E7436C0B60836C4B60C36C9B
:106370008B60036DCB60436D0B61836D4B61C36DAF
:106380008B61036E0020CB61704700000323F0B5E2
:1063900080F834308BB0436C04460D46032B02D09A
:1063A000B1F5805F03D1A36B43F080535DE0B1F59D
:1063B000006F006837D10021CDE9041100F04EFCD8
:1063C000800149D404A92046FFF753FC60B9059B1E
:1063D000590344D5216D2068090400F0B5FD18B9B2
:1063E0000221206800F0C8FDA36B1843A063A66BD0
:1063F0002768002E3BD0294B0125BB6384F834501D
:106400004FF40071206800F0F5FC30B123680125DD
:10641000224A9A63A36B1843A0630123284684F899
:1064200034300BB0F0BDE9B9CDE9041100F016FC31
:10643000820111D404A92046FFF71BFC0028D3D108
:10644000059BDB030BD5216D2068090400F07CFD62
:106450000028C9D10146C4E74FF40060C4E74FF0FB
:106460008060C1E7A36B43F00063A363BFE7636889
:106470000493A3680593E368CDE90635636935465F
:106480000893A36909930AAB13E9070004AB8DE8ED
:10649000070038460ECB00F0A7FBB1E7FF05400030
:1064A000016D10B509040446006800F095FD014631
:1064B00028B9206800F0D2FBC0F3432010BDA06BC8
:1064C0000843A0630020F7E710B5846BFCF789FF51
:1064D000022826D0236C5A6DE36B012A5B6D01D034
:1064E000012B1BD1236820460E4A9A63DA6B22F4F3
:1064F0009D72DA63A36B43F08043A363FFF7D0FF81
:106500000538012805D8206800F0ECFCA36B18437F
:10651000A063012384F83430002323632046FFF76F
:106520002BFD10BDFF05400038B50D460446C8B12F
:1065300090F82C3003F0FF021BB980F82D20FAF7F9
:10654000B5FF0223211D206884F82C3000F0BFFA2B
:1065500062682946206800F0F5FA0123002084F8DB
:106560002C3038BD0120FCE770B590F82C30054682
:106570000E46022BD8B210D000F0FB04012C10D133
:106580000223286885F82C3000F012FB3368022BB8
:1065900004D1052385F82C30002070BD85F82C40EF
:1065A000FAE70120F9E738B590F82C300446022BC1
:1065B000D8B20DD094F82C30012BDDB209D10223D2
:1065C000206884F82C3000F005FB002084F82C5063
:1065D00038BD0120FCE7000090F83D30012B33D19D
:1065E000022380F83D300368DA6842F00102DA6085
:1065F000164A93421AD0B3F1804F17D0A2F57C42CD
:10660000934213D002F5806293420FD002F580626C
:1066100093420BD002F57842934207D002F57052B4
:10662000934203D0A2F59432934207D19968084A65
:106630000A40062A06D0B2F5803F03D01A6842F01D
:1066400001021A60002070470120704700000140DD
:1066500007000100704770477047704703681A6968
:10666000910710B504460FD5DA6892070CD56FF084
:1066700002021A61012202779B69990700F0858066
:10668000FFF7E9FF0023237723681A69520710D523
:10669000DA6850070DD56FF0040220461A61022215
:1066A00022779B6913F4407F75D0FFF7D4FF002356
:1066B000237723681A6911070FD5DA6812070CD5FA
:1066C0006FF0080220461A6104222277DB699B07DB
:1066D00067D0FFF7C0FF0023237723681A69D0062D
:1066E00010D5DA68D1060DD56FF0100220461A6178
:1066F00008222277DB6913F4407F58D0FFF7ABFF05
:106700000023237723681A69D20708D5DA68D007EF
:1067100005D56FF0010220461A61FBF7C9FB23681B
:106720001A69110608D5DA68120605D56FF08002DD
:1067300020461A6100F0C9F923681A69D00508D506
:10674000DA68110605D56FF4807220461A6100F0F0
:10675000BDF923681A69520608D5DA68500605D5CE
:106760006FF0400220461A61FFF777FF23681A692D
:10677000910622D5DA6892061FD56FF020022046D6
:106780001A61BDE8104000F09FB9FFF763FF204693
:10679000FFF762FF76E7FFF75DFF2046FFF75CFF3C
:1067A00085E7FFF757FF2046FFF756FF93E7FFF710
:1067B00051FF2046FFF750FFA2E710BD304A0368A3
:1067C000904212D0B0F1804F0FD0A2F57C4290429F
:1067D0000BD002F58062904207D002F580629042B1
:1067E00003D002F57842904219D14A6823F0700331
:1067F0001343234A904229D0B0F1804F26D0A2F50E
:106800007C42904222D002F5806290421ED002F576
:10681000806290421AD002F57842904216D0194A0E
:10682000904213D002F5806290420FD002F5806250
:1068300090420BD0A2F59832904207D002F58062C8
:10684000904203D002F58062904203D123F440735A
:10685000CA6813434A6923F08003134303608B68BB
:10686000C3620B688362064B984203D003F58063D2
:10687000984201D10B69036301234361704700BF54
:10688000000001400040014010B5044650B390F8AC
:106890003D3003F0FF021BB980F83C20FBF722FDDE
:1068A00002232068211D84F83D30FFF787FF012374
:1068B000002084F8483084F83E3084F83F3084F873
:1068C000403084F8413084F8423084F8433084F812
:1068D000443084F8453084F8463084F8473084F8F2
:1068E0003D3010BD0120FCE7114310B5846841EA3A
:1068F000032324F47F442343836010BD70B590F8D4
:106900003C300446012B4FF0020300F08F8001223F
:1069100080F83D30464B80F83C20006885682B406D
:1069200083600B68602B52D033D8402B67D016D8C9
:10693000202B0DD00AD833F0100109D0012384F8A0
:106940003D30002384F83C30104670BD302BF5D12B
:10695000826822F07002134343F0070317E0502BC4
:10696000ECD14A68CE68016A056A21F00A0125F077
:1069700001050A430562836923F0F00343EA061325
:1069800083610262836823F0700343F057038360DE
:1069900011E0B3F5805F0ED0B3F5005F0DD0702B22
:1069A000CCD1CB68D1E90121FFF79EFF2268936823
:1069B00043F0770393600022C0E7CB68D1E901215F
:1069C000FFF792FF2268936843F48043F2E74D6833
:1069D000CE68016A21F0100101628269036A22F423
:1069E000704223F0A00342EA063243EA05138261B3
:1069F0000362836823F0700343F06703C7E74A68C4
:106A0000CE68016A056A21F00A0125F001050A43F2
:106A10000562836923F0F00343EA0613836102628F
:106A2000836823F0700343F04703B0E71A468BE70F
:106A30008800FEFF30B590F83C30012B4FF0020388
:106A40003DD080F83D301F4D0368AB425A689C68CA
:106A500003D005F58065AB4203D122F470024D6886
:106A60002A430D6822F070022A435A60154A934265
:106A70001AD0B3F1804F17D0A2F57C42934213D0C5
:106A800002F5806293420FD002F5806293420BD0F0
:106A900002F57842934207D002F57052934203D038
:106AA000A2F59432934204D1896824F080020A430B
:106AB0009A60012380F83D30002380F83C3018466E
:106AC00030BD00BF000001407047704770472DE99E
:106AD000F0430A68D1F82490D1E90743D1E901587D
:106AE000D1E903ECD1E905762343A2B943EA0902CF
:106AF00001682A4321F4FF4142EA080321F07F01A3
:106B000043EA0E0343EA0C033B4333430B43036066
:106B10000020BDE8F083026843EA090322F4F8424A
:106B20001343036045EA0803426843EA0E0322F474
:106B3000FF4243EA0C0322F07F023B4333431343FB
:106B40004360E5E7CB6803F1FF3C4B69F0B5013BDF
:106B50000F684C688E681B050D69013C8969013E10
:106B6000013D013F0139240136022D04090643EAA3
:106B70000C335AB93B438268234302F070423343DB
:106B80002B430B43134383600020F0BD826822F443
:106B9000700222F470421A4344EA06033B438260C7
:106BA000C2682B4302F070420B431343C360EBE710
:106BB000026910B5D1E90034920D2343CC689205E7
:106BC00043EA442313438A68013A43EA42130361C8
:106BD000002010BD436923F47F5323F03E0343EAB2
:106BE000410141610020704784B010B503AC84E8D6
:106BF0000E000B46049942680B43059922F4FD42AE
:106C00000B43069922F07F020B4307990B43089927
:106C10000B43BDE81040134304B0436000207047AD
:106C2000D0F880007047032303600020704700689D
:106C300000F0030070470B6810B58360C268D1E9AB
:106C4000013422F47F622343CC68096922F00F02E9
:106C500023430B431343C360002010BD143040583E
:106C600070470B6810B543624B688362C26AD1E912
:106C7000023422F0F70223430C69496923430B4392
:106C80001343C362002010BD10B5002386B0044634
:106C900001A9CDE90133CDE903334FF480630593B6
:106CA000FFF7C9FF0A4B4FF4FA521B68B3FBF2F32C
:106CB00041F288325343013B07D3626B1206FAD587
:106CC000C5230020A36306B010BD4FF00040FAE7D3
:106CD00008000020454B10B51B6804464FF4FA50DD
:106CE000B3FBF0F35A43002A49D0636B13F0450F0E
:106CF00007D01B0505D4636B580704D50420A06397
:106D000010BD013AEFE7606B10F0010002D00123E3
:106D1000A363F5E7C523A3632369DBB2994231D1AD
:106D20006369334818400028EAD0002B2CDB5A0056
:106D30002DD49C002DD4D9002DD41A012ED45C0161
:106D40002FD4D90130D41A0231D45C0232D4990242
:106D500033D4DA0234D45C0335D4990336D4DA035D
:106D600037D41C0438D4590439D49A043AD413F0D3
:106D7000080F14BF4FF400004FF48030C0E74FF00D
:106D80000040BDE70120BBE74FF00070B8E74020AE
:106D9000B6E78020B4E74FF48070B1E74FF400709D
:106DA000AEE74FF48060ABE74FF40060A8E74FF424
:106DB0008050A5E74FF40050A2E74FF480409FE7D2
:106DC0004FF400409CE74FF4003099E74FF48020E7
:106DD00096E74FF4002093E74FF4801090E74FF4CC
:106DE00000108DE74FF480008AE700BF0800002004
:106DF00008E0FFFD30B5402387B01025002204468F
:106E0000019101A9CDE902534FF48063CDE9042338
:106E1000FFF711FF41F2883229462046FFF75AFF5B
:106E200007B030BD30B5402387B01125002204469D
:106E3000019101A9CDE902534FF48063CDE9042308
:106E4000FFF7F9FE41F2883229462046FFF742FF5C
:106E500007B030BD30B5402387B01225002204466C
:106E6000019101A9CDE902534FF48063CDE90423D8
:106E7000FFF7E1FE41F2883229462046FFF72AFF5C
:106E800007B030BD30B5402387B018250022044636
:106E9000019101A9CDE902534FF48063CDE90423A8
:106EA000FFF7C9FE41F2883229462046FFF712FF5C
:106EB00007B030BD30B5402387B019250022044605
:106EC000019101A9CDE902534FF48063CDE9042378
:106ED000FFF7B1FE41F2883229462046FFF7FAFE5D
:106EE00007B030BD30B5002387B00C2540220446E2
:106EF00001A9CDE90323CDE901354FF48063059362
:106F0000FFF799FE034A29462046FFF7E3FE07B044
:106F100030BD00BF00E1F50530B5402387B007253F
:106F200004460192002201A9CDE902534FF4806387
:106F3000CDE90423FFF77FFE41F28832294620463F
:106F4000FFF7C8FE07B030BD30B5402387B0372506
:106F500000220446019101A9CDE902534FF4806358
:106F6000CDE90423FFF767FE41F288322946204627
:106F7000FFF7B0FE07B030BD30B5402387B006251F
:106F800000220446019101A9CDE902534FF4806328
:106F9000CDE90423FFF74FFE41F28832294620460F
:106FA000FFF798FE07B030BD30B5002387B033251A
:106FB0004022044601A9CDE90323CDE901354FF470
:106FC00080630593FFF737FE41F288322946204659
:106FD000FFF780FE07B030BD30B5402387B00D25E8
:106FE00000220446019101A9CDE902534FF48063C8
:106FF000CDE90423FFF71FFE41F2883229462046DF
:10700000FFF768FE07B030BD114B4FF4FA5102464E
:107010001B68B3FBF1F341F288314B43013B13D3BF
:10702000516B11F0450FF9D00905F7D4536B5B078D
:1070300002D5042090637047506B10F0010014BF1C
:107040000123C523936370474FF00040704700BF92
:107050000800002010B5002386B00222044601A9D2
:10706000CDE90132C022CDE903234FF480630593BB
:10707000FFF7E1FD2046FFF7C7FF06B010BD10B5D2
:10708000092286B0C023044601910021CDE90223E4
:107090004FF48063CDE9041301A9FFF7CCFD20462E
:1070A000FFF7B2FF06B010BD0F4B4FF4FA51024686
:1070B0001B68B3FBF1F341F288314B43013B0FD323
:1070C000516B11F0450FF9D00905F7D4506B10F052
:1070D000040002D0042090637047C5239363704777
:1070E0004FF00040704700BF0800002041F0004111
:1070F0002922402341F4801110B586B00446CDE921
:10710000022301914FF480630021CDE9041301A90A
:10711000FFF791FD2046FFF7C7FF06B010BD000046
:107120001F4B10B51B6804464FF4FA50B3FBF0F345
:1071300041F288304343013B29D3606B10F0450F87
:10714000F9D00005F7D4636B580702D50420A0637B
:1071500010BD606B10F0010002D00123A363F7E7BC
:107160002369DBB2994215D1C523A363636913F484
:10717000604002D11B0C1380EAE75A040CD413F4CC
:10718000004F14BF4FF480504FF48030E0E74FF0D1
:107190000040DDE70120DBE74FF40050D8E700BFF7
:1071A0000800002030B589B0002303250446019172
:1071B0004021CDE90335CDE905134FF4806303A9E0
:1071C0000793FFF738FD019A29462046FFF7A8FFED
:1071D00009B030BD134B4FF4FA5102461B68B3FBA4
:1071E000F1F341F288314B43013B17D3516B11F05E
:1071F000450FF9D00805F7D4536B590702D5042081
:1072000090637047506B10F0010002D0012393632C
:107210007047536B5B0603D54023F8E74FF00040FF
:10722000704700BF0800002010B54FF4D57286B03B
:10723000082340210446CDE901230023CDE90313AF
:107240004FF4806301A90593FFF7F5FC2046FFF793
:10725000C1FF06B010BD000082B00023104A0193A8
:10726000019B01330193019B934216D80369002BC4
:10727000F6DA00230A4A0193036943F0010303612C
:10728000019B01330193019B934206D8036913F0DC
:107290000103F5D1184602B070470320FBE700BF99
:1072A000400D030084B038B505AD044685E80E00F6
:1072B0000A9B012B26D1836B23F480338363C3683D
:1072C00023F4840323F04003C360C36823F4401312
:1072D000C360119B012B03D1C36843F48013C360C7
:1072E0002046FFF7B9FF089B012B07D1A36843F0A5
:1072F0000603A360A36843F02003A360BDE8384001
:1073000004B07047C36843F04003C360FFF7A4FFB5
:10731000A36B43F48033A363E5E70000022A4AD15C
:10732000274B284A0B44934239D9274B274A0B4411
:10733000934236D9A1F57403254AA3F5105393421D
:1073400031D9A1F18373234AA3F5E74393422CD3A8
:10735000214B224A0B44934229D9214B214A0B4409
:10736000934226D3204B214A0B44934223D3A1F1CD
:10737000B7731F4AA3F5585393421ED31D4B1E4AA1
:107380000B44934234BF07230623C26822F4705291
:10739000C260C26842EA8323C360002070470F23A3
:1073A000F3E70E23F1E70D23EFE70C23EDE70B23C3
:1073B000EBE70A23E9E70923E7E70823E5E700BF4E
:1073C000405327FFFF340C00401E1BFF3F420F00BD
:1073D0007F4F120020D6130060B6E5FE5FE3160073
:1073E00000D3CEFE40771B00C05BB3FEC0912100EE
:1073F00020753800E05459FEE09C4100836843F05A
:107400000103836000207047836823F001038360D9
:107410000020704738B5C3680129054623F0C043F2
:10742000C3600FD1C368002443F00053C360012040
:107430000134FBF717FE6B69D90714D4322CF6D14F
:10744000012038BD0029FBD1C3680C4643F08043BE
:10745000C36001200134FBF705FE6B69DA0702D532
:10746000322CF6D1ECE7A4F1320358425841E8E758
:1074700082B00023104A0193019B01330193019BC9
:10748000934216D80369002BF6DA890100230A4AD1
:1074900041F0200101930161019B01330193019BA4
:1074A000934206D8036913F02003F5D1184602B0C1
:1074B00070470320FBE700BF400D030082B00023AC
:1074C0000F4A0193019B01330193019B934214D80E
:1074D0000369002BF6DA0023094A019310230361A4
:1074E000019B01330193019B934206D8036913F07A
:1074F0001003F5D1184602B070470320FBE700BF28
:10750000400D0300D0F800381943C0F800180020DF
:107510007047000084B02DE9F843044609A80E46E0
:10752000139D80E80E000023194603F14002013349
:1075300004EB82020F2B5160F7D104F50067002D98
:107540006CD17B6843F002037B60A36B23F40013D0
:10755000A363236843F040032360236843F0800360
:1075600023600023C4F8003ED4F80038C4F8003883
:107570000E9B012B59D10B99002954D120464FF66F
:107580007F38FFF7BFFF10212046FFF771FF01464C
:107590002046FFF793FF0843002304F51062C0B2B2
:1075A0004FF0904C19464FF0006E00383B617B6104
:1075B00018BF0120FB61B34239D1002204F53063CA
:1075C0004FF0904C4FF0006E11464FF67F38B242AC
:1075D00040D13B6923F480733B610023A3616FF0CA
:1075E000804363610C9B1BB9A36943F01003A36143
:1075F000A269224B1343A3610F9B1BB1A36943F004
:107600000803A361012D05D1A36943F0804343F032
:107610000403A361BDE8F84304B07047A36B43F4CF
:107620000013A3639DE71946A8E70321A6E7D2F854
:107630000090B9F1000F0BDA3BB9C2F800E011611C
:107640000133C2F808802032B5E7C2F800C0F6E77F
:107650001160F4E7D3F80090B9F1000F0BDA3AB9F2
:10766000C3F800E019610132C3F808802033AEE7A7
:10767000C3F800C0F6E71960F4E700BF00383C80AB
:10768000D0F8083813F0060004D013F0020F14BF2E
:1076900002200F20704730B50D78012400F50062FC
:1076A00005F00F0300EB45109C404B78012BD3698C
:1076B00018D11C43D461D0F800391A0410D4CA6818
:1076C000D0F80049C2F30A030A79234343EA82430C
:1076D00043EA855343F0805343F40043C0F8003934
:1076E000002030BD43EA0444D461D0F8003B1B04C1
:1076F000F6D4CB68D0F8002BC3F30A0313430A79FE
:1077000043EA824343F0805343F40043C0F8003B14
:10771000E6E7000010B50A78497800EB421300F55F
:107720000060012902F00F0222D1D3F800190029CC
:107730000BDAD3F8001941F00061C3F80019D3F84F
:10774000001941F08041C3F800190121C46B01FA0E
:1077500002F224EA0204C463C16921EA0202C2619E
:10776000154AD3F800190A40C3F80029002010BDBB
:10777000D3F8001B00290BDAD3F8001B41F000619D
:10778000C3F8001BD3F8001B41F08041C3F8001B75
:107790004FF48031C46B01FA02F224EA0204C4639C
:1077A000C16921EA0202C261044AD3F8001B0A40FF
:1077B000C3F8002BDAE700BF007833EC0078F3EF72
:1077C0004B78DFF8ECC0012BF0B50E788D6900EB3B
:1077D0004614364F46D104F51063BDB91D692F40DC
:1077E0001F611D6945F400251D611D6905EA0C0531
:1077F000012A1D6123D14A6902B15A61D4F80039C6
:1078000043F00443C4F800390020F0BDD3F810E081
:107810000EEA0C0CC3F810C0D3F810C00CEA07072E
:107820001F61CF68AF421D6945F4002538BF8F61E5
:107830001D618D691F69C5F312053D43D8E7D4F872
:10784000003943F00443C4F800398B69002BDBD0C6
:1078500006F00F060123D0F83428B3401343C0F8D4
:107860003438D1E7D4F8100B04F5306300EA0C008B
:107870001861186938401861C86805B188611D69C8
:10788000012AC861C0F3120045F400251D611D697D
:1078900040EA0500186102D10A6902B15A61D4F8C0
:1078A000003B43F00443C4F8003BADE7FFFF07E0B3
:1078B0000000F8FF002382B04A780193012A0B7878
:1078C0004FEA43131ED100F51060C258C118002AB8
:1078D00002DB002002B07047C25842F00062C25082
:1078E000C25842F08042C25042F21072019B0133F2
:1078F0000193019B934201D90120EBE70B68002B18
:10790000F4DBE6E700F53060C258C118002AE0DA7F
:10791000C25842F00062C250C25842F08042C25087
:1079200042F21072019B01330193019B9342E3D811
:107930000B68002BF6DBCCE710B59DF8084044B986
:10794000033301329B0800EB023001EB83038B42CF
:1079500001D1002010BD51F8042B0260F7E70000B0
:107960002DE9F3414D780F78012D8B6900EB471419
:107970000E79DFF8B4C1DFF8B4E140F08E8004F591
:107980001065D5F810806BBB08EA0C0CC5F810C068
:10799000D5F810C04CF4002CC5F810C0D5F810C0B4
:1079A0000CEA0E0EC5F810E0012A4ED14B6903B166
:1079B0006B61012E0CD1D0F8083813F4807FD4F815
:1079C00000390CBF43F0005343F08053C4F8003932
:1079D000D4F8003943F00443C4F80039002002B061
:1079E000BDE8F08108EA0E0E012EC5F810E0D5F8CA
:1079F00010E00EEA0C0CD1F80CE0C5F810C00EEB4C
:107A0000030CD5F810800CF1FF3CBCFBFEFEDFF848
:107A100020C10CEACE4C4CEA080CC5F810C0C3F3E8
:107A2000120CD5F810E04CEA0E0CC5F810C0BBD112
:107A3000D5F810C02CF0C04CC5F810C0D5F810C057
:107A40004CF0005CC5F810C0AEE7D4F80059012E28
:107A500045F00445C4F800590BD0002BBED007F008
:107A60000F020127D0F8343897401F43C0F834780C
:107A7000B4E7D0F808589BB215F4807FD4F80059C9
:107A80000CBF45F0005545F08055C4F800590092F0
:107A90003A460969FFF750FFA0E7D4F8105B04F5F8
:107AA000306705EA0E053D613D6905EA0C053D615B
:107AB000CD681BBB3B69C5F312051D433D613B69A6
:107AC00043F400233B61012A02D10B6903B17B61BE
:107AD000012E0CD1D0F8083813F4807FD4F8003B85
:107AE0000CBF43F0005343F08053C4F8003BD4F87C
:107AF000003B43F00443C4F8003B6FE72B44DFF83E
:107B000030C0D7F810E0013BB3FBF5F39BB25D4307
:107B10000CEAC34343EA0E03CD61C5F312053B6192
:107B20003B691D433D61CEE7FFFF07E00000F8FF22
:107B30000000F81F0346900802F0030270B500240D
:107B400003F58055844210D301EB800062B103F548
:107B500080531C680023D90024FA01F1C154013379
:107B600099B28A42F7D1104470BD2E6841F8246062
:107B70000134E7E74A780B78012A00EB431012D171
:107B8000D0F80029002A06DB2BB1D0F8003923F009
:107B90008043C0F80039D0F8003943F40013C0F82E
:107BA000003900207047D0F8002B002A06DB2BB1EB
:107BB000D0F8003B23F08043C0F8003BD0F8003BF6
:107BC00043F40013C0F8003BEBE70B784A7800EB76
:107BD00043100B79012AA3F10203DBB20FD1D0F8D5
:107BE0000029012B22F40012C0F8002905D8D0F892
:107BF000003943F08053C0F8003900207047D0F8B6
:107C0000002B012B22F40012C0F8002BF5D8D0F87D
:107C1000003B43F08053C0F8003BEEE7D0F800385B
:107C2000090123F4FE6301F4FE61C0F80038D0F8C6
:107C300000381943C0F8001800207047D0F8003E03
:107C400023F00303C0F8003ED0F8043823F0020309
:107C5000C0F8043800207047D0F8003E23F003033A
:107C6000C0F8003ED0F8043843F00203C0F80438EE
:107C7000002070474269806910407047D0F818387A
:107C800000F50060C0691840000C7047D0F8183843
:107C900000F50060C069184080B2704700EB4111E8
:107CA00000F50060D1F8082B40691040704710B50E
:107CB000D0F81048D0F8343800EB411001F00F0133
:107CC00000F51060CB408068DB01DBB22343184035
:107CD00010BD406900F001007047D0F8003923F46E
:107CE000FF6323F00703C0F80039D0F8043843F4E9
:107CF0008073C0F8043800207047000030B5056C70
:107D000000F530630F4CA54203D9D0F8004B002C8E
:107D100016DB002401291C611C6944F400241C6149
:107D20001C6944F018041C611C6944F0C0441C61C7
:107D300006D15A61D0F8003B43F08023C0F8003BE5
:107D4000002030BD0A30544F08B50349034800F005
:107D5000F7FF034B187008BD5818002034060608BA
:107D60005C18002008B513460A4601460348FDF793
:107D7000E7FF003818BF012008BD00BF54140020E1
:107D800008B513460A4601460348FEF769F800386D
:107D900018BF012008BD00BF5414002008B50348D7
:107DA000FEF77EFB043818BF012008BD54140020E4
:107DB00001460148FEF7D7BA5414002008B500F078
:107DC00013F908BD012307B58DF8073000F01EF840
:107DD00008B98DF807009DF8070003B05DF804FBB3
:107DE00008B5FFF7EFFF01280CD10748FEF7A0FA0E
:107DF00038B94FF400610448FEF7C8FA003818BFDC
:107E0000012008BD0220FCE7541400204FF400516B
:107E1000034808B5FBF76AFEB0FA80F0400908BDD8
:107E200000080240134B30B51C7889B0154614F099
:107E300001041BD1032903D8DFE801F01A060C1254
:107E40000424204609B030BD6846FFF7B1FF069B09
:107E50002B60F6E76846FFF7ABFF079B2B80F0E748
:107E60006846FFF7A5FF079B5B0AF1E70324E8E7F5
:107E70000C46E6E74400002010B50123054C2370B2
:107E8000FFF78CFF18B9237803F0FE0323702078E6
:107E900010BD00BF4400002038B500F085FF47F258
:107EA0002F55044600F080FF031BAB4202D94FF070
:107EB000FF3003E0FFF772FF0028F3D138BD000068
:107EC00030B585B00C4601920093FFF7E5FF00281E
:107ED000DDE9002102DA012005B030BD2046FFF7C0
:107EE0004FFF02460028F6D10E4847F230530DF1FD
:107EF0000E01006801F002F90028ECD1BDF80E3047
:107F0000022BE8D100F050FF47F22F55044600F055
:107F10004BFF031BAB42DED8FFF740FF0028F6D132
:107F2000DAE700BF6018002030B585B00C4601923A
:107F30000093FFF7B1FF0028DDE9002102DA0120FC
:107F400005B030BD2046FFF70DFF02460028F6D1F0
:107F50000E4847F230530DF10E01006801F0CEF8E3
:107F60000028ECD1BDF80E30012BE8D100F01CFF49
:107F700047F22F55044600F017FF031BAB42DED833
:107F8000FFF70CFF0028F6D1DAE700BF60180020E9
:107F900038B5134C0125257000F0D6FE02281DD1FE
:107FA000FFF71EFF50B92570FFF7F8FE18B92378C8
:107FB00003F0FE0323702378DBB223702378012BB8
:107FC0000CD0084D2A684AB902210A2001F00EF8A7
:107FD000286018B9237843F001032370207838BD56
:107FE0004400002060180020012307B5ADF80630DA
:107FF000002305480DF106011A46006801F03CF81F
:1080000003B05DF804FB00BF60180020D0F8D43244
:1080100000EB830010B5D0F8C04284B1D0F8C43270
:108020005BB194F80002FF2807D09B68214694F8C2
:1080300001229847FF2384F80032002000E003204B
:1080400010BD00000A23038000487047C4000020D0
:1080500070B5822106460F4800F094FB01210546C9
:108060000C4800F08FFB812104460A4800F08AFB8F
:108070000DB11022AA711CB140222271002262713E
:1080800018B140220271002242714323014833801B
:1080900070BD00BF80000020FFF7DABF70B58221FD
:1080A00006460F4800F06EFB012105460C4800F023
:1080B00069FB812104460A4800F064FB0DB11022DF
:1080C000AA711CB1002222710222627118B1002231
:1080D00002710222427143230148338070BD00BF08
:1080E0008000002038B5D0F8D4320446B03350F8C0
:1080F00023508DB12EF05DFFC5F80C02D4F8D402E8
:1081000005F5037104EB8004D5F80402D4F8C432F9
:10811000DB689847002038BD0320FCE7F8B5D0F8AD
:10812000D4620A4600EB8606D6F8C05245B301F089
:108130000F0C142707FB0C07BC6994B1D0F8C832A8
:108140004FF0240E0EFB0C339B6CB4FBF3FC03FBD3
:108150001C4434B923462246BC612EF0A2FF2046BF
:108160000DE0D6F8C43200271C69C5F81472002C43
:10817000F5D005F50471D5F80802A0473846F8BDDA
:108180000320FCE7D0F8D43200EB83032DE9F34160
:108190004FF00008D3F8C07205460E468DF80580F2
:1081A000ADF80680002F6ED00A7812F060042ED051
:1081B000202C64D1CC8891F801C00CB3120613D5E1
:1081C000D3F8C4322246394660469B689847F28805
:1081D00039462846072A28BF072200F050FD4446AA
:1081E000204602B0BDE8F081402C394687F800C235
:1081F00028BF4024224687F8014200F055FDEEE7F3
:10820000D3F8C432224660469B689847E8E74F7827
:108210000B2F34D801A353F827F000BF4D8200087C
:10822000E18100087F8200087F8200087F820008C9
:108230007F8200087F8200087F8200087F8200081A
:108240007F820008638200087782000890F89C32E1
:10825000032B14D102220DF106013C4600F00FFD64
:10826000BEE790F89C32032B09D101220DF10501E4
:1082700000F005FDB4E790F89C32032BB0D03146F6
:10828000284600F0D5FC0324AAE700BF38B5044611
:10829000002581212EF0E1FE0121204625872EF0C8
:1082A000DCFE82212046A4F878512EF0D6FED4F8C8
:1082B000D432E56404EB8303D3F8C0228AB1D3F847
:1082C000C4325B689847D4F8D432B03354F82300F2
:1082D0004EF0C8FAD4F8D432B03344F82350C4F87E
:1082E000BC52002038BD70B504464FF407704EF004
:1082F000B1FA054630B9D4F8D432B03344F823008B
:10830000022547E04FF4077200214EF025FBD4F818
:10831000D432B03344F82350237CC4F8BC52002B31
:108320003AD14FF400730222812120462EF089FEBB
:1083300001264FF4007326873146022220462EF094
:1083400080FE102303228221A4F878612046A4F83D
:108350004E3008232EF075FED4F8D43200260121C9
:1083600004EB8303A4F84C10D3F8C432C5F80462BC
:108370001B689847D5F80422C5F81462C5F818623E
:10838000002ABDD0257C012185B94FF40073204619
:108390002EF090FE284670BD012640230222812146
:1083A00020462EF04EFE40232687C5E74023204678
:1083B00035462EF07FFEEDE739B1D0F8D43200EB30
:1083C0008300C0F8C4120020704703207047D0F823
:1083D000D432B03350F823302BB10020C3F8081248
:1083E000C3F81022704703207047D0F8D432B0335E
:1083F00050F823301BB10020C3F80412704703204B
:108400007047D0F8D432B03350F8232010B57AB189
:10841000D2F8144201236CB9C2F814328121D2F887
:108420001032D2F80822C3622EF03BFE204610BD67
:108430000320FCE71846FAE7D0F8D422B03250F80F
:10844000222010B582B1047CD2F8042234B94FF452
:10845000007301212EF02EFE204610BD4023012185
:1084600000242EF027FEF7E70324F5E778B1002378
:10847000C0F8B832C0F8C432C0F8D03209B1C0F880
:10848000B4120123027080F89C322EF051BD0320FB
:108490007047002313B50446ADF8063081B1CB6AAE
:1084A000C0F8B81223B10DF106009847C4F8D00205
:1084B000D4F8D83200200133C4F8D83202B010BD4D
:1084C0000320FBE72EF0B4BDD0F8B8320BB11B6827
:1084D00018471846704708B5D0F8B8325B68984717
:1084E000002818BF032008BD38B500F2AA250446AD
:1084F000284600F092FB012394F8AA12C4F89432A3
:10850000B4F8B032C4F8983201F01F03012B08D040
:10851000022B0CD08BB929462046BDE8384000F02C
:108520004FB929462046BDE8384000F0A7BA294691
:108530002046BDE8384000F0D0BA204601F0800166
:10854000BDE838402EF092BD70B50446164609BB12
:10855000D0F89432032B0CD1D0E9573293420AD988
:108560009B1A31469A42C0F85C3128BF1A4600F087
:10857000A8FB002070BD90F89C32032B06D1D0F8E8
:10858000B8321B6913B1C0F8D4129847204600F0E6
:10859000A0FBEEE790F89C32032BEAD1D0F8B8327A
:1085A0009B69002BE5D00022BDE87040C0F8D422C2
:1085B000184773B504461646002941D1D0F89422D5
:1085C000022A0FD1D0E90752954214D9AA1A019173
:1085D0003146C26100F060FB019B1A4619462046F5
:1085E0002EF068FD94F8A03213B1002384F8A03275
:1085F000002002B070BD0ED1826995420BD8D0F830
:108600009852AA4207D20A46019100F045FB019B0D
:10861000C4F89832E1E794F89C32032B08D1D4F8DF
:10862000B832DB6823B100222046C4F8D422984730
:10863000802120462EF01AFD204600F055FBD1E7A0
:1086400090F89C32032BD3D1D0F8B8325B69002B61
:10865000CED00022C0F8D42202B0BDE87040184746
:10866000F8B501230021044680F89C32D0F8B832D6
:10867000C0F894124160C0F8A41280F8A012B3B9F7
:1086800000260022402501274023114620462EF0D7
:10869000D8FC2B46002280212046A4F86471C4F83F
:1086A00060512EF0CEFC3046A7842562F8BD5B6891
:1086B000002BE5D098470028E2D00326E1E70174BB
:1086C0000020704790F89C32DBB280F89D32042382
:1086D00080F89C320020704790F89C32042B04D123
:1086E00090F89D32DBB280F89C320020704708B5CC
:1086F00090F89C22032A05D1D0F8B83213B1DB6977
:1087000003B19847002008BDD0F8D422AE3250F80B
:10871000222008B542B190F89C32032B02D1136A93
:1087200023B19847002000E0032008BD1846FCE76D
:10873000D0F8D422AE3250F8222008B542B190F8D9
:108740009C32032B02D1536A23B19847002000E0EA
:10875000032008BD1846FCE700207047012208B539
:1087600080F89C22D0F8B8220AB9002008BD5268CF
:10877000017990470028F8D00320F7E700207047E0
:108780000020704710B5428803789A420AD90478CD
:108790002044234444789BB2052CF6D184788C4243
:1087A000F3D110BD0020FCE710B5044680212EF067
:1087B0005DFC00212046BDE810402EF057BC0000B3
:1087C0002DE9F3410D7804460E4605F06005202D95
:1087D00014D0402D12D0002D40F012814F78092F77
:1087E00000F20E81DFE817F013013C010C012B01B0
:1087F0000C018E0016000C01FB00AA00D4F8D43244
:1088000031462046AE3354F823309B6802B0BDE8B1
:10881000F04118470023ADF806304B881A0A013A98
:108820000E2A0DD8DFE802F0132C390C0C59630C1A
:108830000C0C0C0C0C0C0800D0F8B432DB694BB9F2
:108840002046FFF7B1FF284602B0BDE8F081D0F81E
:10885000B4321B680DF10601207C9847F288002A8B
:1088600000F0FA80BDF80630002BE9D09A420146AC
:1088700028BF1A46ADF80620204600F000FAE2E7CD
:10888000027CD0F8B83232B99B6A0DF106009847E5
:1088900002234370E2E7DB6AF7E7DBB2052BCFD8B0
:1088A000DFE803F003070B0F1317D0F8B4325B684F
:1088B000C5E7D0F8B4329B68C1E7D0F8B432DB68C2
:1088C000BDE7D0F8B4321B69B9E7D0F8B4325B69C0
:1088D000B5E7D0F8B4329B69B1E7037C002BAFD188
:1088E000D0F8B8320DF106005B6B9847B6E7037C11
:1088F000002BA5D1D0F8B8320DF106001B6B9847BC
:108900000723C6E78B88002B9AD1CB88002B97D101
:108910004E887F2E94D890F89C32032B90D0F1B2E1
:1089200080F89E122EF0B4FB204600F0D2F91EB162
:10893000022384F89C3286E70123FAE78E784E4FB3
:10894000012E3E7003D9FFF72FFF03257BE790F838
:108950009C32022B5FFA83F809D0B8F1030F18D0CC
:10896000FFF722FF39782046FFF7B5FDEDE7002E2F
:1089700072D001214160FFF7A7FD0546204625B1D1
:10898000FFF712FF84F89C825DE700F0A2F9032351
:10899000CFE75EB902233146466080F89C32FFF78C
:1089A0009AFD204600F095F935464CE741680129CB
:1089B00052D0C9B2FFF78FFD397820466160FFF7CA
:1089C00083FD0646002847D02046FFF7EDFE2179BB
:1089D0002046FFF780FD022384F89C32E4E7CA8832
:1089E000012A7FF42DAF90F89C120229CBB205D852
:1089F00033B10146002341F8083F3DE7032B04D083
:108A000020460025FFF7D0FE1DE7011D34E790F852
:108A10009C32013B022BF3D8CB88022B7FF410AFA2
:108A20000123C360D0F8A4320BB10323C360022238
:108A300004F10C0120463D4600F021F903E74B8884
:108A4000012B02D1C4F8A43206E0022B7FF4F8AE69
:108A50008B881B0A80F8A032204600F03AF9F2E633
:108A600090F89C32013B022BCAD84B88012B7FF433
:108A7000EAAE0023E6E700BF6418002070B50B786B
:108A800004460E4603F06002402A01D05B061FD464
:108A900094F89C32013B022B1AD8317920460129E7
:108AA00017D8FFF76BFE88B9D4F8B8329B686BB162
:108AB000C4F8D4023146204698470546F3881BB9CE
:108AC00015B9204600F005F9284670BD0325F5E7E5
:108AD00020460025FFF768FEF6E770B50B780446E0
:108AE0000D468A8803F060030E79202B53D0402B6B
:108AF00051D063BB4B78012B3BD0032B20D033BB31
:108B000090F89C32022BD9B261D003291FD106F014
:108B10000F0312F0800F4FF0140202FB030367D023
:108B20009B8CA3B106F07F05013505EB850500EBB5
:108B3000850516F07F0367D12B600222294653E09A
:108B400090F89C32022BDAB237D0032A03D02046A9
:108B5000FFF72AFE0BE04B8833B9710604D0EB888F
:108B600013B931462EF082FA204600F0B2F8002008
:108B700070BD90F89C32022BDAB21ED0032AE6D1E7
:108B80004B88002BF3D1730602D031462EF077FAD2
:108B9000204600F09EF831462046FFF7F1FD002800
:108BA000E5D1D4F8B832C4F8D4029B68002BDED0EB
:108BB00029462046BDE8704018477206C7D03146A6
:108BC0002EF054FA802120462EF050FACFE771069D
:108BD000BDD113064FF000034FF002024CBF00F16D
:108BE000140100F5AA710B60204600F048F8BEE7BA
:108BF000B3F86431002BAAD006F07F05142303FBE1
:108C0000050505F5AA7594E7314620462EF0BEF914
:108C100008B1012390E728608FE70B7803704B7849
:108C200043704B8843808B888380CB88C380704798
:108C300010B5044680212EF019FA00212046BDE827
:108C400010402EF013BA30B588B100240138234605
:108C50000134055D002DFAD1DBB201335B001380D6
:108C60000B7003234B70022310F8012F02B930BDA3
:108C7000CA545A1C0233D2B2DBB28D54F4E710B599
:108C800002241346C0F89442C0E906220A46002195
:108C90002EF007FA002010BD08B513460A46002141
:108CA0002EF0FFF9002008BD10B503241346C0F8CC
:108CB0009442C0E956220A4600212EF0FBF900201A
:108CC00010BD08B513460A4600212EF0F3F9002026
:108CD00008BD08B504220023C0F8942219461A469C
:108CE0002EF0DFF9002008BD08B505220023C0F8EA
:108CF000942219461A462EF0DDF9002008BD000026
:108D00000E4B30B55C7A054604F0FF00A4B95C7ADE
:108D100018555C7A03EB840465605C7A1C4422720B
:108D20005A7A541C3032E4B25C723A230A704B70A7
:108D30002F23C8708B7030BD0120FCE7681800201D
:108D40000022FFF7DDBF000008B501F0FDFB38B1E0
:108D5000022804D0034B1868431E5842584108BDEE
:108D60000320FCE7341B002008B5EFF3058313B1A3
:108D70006FF0050008BDEFF310820A4B12B9EFF354
:108D8000118212B11A68022AF2D01A68012A05D19A
:108D900002221A6001F01EF90020EBE74FF0FF30CD
:108DA000E8E700BF341B0020EFF305830BB101F0AF
:108DB00073B9EFF3108313B9EFF311831BB1034BB6
:108DC0001B68022BF3D001F061B900BF341B0020F7
:108DD000F0B5144687B000220B460592EFF30582EA
:108DE00022BBEFF3108212B9EFF311821AB1224ABB
:108DF0001268022A1AD0C8B1002C2FD0A569002D04
:108E000008BF18256A1EAC46372A2BD86268D207DD
:108E100028D466696EB1B2082168D4E9027E57B1E0
:108E2000BEF1BF0F02D9246904B1EEB9059807B0AD
:108E3000F0BD8022F0E7BEF1000FF7D12469002CCD
:108E4000F4D10C4605A992B2CDE900C1214601F04A
:108E500093F801281CBF00230593E7E74FF0180C97
:108E60008022EFE70020E2E7CDE90147009501F01D
:108E700045F80590DAE700BF341B002001F05EBB27
:108E800008B5EFF3058313B16FF0050008BDEFF3EC
:108E9000108313B9EFF311831BB1054B1B68022B31
:108EA000F2D00028F2D001F00DFA0020EEE700BF6A
:108EB000341B002070B50546EFF3058616B100247B
:108EC000204670BDEFF3108212B9EFF311821AB190
:108ED000184A1268022AF2D015B16E683307EED430
:108EE00006F001067DB1D5E9021351B14F2BE6D949
:108EF000DEB1042000F0ADFB04460028DFD02D6871
:108F00000AE0002BDBD196B1042000F0D7FB044629
:108F10000028D4D0002DF2D12946204600F03EFE94
:108F2000002ECDD044F00104CAE70120E2E7012081
:108F3000EBE700BF341B0020034620F0010010B512
:108F400003F001030C46EFF3058212B16FF0050048
:108F500010BDEFF3108212B9EFF311821AB10D4A6E
:108F60001268022AF2D088B1214663B100F09CFD5C
:108F7000012801D10020EBE7002C14BF6FF00100A5
:108F80006FF00200E4E700F0C4FCF1E76FF00300CB
:108F9000DEE700BF341B002008B5034620F00100C7
:108FA00003F00103EFF3058212B16FF0050008BD75
:108FB000EFF3108212B9EFF311821AB10A4A126864
:108FC000022AF2D068B13BB100F058FB01280CBF77
:108FD00000206FF00200EAE71A46194600F07EFA18
:108FE000F4E76FF00300E2E7341B002073B514468A
:108FF000EFF305831BB10025284602B070BDEFF3E7
:10900000108313B9EFF311831BB11A4B1B68022BAA
:10901000F1D00028EFD00029EDD0ECB1D4E9023234
:1090200093B14F2AE7D92269002AE4D001FB00F569
:109030006669AE42DFD30025009500F012FA0546BE
:109040000028D8D024680FE0002AD4D12369002B4F
:10905000D1D16369002BCED1002200F016FA05466B
:109060000028C8D0002CEDD12146284600F096FDFE
:10907000C2E700BF341B002013B51C46EFF3058385
:1090800023B1D8B96FF0030002B010BDEFF3108325
:1090900013B9EFF311831BB1174B1B68022BF0D0F0
:1090A0000028EFD00029EDD00023224600F016FA68
:1090B000012810D0E4B96FF00200E5E70029E1D003
:1090C000002CDFD1234601AA019400F014FB0128F3
:1090D000F1D1019B0BB90020D6E74FF0E0234FF010
:1090E0008052C3F8042DBFF34F8FBFF36F8FF2E7A9
:1090F0006FF00100C8E700BF341B002013B51C4609
:10910000EFF3058323B1D0B96FF0030002B010BDB7
:10911000EFF3108313B9EFF311831BB1164B1B68E8
:10912000022BF0D00028EFD00029EDD0224600F02D
:109130004BFB01280FD0DCB96FF00200E6E70029F5
:10914000E2D0002CE0D101AA019400F0D1FC01286A
:10915000F2D1019B0BB90020D8E74FF0E0234FF08C
:109160008052C3F8042DBFF34F8FBFF36F8FF2E728
:109170006FF00100CAE700BF341B0020034B0360FF
:10918000034B0B6080231360704700BF741A0020EC
:1091900074180020034B0360034B0B604FF4807383
:1091A00013607047381F0020381B002000F10803AF
:1091B0004FF0FF3243600361C0E9022300230360E4
:1091C000704700230361704743689A684B608A6068
:1091D0009A685160996003680861013303607047C1
:1091E00030B50C68631C0AD103695A684A60916003
:1091F0008B605960036808610133036030BD00F182
:109200000802134652681568A542FAD9EDE70369CA
:10921000D0E901128A6051605968814208BF5A60E2
:10922000002202611A68013A1A601868704710B586
:10923000044601F0DFFCA46B01F000FDB4FA84F0F9
:10924000400910BDF8B51546026C0446866B52B94C
:10925000076847BB806801F0C7F90546A76001367B
:109260002846A663F8BD65B940684DF04DFB6368BC
:10927000226C1344A26893426360F0D32368636056
:10928000EDE7C0684DF040FB226CE36851429B1A49
:1092900022689342E3603EBFA3685B18E360022D3F
:1092A00001D116B1013E0025D9E73546D7E703467F
:1092B00008461A6C10B462B1DC68996814448C4298
:1092C000DC605DF8044B24BF1968D960D9684DF0A3
:1092D0001BBB5DF8044B704770B5044601F08AFC77
:1092E00094F8455004F124066DB2002D14DCFF23E0
:1092F00004F1100684F8453001F0A0FC01F07AFC7E
:1093000094F844506DB2002D12DCFF2384F84430F1
:10931000BDE8704001F092BC636A002BE7D0304694
:1093200001F074F808B101F003F9013D6DB2DCE71A
:109330002369002BE9D0304601F068F808B101F04C
:10934000F7F8013D6DB2DEE738B50D46044650B979
:109350004FF0500372B683F31188BFF36F8FBFF3E2
:109360004F8F62B6FEE701F045FC2268D4E90F3169
:1093700062604B43D0185B1A1344A0600020E36086
:10938000FF23A06384F8443084F84530A5B92369ED
:1093900073B104F1100001F039F848B14FF0E02347
:1093A0004FF08052C3F8042DBFF34F8FBFF36F8F80
:1093B00001F044FC012038BD04F11000FFF7F6FE77
:1093C00004F12400FFF7F2FEF2E713B51C4653B98F
:1093D0004FF0500372B683F31188BFF36F8FBFF362
:1093E0004F8F62B6FEE75AB1B1B94FF0500372B673
:1093F00083F31188BFF36F8FBFF34F8F62B6FEE721
:1094000051B14FF0500372B683F31188BFF36F8FE1
:10941000BFF34F8F62B6FEE750230193019B502BA1
:109420000AD04FF0500372B683F31188BFF36F8FE9
:10943000BFF34F8F62B6FEE7002908BF2246019BAB
:109440000123226084F84630C4E90F011946204602
:10945000FFF77AFF9DF81030204684F84C3002B0B8
:1094600010BD10B49DF8044050B94FF0500372B6CF
:1094700083F31188BFF36F8FBFF34F8F62B6FEE7A0
:1094800001945DF8044BFFF7A0BFF8B50D461746F1
:10949000064650B94FF0500372B683F31188BFF3FC
:1094A0006F8FBFF34F8F62B6FEE74843503001F035
:1094B000DFFC044670B1002380F8463065B100F14E
:1094C0005003012120462360C4E90F65FFF73CFFEC
:1094D00084F84C702046F8BD0346F2E72DE9F043CE
:1094E00085B088461F460446019250B94FF050039C
:1094F00072B683F31188BFF36F8FBFF34F8F62B6DD
:10950000FEE761B9036C53B14FF0500372B683F3B9
:109510001188BFF36F8FBFF34F8F62B6FEE7022F44
:109520000DD1E36B012B0AD04FF0500372B683F3D9
:109530001188BFF36F8FBFF34F8F62B6FEE701F064
:1095400003F8064660B9019B5BB14FF0500372B659
:1095500083F31188BFF36F8FBFF34F8F62B6FEE7BF
:1095600000264FF0000937E0019D1DB901F066FBB0
:10957000002052E016B902A800F08EFF01F05EFB59
:1095800000F07CFD01F036FB94F84430FF2B01D154
:1095900084F8449094F84530FF2B01D184F845902D
:1095A00001F04CFB01A902A800F082FF00284AD17B
:1095B00001F020FBA26BE36B9A4231D101F03EFB3C
:1095C000019904F1100000F0E5FE2046FFF784FE4B
:1095D00000F002FE60B3012601F00CFBA26BE36B0E
:1095E0009A4201D3022FBFD13A4641462046FFF7A7
:1095F00029FE636A1BB104F1240000F007FF48B1A3
:109600004FF0E0234FF08052C3F8042DBFF34F8F8B
:10961000BFF36F8F01F012FB012005B0BDE8F083AE
:1096200001F00CFB2046FFF757FE00F0D5FDD2E716
:109630004FF0E0234FF08052C3F8042DBFF34F8F5B
:10964000BFF36F8FC7E72046FFF746FE00F0C4FD6B
:109650008EE700220B4613B5114600900120FFF75C
:10966000B4FE044638B100231A46194683600360ED
:10967000C360FFF733FF204602B010BD38B5044683
:1096800050B94FF0500372B683F31188BFF36F8F58
:10969000BFF34F8F62B6FEE7856800F04FFF85424B
:1096A0000AD1E368013BE36023B91A461946204614
:1096B000FFF714FF012000E0002038BD70B506461A
:1096C000502001F0D5FB044698B10025012100602F
:1096D00080F84650C0E90F15FFF736FE2B462A46A4
:1096E0002946204684F84C60A5602560E560FFF7B8
:1096F000F5FE204670BD2DE9F843894690461F4689
:10970000044650B94FF0500372B683F31188BFF38B
:109710006F8FBFF34F8F62B6FEE761B9036C53B131
:109720004FF0500372B683F31188BFF36F8FBFF30E
:109730004F8F62B6FEE7022F0DD1E36B012B0AD0EB
:109740004FF0500372B683F31188BFF36F8FBFF3EE
:109750004F8F62B6FEE701F035FBEFF311864FF055
:10976000500372B683F31188BFF36F8FBFF34F8F2F
:1097700062B6A26BE36B9A4201D3022F22D194F816
:1097800045503A46494620466DB2FFF75BFD6B1CDB
:1097900013D1636A0BB901200BE004F1240000F03F
:1097A00035FE0028F7D0B8F1000FF4D00120C8F83A
:1097B000000086F31188BDE8F88301356DB284F8A6
:1097C0004550E8E70020F4E72DE9FF410F46044645
:1097D000019250B94FF0500372B683F31188BFF372
:1097E0006F8FBFF34F8F62B6FEE761B9036C53B161
:1097F0004FF0500372B683F31188BFF36F8FBFF33E
:109800004F8F62B6FEE700F09FFE064660B9019BEF
:109810005BB14FF0500372B683F31188BFF36F8FC3
:10982000BFF34F8F62B6FEE700264FF000083DE021
:10983000019D1DB901F002FA002056E016B902A8F8
:1098400000F02AFE01F0FAF900F018FC01F0D2F95C
:1098500094F84430FF2B01D184F8448094F84530CB
:10986000FF2B01D184F8458001F0E8F901A902A895
:1098700000F01EFE002841D12046FFF7D8FCB8B307
:10988000019904F1240000F085FD2046FFF724FD36
:1098900000F0A2FC48B94FF0E0234FF08052C3F82B
:1098A000042DBFF34F8FBFF36F8F012601F0A2F994
:1098B000A56B002DBCD0013D39462046FFF7F7FCD3
:1098C000A563236973B104F1100000F09FFD48B156
:1098D0004FF0E0234FF08052C3F8042DBFF34F8FB9
:1098E000BFF36F8F01F0AAF9012004B0BDE8F08149
:1098F0002046FFF7F1FC00F06FFCD6E72046FFF7AB
:10990000EBFC00F069FC2046FFF791FC0028CCD06E
:1099100092E7F0B585B00446019150B94FF050037D
:1099200072B683F31188BFF36F8FBFF34F8F62B6A8
:10993000FEE7056C55B14FF0500372B683F3118802
:10994000BFF36F8FBFF34F8F62B6FEE700F0FCFDF1
:10995000064660B9019B6BB14FF0500372B683F3BA
:109960001188BFF36F8FBFF34F8F62B6FEE72E46AD
:10997000002755E00546FBE7019B73B955B14FF051
:10998000500372B683F31188BFF36F8FBFF34F8F0D
:1099900062B6FEE701F052F962E016B902A800F0E3
:1099A0007BFD01F04BF900F069FB01F023F994F81D
:1099B0004430FF2B01D184F8447094F84530FF2BDC
:1099C00001D184F8457001F039F901A902A800F02D
:1099D0006FFD00284DD12046FFF729FC002842D01A
:1099E00023683BB901F006F9A06800F0BDFD05460B
:1099F00001F024F9019904F1240000F0CBFC204689
:109A0000FFF76AFC00F0E8FB48B94FF0E0234FF0A5
:109A10008052C3F8042DBFF34F8FBFF36F8F012621
:109A200001F0E8F8A36B002BA6D0013BA3632368E9
:109A300013B900F077FEA060236973B104F1100040
:109A400000F0E4FC48B14FF0E0234FF08052C3F83F
:109A5000042DBFF34F8FBFF36F8F012501F0EEF898
:109A6000284605B0F0BD2046FFF736FC00F0B4FBF9
:109A7000D5E72046FFF730FC00F0AEFB2046FFF7AD
:109A8000D6FB0028CBD0002DEAD001F0B3F8616AF4
:109A900019B1236B1968C1F13801A068002500F0E5
:109AA000EBFD01F0CBF8DBE737B5044650B94FF0DA
:109AB000500372B683F31188BFF36F8FBFF34F8FDC
:109AC00062B6FEE78568019100F038FD8542019994
:109AD00005D1E36801200133E36003B030BD2046C7
:109AE000FFF717FF0028F8D0E3680133E360F4E7DD
:109AF0002DE9F84389469046054650B94FF050038A
:109B000072B683F31188BFF36F8FBFF34F8F62B6C6
:109B1000FEE761B9036C53B14FF0500372B683F3A3
:109B20001188BFF36F8FBFF34F8F62B6FEE701F06E
:109B300049F9EFF311874FF0500372B683F31188A0
:109B4000BFF36F8FBFF34F8F62B6AC6B1CB395F84A
:109B5000446049462846013C76B2FFF7A8FBAC6357
:109B6000731C13D12B690BB901200BE005F1100018
:109B700000F04CFC0028F7D0B8F1000FF4D0012021
:109B8000C8F8000087F31188BDE8F883013676B283
:109B900085F84460E8E72046F4E700000023074A20
:109BA00010B552F833402CB942F8331002EBC3031E
:109BB000586010BD0133082BF3D1FAE7F81F0020DD
:109BC00070B504460D46164601F014F894F844307A
:109BD000FF2B02D1002384F8443094F84530FF2B4A
:109BE00002D1002384F8453001F028F8A36B2BB98B
:109BF0003246294604F1240000F0E8FB2046BDE887
:109C00007040FFF769BB00002DE9F041044600F009
:109C1000F1FF2F4B2F4E1A682F4F01321A60356813
:109C2000002D4AD134601B68012B1FD1B846013585
:109C30004046FFF7BBFA08F11408382DF7D1DFF8DA
:109C4000C080264D4046FFF7B1FA2846FFF7AEFA2E
:109C50002348FFF7ABFA2348FFF7A8FA2248FFF79B
:109C6000A5FA224BC3F80080214B1D60214A1368DE
:109C700001331360204A63641168E36A8B4200D9A0
:109C800013601420211D00FB0370FFF79DFA00F004
:109C9000D5FF1A4B1B6873B13368DA6AE36A9A42DC
:109CA00009D24FF0E0234FF08052C3F8042DBFF3E8
:109CB0004F8FBFF36F8FBDE8F081104B1B68002BF7
:109CC000D4D13368DA6AE36A9A42CFD83460CDE7F8
:109CD000A42400203820002044200020D02400208C
:109CE000EC24002018250020042500203C20002022
:109CF00040200020B4240020B824002000250020AB
:109D0000BC240020F8B5154B0446154E0F461D68BF
:109D100030680430FFF77BFA631C07D137B1316834
:109D200010480431BDE8F840FFF74EBA2C193368EB
:109D30005C6007D30C4B18683168BDE8F84004310B
:109D4000FFF74EBA094B186831680431FFF748FA3B
:109D5000074B1A68A24200D91C60F8BD2C250020D0
:109D60003820002004250020402000203C20002036
:109D7000E4240020064A13681968064B19B94FF00D
:109D8000FF321A6070471268D268D2685268F8E7EA
:109D90003C200020E424002010B5044658304DF04B
:109DA000FDFC94F8BD303BB9206B01F0F5F820467E
:109DB000BDE8104001F0F0B8012BF8D0022B0AD01A
:109DC0004FF0500372B683F31188BFF36F8FBFF368
:109DD0004F8F62B6FEE710BD80B5134C134F144D84
:109DE000236873B9134B1B68012BF8D94FF0E0239C
:109DF0004FF08052C3F8042DBFF34F8FBFF36F8F26
:109E0000EDE700F0F7FEFB68DE68301DFFF7FFF9B5
:109E10002B68013B2B602368013B236000F00EFFA1
:109E20003046FFF7B9FFDBE7A82400201825002003
:109E3000A4240020442000202DE9F0474FEA8209A5
:109E400006460D46A5214A461F46A9F10409DDE94B
:109E50000984206B4CF080FD226B914429F00709A6
:109E6000002D42D06B1E04F134020F3513F8010FA0
:109E700002F8010B08B1AB42F8D1002384F843305B
:109E8000089D4FF0000A201D372DC4F850A028BFB0
:109E90003725E562E564C5F13805FFF792F904F16D
:109EA0001800FFF78EF960225146C4F8B8A004F1FB
:109EB00058002461A5616462C4F854A084F8BCA071
:109EC0004CF04AFD0A4B3A463146E3654846094B99
:109ED0002366094B636600F069FE2060B8F1000F4D
:109EE00001D0C8F80040BDE8F08784F83450C7E7D7
:109EF000404E0708604E0708204E070870B586B030
:109F0000DDE90B5455B94FF0500372B683F3118855
:109F1000BFF36F8FBFF34F8F62B6FEE754B94FF0B8
:109F2000500372B683F31188BFF36F8FBFF34F8F67
:109F300062B6FEE7C0260596059EC02E0AD04FF0F9
:109F4000500372B683F31188BFF36F8FBFF34F8F47
:109F500062B6FEE725630225059E84F8BD5004AD78
:109F6000029401950A9D0095FFF766FF2046FFF7D2
:109F70004BFE049806B070BD2DE9F043074685B04E
:109F8000900088461646994600F072FF0546E8B1F3
:109F9000C02000F06DFF0446A8B1002305633246DF
:109FA000414680F8BD300D9B0290384601930C9BD2
:109FB00000934B46FFF740FF2046FFF725FE0120A8
:109FC00005B0BDE8F083284600F0E6FF4FF0FF3013
:109FD000F6E7000010B588B0002407AA06A905A876
:109FE000CDE90544FFF7CAF8059B079A0293069B43
:109FF0001B491C48CDE900432346FFF77FFF00289B
:10A000002CD000F0EDFB01281BD14FF0500372B6AD
:10A0100083F31188BFF36F8FBFF34F8F62B6124B7C
:10A02000124A1B68583313604FF0FF32104B1A600E
:10A03000104B1860104B1C6008B0BDE8104000F0D9
:10A040005BBE01300AD14FF0500372B683F3118822
:10A05000BFF36F8FBFF34F8F62B6FEE708B010BD3E
:10A0600048060608D99D000838200020141000205A
:10A07000E4240020002500202C250020024A13683B
:10A0800001331360704700BFB0240020014B1868F3
:10A09000704700BF2C25002008B500F093FE014B4F
:10A0A000186808BD2C250020404B1B682DE9F74F90
:10A0B000002B74D13E4B1D6801351D60CDB93D4B61
:10A0C0001A68126852B14FF0500372B683F31188C8
:10A0D000BFF36F8FBFF34F8F62B6FEE7364A196842
:10A0E000106818601160354A136801331360FFF778
:10A0F00041FE334E0024334F3368DFF8D480AB4247
:10A1000011D9D8F800301422DB6A5343FB58022BD4
:10A1100028BF01242C4B1B68002B0CBF20460120BC
:10A1200003B0BDE8F08FDFF88C90DFF8A8A0D9F875
:10A1300000301B681BB94FF0FF333360E1E7D9F8FB
:10A140000030DB68D3F80CB0DBF80420954201D274
:10A150003260D6E70BF1040108460191FFF757F88A
:10A16000DBF82820019922B10BF11800FFF74FF816
:10A170000199DBF82C00DAF80020904201D9CAF8E6
:10A180000000142303FB0070FFF71EF8D8F800103E
:10A19000DBF82C20CB6A9A4228BF0124C7E70B4A80
:10A1A0000024136801331360B4E700BFB02400201B
:10A1B0002C2500203C20002040200020E824002006
:10A1C000E42400204420002030250020AC2400207E
:10A1D00038200020B8240020F7B5324C236853B94A
:10A1E0004FF0500372B683F31188BFF36F8FBFF344
:10A1F0004F8F62B6FEE700F0FDFC2368013B236051
:10A2000024682CB1002400F019FD204603B0F0BDF5
:10A21000254B1B68002BF5D0244D254E254F1EE005
:10A22000EB68DC6804F11800FEF7F1FF211D084619
:10A230000191FEF7ECFFE36A32680199934200D97D
:10A240003360142000FB0370FEF7BEFF1A4BE26A76
:10A250001B68DB6A9A4202D3184B01221A602B68F2
:10A26000002BDDD10CB1FFF785FD154D2C6844B1F5
:10A27000124E0127FFF718FF00B13760013CF9D1FA
:10A280002C600E4B1B68002BBCD04FF0E0234FF02E
:10A290008052C3F8042DBFF34F8FBFF36F8F01249B
:10A2A000B1E700BFB0240020A4240020EC2400204B
:10A2B000B824002044200020382000203025002031
:10A2C000AC24002008B550B94FF0E0234FF0805285
:10A2D000C3F8042DBFF34F8FBFF36F8F08BD0B4B37
:10A2E000196851B14FF0500372B683F31188BFF370
:10A2F0006F8FBFF34F8F62B6FEE7FFF7BFFEFFF72A
:10A3000001FDFFF769FF0028DED0E7E7B024002059
:10A310001A4B1A681A4B70B512B101221A6070BD3F
:10A32000184D14261A6018492A6806FB02F3CC5807
:10A33000C818ACB14468083364680B449C4244605C
:10A3400004BF63684360142303FB02114B68D968A0
:10A350000E4B19602A601B680D4A58331360DEE704
:10A3600052B94FF0500372B683F31188BFF36F8F69
:10A37000BFF34F8F62B6FEE7013AD6E7B024002064
:10A3800030250020B8240020442000203820002060
:10A390001410002010B50C4650B94FF0500372B69F
:10A3A00083F31188BFF36F8FBFF34F8F62B6FEE761
:10A3B000054B19681831FEF713FF20460121BDE84F
:10A3C0001040FFF79FBC00BF3820002038B50D4675
:10A3D000144650B94FF0500372B683F31188BFF39F
:10A3E0006F8FBFF34F8F62B6FEE7074B19681831C6
:10A3F000FEF7EAFE002C21460CBF28464FF0FF3046
:10A40000BDE83840FFF77EBC38200020C36813B594
:10A41000DC6854B94FF0500372B683F31188BFF370
:10A420006F8FBFF34F8F62B6FEE704F11801084645
:10A430000191FEF7ECFE124B01991B68E3B9211D57
:10A4400008460191FEF7E3FE0E4AE36A106801999F
:10A45000834200D913600C4A142000FB0320FEF74E
:10A46000B3FE0A4BE26A1B68DB6A9A4206D90120F6
:10A47000074B186002B010BD0648F0E70020F9E76E
:10A48000B0240020B82400204420002038200020E0
:10A4900030250020EC240020034B1B680360034B95
:10A4A0001B684360704700BFE82400202C25002073
:10A4B00070B50C46054650B94FF0500372B683F3A1
:10A4C0001188BFF36F8FBFF34F8F62B6FEE751B9AC
:10A4D0004FF0500372B683F31188BFF36F8FBFF351
:10A4E0004F8F62B6FEE700F085FB0F4B19682368BB
:10A4F0005A1C10D00D482E6800686A68864201D048
:10A500008A420FD9881A83420AD95B1A2846134413
:10A510002360FFF7C1FF002400F090FB204670BDD0
:10A52000002323600124F7E72C250020E8240020E5
:10A53000014B01221A60704730250020014B18683A
:10A54000704700BF38200020054B1B6833B1054B16
:10A550001B68002B0CBF02200020704701207047B1
:10A5600000250020B024002073B5044640B31B4DE5
:10A57000C36A2A68D26A934228D28269002A04DB1D
:10A580002A68D26AC2F1380282611422144E02FB98
:10A59000036362699A4215D1211D08460191FEF7B5
:10A5A00036FE2B680F4ADB6A106801998342E3622A
:10A5B00000D91360142000FB0360FEF705FE0120A4
:10A5C00002B070BD2B68DB6AE362F8E72B68C06CF1
:10A5D000DC6AA0422CBF00200120F1E738200020D7
:10A5E00044200020B824002013B510B9002002B088
:10A5F00010BD1E4B1C6884420AD04FF0500372B647
:10A6000083F31188BFF36F8FBFF34F8F62B6FEE7FE
:10A61000236D53B94FF0500372B683F31188BFF323
:10A620006F8FBFF34F8F62B6FEE7E16A013BE26CCA
:10A6300023659142DAD0002BD8D1211D0846019123
:10A64000FEF7E5FDE36C0199C3F13802E362A26114
:10A65000074A1068834200D91360064A142000FBA1
:10A660000320FEF7B1FD0120C1E700BF3820002024
:10A67000B82400204420002037B50446002848D0E4
:10A68000026D52B94FF0500372B683F31188BFF3D5
:10A690006F8FBFF34F8F62B6FEE7C36C994238BF2E
:10A6A0001946C36A8B4234D0012A32D11A4A126841
:10A6B00082420AD14FF0500372B683F31188BFF380
:10A6C0006F8FBFF34F8F62B6FEE78269134D002A8A
:10A6D0004FF01402C16202FB0353A8BFC1F138015D
:10A6E0004269A8BF81619A4213D1011D08460191B8
:10A6F000FEF78DFD0A4AE36A10680199834200D98A
:10A700001360142000FB035003B0BDE83040FEF797
:10A710005BBD03B030BD00BF3820002044200020C6
:10A72000B8240020044B1A681AB119680A6D013266
:10A730000A651868704700BF38200020F7B5114C33
:10A7400000F058FA2568BDB90F4F104E3846FEF795
:10A750002DFD3046FEF72AFD0D4B0E4A10211F60DD
:10A760000A200D4B1E600D4B0095FEF77AFE20600F
:10A7700010B10B49FFF712FA03B0BDE8F04000F04A
:10A780005DBA00BF58260020DC250020F0250020FF
:10A79000342500203C2500203825002008260020F4
:10A7A0004D060608914208B5416000610AD8D21AE8
:10A7B00083699A420DD2011D074B1868FEF710FD00
:10A7C000002008BD9A4201D2994202D2011D034BDA
:10A7D000F3E70120F5E700BF3825002034250020ED
:10A7E00010B588B0FFF7AAFF134B1B68B3B1002464
:10A7F00007AA06A905A8CDE90544FEF7CBFC059BF1
:10A80000079A0293069B0D49019302230C4800937B
:10A810002346FFF773FB0B4B186050B94FF0500302
:10A8200072B683F31188BFF36F8FBFF34F8F62B699
:10A83000FEE7012008B010BD582600205206060889
:10A8400051A900085C2600207FB5164604461A462A
:10A8500050B94FF0500372B683F31188BFF36F8F76
:10A86000BFF34F8F62B6FEE70C4D286878B105291B
:10A870000294CDE900160CDCFFF766FE00230228E7
:10A88000694628680CBF089A1A46FEF727FE04B0EE
:10A8900070BD00236946FEF72EFFF8E7582600201A
:10A8A0002DE9FF47DFF8A4800646FFF7EFFB0546DA
:10A8B000D8F80030834242D9224F4FF000093B685C
:10A8C0001A685AB9204A1168136001233960284672
:10A8D0003360C8F8005004B0BDE8F087DB68DC687E
:10A8E000D3F800A0211D08460391FEF790FC236ACF
:10A8F0002046984794F82830039913F0040FDED0CF
:10A90000A36953449A4505D2386863602461FEF711
:10A9100067FCD4E7002352462046CDF80090194644
:10A92000FFF792FF0028CAD14FF0500372B683F3AD
:10A930001188BFF36F8FBFF34F8F62B6FEE700231E
:10A94000C5E700BF3425002038250020042600205C
:10A950002DE9F043714D89B0714E2B68D3F800801A
:10A96000B8F1000F37D0DB680024D3F80080FFF780
:10A9700085FB04A8FFF794FF049B8146002B6BD155
:10A98000002C4ED1404552D3FFF726FC2B68DB68E4
:10A99000DF68381DFEF73BFC97F8283058071CD5B8
:10A9A000B96943464A4638464144FFF7FBFEC0B109
:10A9B00023464246214638460094FFF745FF80B9BA
:10A9C0004FF0500372B683F31188BFF36F8FBFF35C
:10A9D0004F8F62B6FEE70124C9E723F0010387F831
:10A9E00028303B6A38469847002204A93068FEF7B1
:10A9F000EBFE0028B1D0049B0698002B2FDB069CB1
:10AA00006369002B32D103A8FFF74AFF049B02467B
:10AA1000092BE9D8DFE803F02E2E2E59607A2E2E6E
:10AA20005960404B1B681C68B4FA84F464092246E0
:10AA3000A8EB09013068FFF7C3F8FFF7CDFB00284A
:10AA4000D2D14FF0E0234FF08052C3F8042DBFF372
:10AA50004F8FBFF36F8FC7E7FFF7BEFBC4E7059BC0
:10AA600007999847049B002BBEDBC8E7201DFEF723
:10AA7000CEFBC8E794F828302046A16943F00103D3
:10AA800084F82830059B1944FFF78CFE0028ABD0D2
:10AA9000236A2046984794F828305907A4D5A2691C
:10AAA00000230599204600930A441946FFF7CCFE7F
:10AAB000002899D14FF0500372B683F31188BFF389
:10AAC0006F8FBFF34F8F62B6FEE794F8283023F004
:10AAD000010384F8283087E794F8283043F0010315
:10AAE00084F828300599A16151B94FF0500372B62E
:10AAF00083F31188BFF36F8FBFF34F8F62B6FEE70A
:10AB0000034601442046FFF74DFE6DE794F82830D8
:10AB10009A07DCD4204600F03FFA65E73425002090
:10AB2000582600203825002008480068006880F377
:10AB300008884FF0000080F3148862B661B6BFF356
:10AB40004F8FBFF36F8F00DF00BF000008ED00E004
:10AB5000DFF80C00016841F47001016070470000EB
:10AB600088ED00E0002382B001930F4B1B68013396
:10AB70000AD04FF0500372B683F31188BFF36F8F82
:10AB8000BFF34F8F62B6FEE74FF0500372B683F308
:10AB90001188BFF36F8FBFF34F8F62B6019B002BFD
:10ABA000FCD002B0704700BFD00000204FF080738F
:10ABB00021F0010140F8202C44380364034BC163A9
:10ABC00083636FF002030362704700BF65AB000848
:10ABD000074B19680868B0E8F04F80F30988BFF3A5
:10ABE0006F8F4FF0000080F311887047AFF3008043
:10ABF000382000204FF0500372B683F31188BFF362
:10AC00006F8FBFF34F8F62B60B4A13680133012B6E
:10AC1000136010D14FF0E023D3F8043DDBB253B101
:10AC20004FF0500372B683F31188BFF36F8FBFF3F9
:10AC30004F8F62B6FEE77047D0000020094A1368C4
:10AC400053B94FF0500372B683F31188BFF36F8F7F
:10AC5000BFF34F8F62B6FEE7013B13600BB983F37E
:10AC600011887047D00000200000000000000000A4
:10AC7000EFF30980BFF36F8F154B1A681EF0100FAA
:10AC800008BF20ED108A20E9F04F10602DE909007F
:10AC90004FF0500072B680F31188BFF34F8FBFF3AF
:10ACA0006F8F62B6FFF734FB4FF0000080F311881E
:10ACB00009BC19680868B0E8F04F1EF0100F08BF13
:10ACC000B0EC108A80F30988BFF36F8F704700BF24
:10ACD000382000204FF0E02200234FF47A711361F6
:10ACE0009361044B1B68B3FBF1F3013B53610723F2
:10ACF00013617047080000202E4B37B51A780021E9
:10AD0000D2B20192FF221A701B782B4ADBB28DF867
:10AD100003309DF8033003F0500313700723274AD4
:10AD200013609DF803005C1E00060ED411B1032BC6
:10AD3000136013D04FF0500372B683F31188BFF342
:10AD40006F8FBFF34F8F62B6FEE79DF8033001218E
:10AD50005B00DBB28DF803302346E2E74FF440732B
:10AD60004FF0E02400251360019B124ADBB2137000
:10AD7000D4F8203D43F47003C4F8203DD4F8203DBE
:10AD800043F07043C4F8203DFFF7A4FF0C4B1D6057
:10AD9000FFF7DEFED4F8343F43F04043C4F8343FBD
:10ADA000FFF7C2FEFFF7B4FA2846FFF7DBFE03B059
:10ADB00030BD00BF00E400E06026002064260020D3
:10ADC000D0000020EFF305830F2B10D9134A9B5CB2
:10ADD000134A12789A420AD94FF0500372B683F39D
:10ADE0001188BFF36F8FBFF34F8F62B6FEE74FF04E
:10ADF000E0230C4AD3F80C3D126803F4E06393425D
:10AE00000AD94FF0500372B683F31188BFF36F8FE6
:10AE1000BFF34F8F62B6FEE7704700BFF0E300E07C
:10AE200060260020642600200F4B10B51A461B68D0
:10AE30008342FBD354681119884201BF4168104610
:10AE400009195160446801198B4207D10749096803
:10AE50008B421FBF59681B6809194160904203600B
:10AE600018BF106010BD00BF7826022068260020A1
:10AE70002DE9F0410446FFF701F94148414D0368CF
:10AE80000BBB41494E07414E1BBFCB1D01F50032A4
:10AE90004FF4003223F007031CBF1946D21A0023D7
:10AEA0000A4431607360083A22F00702C2E90033B5
:10AEB000531A0260C1E90023354A1360354A136012
:10AEC0004FF000432B602F68274254D1002C43D011
:10AED00004F1080361071CBF23F007030833002BAC
:10AEE00049D02C4C26689E4245D3284A156869688B
:10AEF000994204D2D5F800C0BCF1000F17D1006808
:10AF0000A84238D0C91A2868D2F8008010291060E9
:10AF100014D9E81842070DD04FF0500372B683F3EE
:10AF20001188BFF36F8FBFF34F8F62B6FEE72A46DB
:10AF30006546DCE741606B60FFF776FF6B6814499C
:10AF4000F61A1F4308680023266008F108048642A9
:10AF50006F602B6038BF0E60FFF73EF963070CD0BF
:10AF60004FF0500372B683F31188BFF36F8FBFF3B6
:10AF70004F8F62B6FEE70024EEE72046BDE8F08181
:10AF8000682600206C2602206C26002078260220ED
:10AF9000742602207026022010B50446002832D004
:10AFA000194A50F8043C126813420AD14FF050037A
:10AFB00072B683F31188BFF36F8FBFF34F8F62B602
:10AFC000FEE750F8081C51B14FF0500372B683F3FE
:10AFD0001188BFF36F8FBFF34F8F62B6FEE723EA8E
:10AFE000020340F8043CFFF749F8084A54F8043CCF
:10AFF000A4F1080011680B441360FFF715FFBDE8CA
:10B000001040FFF7E9B810BD6C2602207026022020
:10B0100008B5074B00221039186001238160C0E990
:10B0200000230448FDF746FF034B186008BD00BF2E
:10B0300084260220A006060880260220F8B50E46C7
:10B04000054610B900242046F8BD174F0021386886
:10B05000FDF772FF0028F5D1144BE81D1C6820F0A5
:10B06000070034B1636813B1A368834205D2246832
:10B07000F7E73868FDF790FFE5E71B1A103B072B51
:10B0800009DD00F110012568621865500121C2E94F
:10B0900001132260A0600023E6603868103444F891
:10B0A0000C3CFDF779FFCEE78026022084260220A3
:10B0B000F8B50746002848D0244E00213068FDF737
:10B0C0003BFF002841D1224B04461D68002D36D09D
:10B0D00005F11003BB422ED22C462D68F6E7AA6874
:10B0E000CC2138464BF038FC2B68CBB15A68BAB14A
:10B0F00019689A68AB6864B1606850B12160A16852
:10B100000B4420331344A3603068BDE8F840FDF7DA
:10B1100043BF103329601344AB6001236B60F3E736
:10B12000002CFAD06268002AF7D0AA682360A368CE
:10B1300013441033E7E702D16B68002BCFD0054BE7
:10B140008121054A05484AF035FDF8BD80260220D8
:10B15000842602205A0606086006060876060608B7
:10B1600070B50D460E4E002104460160306829601E
:10B17000FDF7E2FE90B90B4B1B6853B1D3E90120F8
:10B180001AB1216801442160F6E72A6802442A6066
:10B19000F2E73068BDE87040FDF7FEBE70BD00BF4D
:10B1A00080260220842602200EB410B5C3B00446C7
:10B1B0004FF4807145AB01A853F8042B00934EF077
:10B1C000B9FF002301A88DF8043154B9F5F77AF8D6
:10B1D000014601A82AF032FD43B0BDE8104003B09B
:10B1E0007047F5F76FF8012C014601A802D12AF04B
:10B1F00039FDF1E72AF04AFDEEE7000008B500F05E
:10B20000C5F8034B00221860024B1A7008BD00BF3E
:10B2100088260220D400002008B5064B1B782BB9E5
:10B2200000F0B4F8044B1B68C01A08BD4EF660204D
:10B23000FBE700BFD40000208826022010B5064C92
:10B2400023783BB9FFF7E8FF4EF65F23984284BFAF
:10B250000123237010BD00BFD400002000F2FF3096
:10B260000A4938B520F47F730A68094C23F00303B8
:10B2700020689A4205D8074B5C21074A07484AF0E4
:10B2800099FCC518D31A25600B6038BD942602209E
:10B290008C260220B0060608C9060608ED06060838
:10B2A00008B54FF04042064B4FF400101A604FF0C3
:10B2B0008072044B1A60FFF7D1FF034B186008BD82
:10B2C0008C26022094260220C026022038B54FF496
:10B2D0000040204CFFF7C2FF1F4B204D1860204656
:10B2E000FFF7BCFF1E4B18602046FFF7B7FF1D4B52
:10B2F00018602046FFF7B2FF28602046FFF7AEFF38
:10B30000194B18602046FFF7A9FF184B186020461C
:10B31000FFF7A4FF164B18602046FFF79FFF154B61
:10B3200018602046FFF79AFF134B18602046FFF77E
:10B3300095FF124B18602046FFF790FF104B1860E6
:10B340004FF48030FFF78AFF0E4B2A6818600E4BCF
:10B350001A6038BD00B80B00B8260220C4260220AF
:10B36000982602209C260220C8260220A026022021
:10B37000A4260220A8260220AC260220B026022005
:10B38000B426022090260220BC260220F7F764BED5
:10B39000FF2810B50FD00B4B0B4A195C002013F897
:10B3A000014B8C4208D1D2ED007AB4EE670AF1EE7F
:10B3B00010FA01D1C0B210BD013004322328EED101
:10B3C000FF20F8E7680706088C07060870B50446F2
:10B3D00040B1074E0025214656F8040BF4F768FFEC
:10B3E00008B9E8B270BD0135232DF4D10020F9E78A
:10B3F000D8000020FF281CBF014B185C704700BF1D
:10B4000068070608FF281DBF034B03EB800090ED83
:10B41000000AB7EE000A70478C070608B0EE407AC3
:10B42000F7EE006A70B50446164DF5EC017AF4EEBD
:10B43000E67AF1EE10FA0DDCF4EEC77AF1EE10FACE
:10B44000F3DD15ED020A2046FFF7A2FFFF28ECD03E
:10B45000044615E00C4E06F1240535ED010AB4EE64
:10B46000660AF1EE10FA0BD0B4EEC07AF1EE10FAE3
:10B4700004DB2046FFF78CFFFF28E9D1B542ECD171
:10B48000204670BD1C08060818080608F0EE407A31
:10B49000064A082332ED010AB4EEE70AF1EE10FA8B
:10B4A00003D4013BF6D19FED020A70473C08060821
:10B4B000CCBC8C2B08B5F0EE407A0146FFF7A2FF1A
:10B4C000B4EEE00AF1EE10FA04DAB4EEE70AF1EEB7
:10B4D00010FA06DBFFF7DAFF0846BDE80840FFF781
:10B4E00057BFFF2008BD000070B50B4EB0EE407A8C
:10B4F000054606F1240434ED010AB4EEC70AF1EE64
:10B5000010FA04D82846FFF743FFFF2802D1B442BF
:10B51000F1D1FF2070BD00BF18080608B0EE407AD8
:10B5200070B505460B4E0024B6EC010AB4EEE00AF5
:10B53000F1EE10FA04DAB4EEC70AF1EE10FA04DB09
:10B540002846FFF725FFFF2803D10134092CEBD152
:10B55000FF2070BD18080608704720EE000A7047EB
:10B56000B7EE007A77EE407AA7EEE77AB0EE470AB8
:10B57000704760EE007A27EE800A704760EE007A2E
:10B5800067EE807A27EE800A704760EE007A67EEF9
:10B59000807A67EE807A27EE800A70479FED087AFE
:10B5A000DFED087A20EE077A60EE277A27EE007A40
:10B5B00060EE677AE7EE007AB0EE670A704700BF88
:10B5C000B0E62C4060CDD93F08B52DED028BB7EE2B
:10B5D000008AF1EE000A38EE400A46F07BFD38EEB4
:10B5E000400ABDEC028B08BD08B52DED028BB7EE0D
:10B5F000008AF1EE040A38EE400A46F06BFD38EEA0
:10B60000400ABDEC028B08BD08B52DED028BF7EEAC
:10B61000008AF0EE080A30EE688AB0EE480A46F07A
:10B6200059FDDFED077A28EE088AE0EE278ADFED84
:10B63000057AB0EE680AA8EE270ABDEC028B08BDB9
:10B64000B0E62C4060CDD93FDFED077A20EE270A27
:10B65000F6EE007A08B520EE270A46F0D5FAF7EEA6
:10B66000007A37EEC00A08BDDB0F4940DFED077AEC
:10B6700008B520EE270A46F0C7FAF7EE007A30EE5A
:10B68000670AF6EE007A20EE670A08BDDB0F494034
:10B69000DFED047A20EE270AF6EE007A20EE270A84
:10B6A00046F0F6BADB0F494008B52DED028BB7EE38
:10B6B000008AF0EE487AE0EE407AB0EE670A46F093
:10B6C00061FD38EE400ABDEC028B08BDB7EE007A92
:10B6D00070EE477AA7EEE77AB0EE470A46F052BD21
:10B6E000DFED1D7A9FED1D7AB4EEE70AF1EE10FA58
:10B6F00004D520EE077A27EE000A7047DFED187AAE
:10B70000B4EEE70AF1EE10FA0AD5DFED167A70EE24
:10B71000677AB6EE080A27EE877AA7EE270A7047FF
:10B72000DFED117AB4EEE70AF1EE10FA0AD5DFED9B
:10B730000F7A70EE677AB6EE0E0A27EE877AA7EEDA
:10B74000870A7047DFED0A7A70EE677A9FED090A83
:10B7500027EE877AE1E700BF8C2EBA3E0000F24068
:10B760008C2E3A3FE9A20B3F2FBA683F5D74513FE0
:10B77000175D743F00007C3FF7EE006A08B536EEB7
:10B78000C00AFFF7ADFF36EEC00A08BDF6EE006A4C
:10B7900070EE007AB7EE006AB4EEE60A08B5F1EE94
:10B7A00010FA08D536EE670AFFF79AFF36EE400A20
:10B7B00020EE260A08BD37EEC60AFFF791FF30EEED
:10B7C000060AF5E7B6EE007AB4EEC70AF1EE10FA13
:10B7D0005BBFF0EE007AF8EE006A70EE007AE0EE01
:10B7E000267A4FBF27EE800AB7EE000A67EEE77AA7
:10B7F000A7EE870A704708B52DED028BB6EE008ADA
:10B80000B4EEC80AF1EE10FA0CD5B1EE007A20EED3
:10B81000077A27EE007A67EE007AB0EE670ABDEC91
:10B82000028B08BDB8EE007AF0EE007AF0EE080A5E
:10B83000E0EE077AB0EE670A46F04CFCF7EE007ACD
:10B84000E0EE487AE9E708B52DED028BB6EE008A06
:10B85000B4EEC80AF1EE10FA0ED5B2EE007A20EE80
:10B86000077A27EE007A27EE007A67EE007AB0EECC
:10B87000670ABDEC028B08BDB8EE007AF0EE007AE4
:10B88000F1EE000AE0EE077AB0EE670A46F022FC1D
:10B89000F7EE007AE0EE487AE9E708B52DED028B85
:10B8A000B6EE008AB4EEC80AF1EE10FA10D5B3EE87
:10B8B000007A20EE077A27EE007A27EE007A27EE4C
:10B8C000007A67EE007AB0EE670ABDEC028B08BD25
:10B8D000B8EE007AF0EE007AF1EE040AE0EE077AB4
:10B8E000B0EE670A46F0F6FBF7EE007AE0EE487A33
:10B8F000E9E70000B5EE400AF1EE10FA09D0F2EEE9
:10B90000047AFAEE040AE0EE270AB0EE000A46F0E6
:10B91000E1BB9FED010A70470000000008B52DED66
:10B92000028BB7EE008AB4EE480AF1EE10FA09D0A5
:10B93000FAEE040A60EE200AB0EE000A46F0CAFBF6
:10B9400038EE400ABDEC028B08BD0000B5EE400A9F
:10B9500008B5F1EE10FA2DED028B2BD0F7EE007A40
:10B96000B4EE670AF1EE10FA12D0B6EE008AB4EE29
:10B97000C80AF1EE10FA0ED5F3EE047AFAEE040AD4
:10B98000E0EE270AB0EE000A46F0A4FB20EE080A1B
:10B99000BDEC028B08BDFBEE047AF2EE040AE0EE89
:10B9A000270AB0EE000A46F095FBF0EE007A37EE7B
:10B9B000C00AEBE79FED010AEAE700BF00000000C4
:10B9C000B6EE007A70EE007AB4EEC70AF1EE10FA25
:10B9D0000CD59FED0F6A67EEA77ADFED0E6AE0EEF9
:10B9E000066A66EEA77A27EE870A7047B0EE000A6D
:10B9F000DFED095ADFED096A77EEC07AE7EEA56A56
:10BA000027EEA76AA6EE260A20EE070A704700BFB7
:10BA1000FF12E640FF1226C0FF126640FF122640CA
:10BA2000B5EE400A08B5F1EE10FA2DED048BB0EE3C
:10BA3000408A23D0F7EE007AB4EE670AF1EE10FAEE
:10BA400017D0B2EE049AFAEE040AE0EE090AB0EE5C
:10BA5000000A46F03FFBDFED0B7AF0EE408A9FEDE7
:10BA60000A0AE8EE097A27EE800A46F011F928EE74
:10BA7000C08AB0EE480ABDEC048B08BD9FED038A76
:10BA8000F7E700BF00002CC1920A0640000000004A
:10BA9000B5EE400A08B5F1EE10FA2DED048BB0EECC
:10BAA000408A25D0B7EE009AB4EE490AF1EE10FABA
:10BAB00019D0FAEE040A60EE200AB0EE000A46F051
:10BAC00009FBB2EE047AFEEE087AF0EE408A9FEDB2
:10BAD0000A0AE8EE077AB0EE498A27EE800A46F0B5
:10BAE000D7F8A8EE808AB0EE480ABDEC048B08BDFA
:10BAF0009FED028AF7E700BF920A064000000000AF
:10BB0000B5EE400A08B5F1EE10FA2DED088BB0EE57
:10BB1000408A45D0F7EE00AAB4EE6A0AF1EE10FAB8
:10BB200020D0F6EE009ADFED208AB3EE04AA9FED56
:10BB30001FBAB4EEE90AF1EE10FA18D5FAEE040ACB
:10BB4000E0EE0A0AB0EE000A46F0C4FAE8EE0A8A0D
:10BB5000B0EE409A28EE8B0A46F09AF820EE490A99
:10BB600020EE298AB0EE480ABDEC088B08BDFBEE3A
:10BB7000047AF2EE040AE0EE270AB0EE000A46F07C
:10BB8000A9FAE8EE0A8AB0EE409AB0EE6A8A28EE88
:10BB90008B0A46F07DF829EE000AA0EE298AE1E73B
:10BBA0009FED038ADEE700BF000032C1C3B8B23F99
:10BBB0000000000008B52DED028BB6EE008AF7EE0E
:10BBC000008AB4EEC80AF1EE10FA1CD570EE007AC5
:10BBD00017EE900AF4F7E2FC02460B46F4F736FD46
:10BBE00002460B4600200F49F4F778FBF5F726F8DC
:10BBF00000EE100A46F0C6FA38EEC00A20EE080A37
:10BC0000BDEC028B08BDB8EE007AF0EE007AE0EEF3
:10BC1000077AB0EE680AA7EEE70A46F0B3FA30EE0C
:10BC2000280AEBE70000F03FF7EE007A08B577EE60
:10BC3000C07A17EE900AF4F7B1FC9FED091B41ECB6
:10BC4000100B46F04FF90020074953EC102BF4F786
:10BC500045FBF4F7F3FF00EE100A08BDAFF30080D8
:10BC600000000000000008400000F03F30EE600AD5
:10BC700032EE412A71EEE00A20EE020AC0EE207A8E
:10BC800037EE810A7047B4EEE00AF1EE10FA06D4FE
:10BC9000B4EE410AF1EE10FA31FE000A7047B0EE40
:10BCA000600A704738B50D46044611462A464CF0E6
:10BCB000F2FE6119002301F8013C38BD8B4270B5DA
:10BCC00028BF0B46164605461A4631461C464CF020
:10BCD000E2FE00232B5570BD37B50C460192054698
:10BCE000F4F7F0FA631E1A1A06D40199284603B035
:10BCF000BDE830404CF0A8BE03B030BD37B50446B7
:10BD00000D460192F4F7DEFA019B291A034A2044FA
:10BD100003B0BDE830404BF0B1BE00BFBA11060819
:10BD200037B504460D460192F4F7CCFA019B291A67
:10BD3000034A204403B0BDE830404BF09FBE00BF33
:10BD40003C080608F7B50D4617461E460446F4F7AC
:10BD5000B9FA044A291A2044CDE900764BF08EFE48
:10BD600003B0F0BD40080608F7B50D4617461E465D
:10BD70000446F4F7A7FA044A291A2044CDE90076CC
:10BD80004BF07CFE03B0F0BD44080608E3B50E4658
:10BD900010EE107A0546F4F795FA361A054438463F
:10BDA000F4F7FCFB044ACDE90001314628464BF08C
:10BDB00065FE02B0E0BD00BF48080608EFB50E46BC
:10BDC00010EE107A05460392F4F77CFA361A054411
:10BDD0003846F4F7E3FB039B044ACDE90001314602
:10BDE00028464BF04BFE04B0E0BD00BF4B080608F0
:10BDF00030B50D4604462DED028BB0EE408AF0EED4
:10BE0000608A83B0F4F75EFA054A291A20448DED62
:10BE1000008B4BF033FE03B0BDEC028B30BD00BF96
:10BE20004808060830B50D4604462DED028BB0EEED
:10BE3000408AF0EE608A85B00392F4F743FA039BE0
:10BE4000291A054A20448DED008B4BF017FE05B0F2
:10BE5000BDEC028B30BD00BF4B080608B7EE007A80
:10BE6000C7EE207A27EE800AB8FE400A80EE270A45
:10BE70007047B4EE400AF1EE10FA14BF0120002022
:10BE8000704708B553EC102B10EE100A1946F4F762
:10BE900045FEB0FA80F0400908BDC3B2092894BF3E
:10BEA00003F1300003F13700C0B27047904210B583
:10BEB0000CDB029C2244824208DD994206DB039897
:10BEC00003448B42D4BF0020012010BD0020FCE7BA
:10BED00082B041788278C37800788DF805108DF8AB
:10BEE00004008DF806208DF80730019802B07047E5
:10BEF0002DE9F7430DF1040C03460144904600265A
:10BF000060464FF00A0E99420BD100202FE0B94253
:10BF10000AD1032EF9D1FF2DF7D8A142F5D10B4656
:10BF20001BE01F4600231D463C4617F8012BA2F1DB
:10BF30003009B9F1090F1DD801330EFB05253C4628
:10BF4000032BA5F13005E2D1FF2DDED8032EE4D07E
:10BF5000234613F8012B2E2AD7D101360CF8015BAA
:10BF6000042ED0D1FFF7B4FFC8F80000012003B0C1
:10BF7000BDE8F083002BC8D02E2AE5D0C5E700002D
:10BF80001FB50346084611461A0E0292C3F3074234
:10BF90000192C3F30722DBB20092034A4BF06EFD1D
:10BFA00005B05DF804FB00BF5008060837B504462D
:10BFB00008461146002C05D10D4A03B0BDE83040BB
:10BFC000FFF770BED8BF64424FF06405D6BF2D2383
:10BFD0002B2324B294FBF5F205FB124412B224B2D7
:10BFE0000092044A01944BF049FD03B030BD00BFFC
:10BFF000680806085C080608704710B50446142156
:10C000002BF061F8204610BD4388DB0710B50DD535
:10C0100084686368013B636043B9236820461B68FA
:10C0200098472046BDE81040FFF742B810BD000019
:10C0300038B555EC104B16A3D3E9002310EE100AC7
:10C040002946F4F77FFD98B92046294612A3D3E983
:10C050000023F4F745F912A3D3E90023F4F720FCF9
:10C060009FED091BBDE8384041EC100B45F03ABF8D
:10C070000DA3D3E9002320462946F4F711FC41EC37
:10C08000100B38BDAFF30080333333333333034009
:10C0900012143FC6DCB5A43F295C8FC2F528AC3F23
:10C0A000E17A14AE47E1F03FD7A3703D0AD72940AB
:10C0B000C36A2DE9F04353F8214005460E462DEDA5
:10C0C000048B91B0002C40F091807E4B4FF47F4761
:10C0D0004FF000084FF000090093224604AB019492
:10C0E0000497CDE90244CDE9068903F09BF80028C6
:10C0F00043D0754B012231462846009308AB01948A
:10C100000897CDE90244CDE90A8903F08BF888B39A
:10C110006E4B02223146284600930CAB01940C97DB
:10C12000CDE90244CDE90E8903F07CF8F8B121464F
:10C1300004A80CF023F8214608A8B0EE409A0CF0B1
:10C140001DF821460CA8F0EE408A0CF017F8B5EE69
:10C15000400AB0EE408AF1EE10FA16D12846C5ED3D
:10C160000D8A02F031FC3146284609F00AFA0CA883
:10C17000FFF74AFF08A8FFF747FF04A8FFF744FFAF
:10C1800011B0BDEC048BBDE8F083EB6A53F82630A8
:10C190001BB13146284608F0D2FF4D491420FEF766
:10C1A0004DFF4C4B044631460360EB6A43F82600D2
:10C1B000284602F05DFC84ED019AC4ED028A84ED0C
:10C1C000038AFFF7E3F84FF0FF33012120611A469D
:10C1D0002846CDE90031314609F036FC0028C6D1A9
:10C1E0003D4A3146284609F087F8C0E794ED018AB8
:10C1F000D4ED027A94ED039AB4EEE78ADFED378A44
:10C20000F1EE10FA2FD5FFF7C1F82369C31A07EE34
:10C21000903AF8EE677A67EE897A87EEA87AD4EDDD
:10C22000027A37EE088AF4EE487AF1EE10FA98BFF7
:10C23000B0EE678A284685ED0D8A02F0C5FBD4ED85
:10C24000027AF4EE487AF1EE10FA23D1314628460C
:10C2500008F075FF3146284611B0BDEC048BBDE8EF
:10C26000F04309F08EB9FFF791F82369C31A07EE7E
:10C27000903AF8EE677A67EE897A87EEA87AD4ED7D
:10C28000027A38EE478AF4EE487AF1EE10FA27FE89
:10C29000888ACFE74FF0FF33012231462846CDE9A7
:10C2A00000321A4609F0D0FB00287FF469AF0A4A31
:10C2B0003146284611B0BDEC048BBDE8F04309F0CF
:10C2C0001BB800BF6C0806088F080608B0080608EF
:10C2D000F43BDC72F8080608D408060800007A442B
:10C2E0002DE9F84F524B1A6802F1010ABAF1010F19
:10C2F000C3F800A04BD14F4B002200244E4D9B466B
:10C300001A80A3F800220FF21819D9E900895046C3
:10C310000AF1010AF4F730F942464B4606460F4649
:10C32000F4F7BEFA0BF1020B41EC100BFFF780FEA5
:10C330003DA3D3E9002351EC100BF4F787F9224613
:10C340002B46F3F7CDFFF4F759FC2246ABF800007B
:10C350002B4630463946F3F7C1FF42464B46F4F7C9
:10C360009FFA41EC100BFFF763FE2FA3D3E90023E4
:10C3700051EC100BF4F76AF922462B46F3F7B0FFA5
:10C38000F4F73CFCBAF5807FABF80002BFD12B4A32
:10C39000136803F1010ABAF1010FC2F800A03AD103
:10C3A000274B00224FF00008DFF88C9003F58061E6
:10C3B00003F1040B1A600A6019A7D7E90067504619
:10C3C0000AF1010AF4F7C8F832463B4604460D4626
:10C3D000F4F766FA41EC100BFFF72AFE51EC100B54
:10C3E000F4F72CFC42464BF8040B4B4620462946FA
:10C3F000F3F774FF32463B46F4F752FA41EC100B68
:10C40000FFF716FE51EC100BF4F718FCBAF5807F1D
:10C41000CBF8FC03D3D1BDE8F88F00BFAFF30080A9
:10C420000000000000E06F4000000000E0FFEF406F
:10C43000D0260220D42E02200000E03FCC2602208D
:10C44000D4260220044B10B504460360406808F06F
:10C450008BFE204610BD00BF5009060810B50446EB
:10C46000FFF7F0FF082120462AF02DFE204610BDE0
:10C47000F8B5836804460D4616461868904208DCF5
:10C48000101A0FF079FC29462046BDE8F84009F063
:10C4900078B8E36A53F821703FB10121786808F059
:10C4A00020FE80B1786808F05FFE21462A463046BB
:10C4B00009F0D8F90121074608F013FE50B13846BB
:10C4C00008F052FEDFE7294620460E4ABDE8F84054
:10C4D00008F012BFE36A53F825301BB12946204605
:10C4E00008F02DFE08490820FEF7A8FD074B064678
:10C4F00029460360E36A43F82500204602F0B8FAB3
:10C500007760F8BD00090608F43BDC7250090608A4
:10C51000C3685B6853F82130B3F92020002A02DA9F
:10C52000024A08F0E9BEFFF7A3BF00BF1F090608D3
:10C530002DE9F84F524B1A6802F1010ABAF1010FC6
:10C54000C3F800A04BD14F4B002200244E4D9B4618
:10C550001A80A3F800220FF21819D9E90089504671
:10C560000AF1010AF4F708F842464B4606460F4620
:10C57000F4F796F90BF1020B41EC100BFFF758FDA5
:10C580003DA3D3E9002351EC100BF4F75FF82246EA
:10C590002B46F3F7A5FEF4F731FB2246ABF800007B
:10C5A0002B4630463946F3F799FE42464B46F4F7A0
:10C5B00077F941EC100BFFF73BFD2FA3D3E90023E4
:10C5C00051EC100BF4F742F822462B46F3F788FEA5
:10C5D000F4F714FBBAF5807FABF80002BFD12B4A09
:10C5E000136803F1010ABAF1010FC2F800A03AD1B1
:10C5F000274B00224FF00008DFF88C9003F5806194
:10C6000003F1040B1A600A6019A7D7E900675046C6
:10C610000AF1010AF3F7A0FF32463B4604460D46F5
:10C62000F4F73EF941EC100BFFF702FD51EC100B53
:10C63000F4F704FB42464BF8040B4B4620462946D0
:10C64000F3F74CFE32463B46F4F72AF941EC100B67
:10C65000FFF7EEFC51EC100BF4F7F0FABAF5807F1F
:10C66000CBF8FC03D3D1BDE8F88F00BFAFF3008057
:10C670000000000000E06F4000000000E0FFEF401D
:10C68000D0260220D42E02200000E03FCC2602203B
:10C69000D426022038B5C36A04460D46012253F859
:10C6A0002130083308F002FF2946204608F047FDF4
:10C6B00029462046BDE8384008F063BFC3685B6880
:10C6C000F0B553F821208FB04FF47F4300260027A8
:10C6D00020320693002304460D460193CDE9023330
:10C6E000174B009306ABCDE9086702F025FDB8B102
:10C6F00005A906A80CF082FD059BD3B94FF602737D
:10C700000A9390B101220AAB0C922946204608F008
:10C71000CDFE0AA8FFF778FC2946204608F031FF35
:10C7200006A8FFF771FC0FB0F0BD0AAB02220C9017
:10C73000EBE7044A2946204608F0DEFDF0E700BF9B
:10C74000580906088009060838B5D0E902320446BF
:10C750000D465268DB6852F82120128C53F82230C3
:10C76000012208F0A3FE29462046BDE8384008F023
:10C7700008BF704710B5044608212AF0A4FC2046E3
:10C7800010BD0000C36A70B553F8214088B005465B
:10C790000E46002C36D14FF47F43002201940493BF
:10C7A0000023CDE90623234B2246009304ABCDE9B9
:10C7B000024402F037FD20B904A8FFF725FC08B0B9
:10C7C00070BDEB6A53F826301BB13146284608F09D
:10C7D000B6FC19490820FEF731FC184B04463146D7
:10C7E0000360EB6A43F82600284602F041F99DF801
:10C7F000103004A81B2B0CBFBDF81830069B6360DB
:10C80000FFF702FC6368002B08DD013B3146284638
:10C81000636008B0BDE8704008F0B3BE31462846FA
:10C8200008F08DFC01223146284608B0BDE8704072
:10C8300008F0A2BEAE090608F43BDC72E009060867
:10C84000704710B5044608212AF03DFC204610BD73
:10C85000C36AF0B553F8216004460D462DED028BF6
:10C8600089B0002E5AD14FF47F43002201960493E1
:10C870000023CDE906233D4B3246009304ABCDE9BE
:10C88000026602F0CFFC002841D0314604A80BF02C
:10C89000F3FBB0EE408AF0EE608AFFF7F2FA88BB55
:10C8A000E36A53F825301BB12946204608F047FCBF
:10C8B0002F490820FEF7C2FB2E4B2946064603608F
:10C8C000E36A43F82500204602F0D2F8FEF75EFD49
:10C8D000B0EE480AF0EE680A074644F0EDFF51EC6E
:10C8E000100BF4F78BF94FF0FF33384401211A464F
:10C8F00070602046CDE90031294609F0A5F830B92D
:10C900001D4A00E01D4A2946204608F0F5FC04A80F
:10C91000FFF77AFB09B0BDEC028BF0BDFEF736FDE8
:10C92000736898420CD32946204608F008FC294633
:10C93000204609B0BDEC028BBDE8F04008F021BEF6
:10C940004FF0FF33012229462046CDE900321A4636
:10C9500009F07AF80028DDD1074A2946204609B0B7
:10C96000BDEC028BBDE8F04008F0C6BCE809060843
:10C97000F43BDC72400A0608D4080608110A0608CF
:10C98000C3692BB1827C1AB1416A184608F0F9BD1F
:10C99000014B1B68184700BF5C02002030B54FF404
:10C9A0007F4389B0002204460493002301920D4680
:10C9B000CDE906230A4BCDE90222009304AB02F035
:10C9C00031FC20B904A8FFF71FFB09B030BD04A853
:10C9D0000BF060FD29460246204608F08DFCF1E789
:10C9E000480A060830B54FF47F4389B00022044658
:10C9F0000493002301920D46CDE906230B4BCDE9AC
:10CA00000222009304AB02F00DFC20B904A8FFF74A
:10CA1000FBFA09B030BD2946204604AB012208F0DC
:10CA200045FD2946204608F0ACFDEFE76C0A0608F4
:10CA3000044B10B5044640F8083BFFF7E5FA2046E2
:10CA400010BD00BF280B060810B50446FFF7F0FF25
:10CA5000182120462AF037FB204610BD38B50D4678
:10CA60000446FFF7D1FA2B7823706B7863706A88DD
:10CA70006280AB68A360EB68E360D30741BFA26844
:10CA800053680133536038BDF8B5C4680346C769BD
:10CA90000E46656827B91A4A08F02EFC0020F8BD3A
:10CAA000046A0CB9174AF7E755F8211094F8225098
:10CAB00091F82000B1F800C040F2EB318C4561687C
:10CAC0000ABF2D180025EDB28D4203D30E4A314620
:10CAD0001846E1E79868A16840683C8A31F815106B
:10CAE00050F824000069814201D3084AEFE7BB6A8D
:10CAF000104603EB0111FFF7B1FF0120CFE700BFA4
:10CB0000960A0608B30A0608D00A0608EE0A0608BE
:10CB10002DE9F04385B04FF47F474FF000084FF008
:10CB200000096A4605460E460097CDE90289FFF7DF
:10CB3000ABFFF8B1EB6A53F8264084B910491820CE
:10CB4000FEF77CFA0F4B8760044603603146EB6AC0
:10CB5000C0E9048943F82600284601F089FF3146E0
:10CB600028466B46002208F0A1FC694604F1080043
:10CB7000FFF774FF6846FFF747FA05B0BDE8F0839A
:10CB8000F43BDC72280B060830B54FF47F438FB0BE
:10CB9000002204460693002301920D46CDE90823A6
:10CBA000174BCDE90222009306AB02F03BFBB8B174
:10CBB00005A906A80CF022FB059BD3B94FF602731A
:10CBC0000A9390B101220AAB0C922946204608F044
:10CBD0006DFC0AA8FFF718FA2946204608F0D1FC98
:10CBE00006A8FFF711FA0FB030BD0AAB02220C9075
:10CBF000EBE7044A2946204608F07EFBF0E700BF39
:10CC0000300B060880090608F8B50D4604461146A3
:10CC100002462B46406808F030FEE36A074653F8A8
:10CC200025301BB12946204608F089FA084908201A
:10CC3000FEF704FA074B064629460360E36A43F809
:10CC40002500204601F014FF30467760F8BD00BF94
:10CC5000F43BDC725C0B0608044B10B50446036021
:10CC6000406808F081FA204610BD00BF5C0B060842
:10CC700010B50446FFF7F0FF082120462AF023FAFA
:10CC8000204610BD08B5C36A53F8213013B9FFF729
:10CC9000BBFF0346586808BDC26A2DE9F04752F849
:10CCA00021602DED028B86B06EB9C3685B6853F8C6
:10CCB000213089B2B3F9202006B0BDEC028BBDE86B
:10CCC000F047FFF7A1BF9FED3E8B7768002440F24D
:10CCD000EB39DFF8F4A0FB681A68A24268D95B68F8
:10CCE00053F824301B884B4541D1FB6A53F824503C
:10CCF00075B34FF47F4302AA2146384602938DED67
:10CD0000048BFFF7C1FE00284FD02A7A05F10808EE
:10CD10009DF8083093421DD04FF0FF3300211A4692
:10CD2000CDE900312146706808F08EFE4046FFF7DD
:10CD30006BF9029BBDF80A20AB6004AB03CBC8F8CB
:10CD40000800D007C8F80C100CD402A8FFF75CF953
:10CD50000134C0E75AF8233002A94046984700281A
:10CD6000F3D1D9E72A69536801335360EDE740F204
:10CD7000E9329342ECD14FF47F4302AA2146384670
:10CD800002938DED048BFFF77FFE70B19DF80830A4
:10CD9000002BDAD04FF0FF3300222146CDE90032DC
:10CDA0001A46706808F050FECFE702A8FFF72CF98A
:10CDB00006B0BDEC028BBDE8F08700BFAFF300808A
:10CDC00000000000000000004804002030B54FF4CF
:10CDD0007F438DB0002204460493002301920D4648
:10CDE000CDE90623124BCDE90222009304AB02F0F9
:10CDF00019FA20B904A8FFF707F90DB030BD0D4AA4
:10CE000004A908A80CF028F908A80BF043FB024677
:10CE100028B103781BB12946204601F0DFFE2046E9
:10CE2000294608F0AEFB08A8FFF7EEF8E2E700BFDE
:10CE3000640B0608EE12980F30B54FF47F420024C1
:10CE400000250260C0E9024530BD0000084B10B566
:10CE5000044640F8283BFFF7D7F804F11800FFF725
:10CE6000D3F804F10800FFF7CFF8204610BD00BF4B
:10CE7000100C060810B50446FFF7E8FF38212046DD
:10CE80002AF021F9204610BD38B50D460446FFF7BB
:10CE9000BBF82B7823706B7863706A886280AB680C
:10CEA000A360EB68E360D30741BFA2685368013316
:10CEB000536038BDC368826A5B682DE9F04753F858
:10CEC000218094B0C36A05460E4653F82140D8F835
:10CED00008301B881B01D35C002B50D014B10024F8
:10CEE00008F02DF904A8FFF7A7FF0023032231461D
:10CEF00001932846CDE90233614B009304AB02F065
:10CF000091F9002837D0002C40F09E8008A8FFF748
:10CF100093FF5C4B224631460093284608ABCDE98F
:10CF2000014402F0C5F918B30CA8FFF785FF564B72
:10CF300001223146009328460CAB0194CDE902440E
:10CF400002F070F988B110A8FFF776FF4F4B02226C
:10CF500031460093284610AB0194CDE9024402F01B
:10CF600061F988B910A8FFF74FF80CA8FFF74CF843
:10CF700008A8FFF749F804A8FFF746F801E0002CDD
:10CF8000B0D114B0BDE8F087EB6A53F826301BB17E
:10CF90003146284608F0D3F83D493820FEF74EF8D0
:10CFA00004463C4B074604F1180A04F1280947F8E7
:10CFB000083B3846FFF740FF5046FFF73DFF484625
:10CFC000FFF73AFFEB6A3146284643F8264001F066
:10CFD0004FFD08A93846FFF757FF10A95046FFF745
:10CFE00053FF0CA94846FFF74FFF10A8FFF70CF8B6
:10CFF0000CA8FFF709F808A8FFF706F89DF810300D
:10D0000004F1280904F118021B2B10A849460CBF93
:10D01000BDF81830069B002B23DD05F012F8002127
:10D0200010A80CF0EBF8074610A8FEF7EDFFDFB1F3
:10D030003146284608F083F8D8F8142031462846AF
:10D04000013A08F099FA96E704F1280704AA10A813
:10D05000394604F07BF9384610A9FFF715FF10A8F0
:10D06000CAE704F0E2FFDAE7314628464B4604F10E
:10D07000080208F09BFA3146284608F082FA7AE75F
:10D08000860B0608A60B0608CA0B0608EA0B06085C
:10D09000F43BDC72100C060808F073BA08F071BAA1
:10D0A0002DE9F043C26885B0C56904460E46536851
:10D0B0002DB9284A05B0BDE8F04308F01DB9076A4C
:10D0C0000FB9254AF6E753F821C01269DCF8083099
:10D0D0001B88934201D3214AECE7826A19014FF47D
:10D0E0007F404FF000084FF0000902EB031300905F
:10D0F000B3F802E0CDE90289525C1EF0010F986896
:10D100008DF800205A78D9688DF8012002AAADF870
:10D1100002E003C21FBF02465368013353609CF80C
:10D12000203097F823201A447B69D2B29A420AD35E
:10D130000B4A3146204608F0DFF86846FEF764FFE8
:10D1400005B0BDE8F0836B46616A284608F0AEF989
:10D15000F3E700BF180C0608360C0608540C060846
:10D16000730C0608704710B50446082129F0ABFF80
:10D17000204610BDC368826A5B6853F821309B6803
:10D180001B881B0170B5D35C05460E469BB1C36A74
:10D1900053F821406CB908490820FDF74FFF074BB1
:10D1A000044631460360EB6A43F82600284601F046
:10D1B0005FFC0123237170BDF43BDC72AC0C0608EC
:10D1C0002DE9F0414FF47F43CAB0002200240693BA
:10D1D0000023019405460E46CDE908231A4B22464A
:10D1E000009306ABCDE9024402F01CF8B8B106A8E2
:10D1F0000BF050F96A680346D2E91087444516D00F
:10D2000057F82420194605931068F3F751F8059B49
:10D2100058B90E4B314628461C6008F0B2F906A8F2
:10D22000FEF7F2FE4AB0BDE8F0810134E6E7084AB5
:10D230004FF480710AA84AF021FC0AAA3146284618
:10D2400008F05AF8EBE700BFB40C06089834022047
:10D25000E20C060838B5C36804460D465B6853F80F
:10D26000213093F820305A1E53425341044A137020
:10D2700011F01AFD29462046BDE8384008F081B972
:10D2800075700220000000002DE9F84F524B1A681B
:10D2900002F1010ABAF1010FC3F800A04BD14F4BC4
:10D2A000002200244E4D9B461A80A3F800220FF264
:10D2B0001819D9E9008950460AF1010AF3F75CF917
:10D2C00042464B4606460F46F3F7EAFA0BF1020BCD
:10D2D00041EC100BFEF7ACFE3DA3D3E9002351EC6B
:10D2E000100BF3F7B3F922462B46F2F7F9FFF3F7E9
:10D2F00085FC2246ABF800002B4630463946F2F753
:10D30000EDFF42464B46F3F7CBFA41EC100BFEF72C
:10D310008FFE2FA3D3E9002351EC100BF3F796F9FE
:10D3200022462B46F2F7DCFFF3F768FCBAF5807F64
:10D33000ABF80002BFD12B4A136803F1010ABAF11E
:10D34000010FC2F800A03AD1274B00224FF000088D
:10D35000DFF88C9003F5806103F1040B1A600A601A
:10D3600019A7D7E9006750460AF1010AF3F7F4F864
:10D3700032463B4604460D46F3F792FA41EC100B59
:10D38000FEF756FE51EC100BF3F758FC42464BF8F3
:10D39000040B4B4620462946F2F7A0FF32463B4697
:10D3A000F3F77EFA41EC100BFEF742FE51EC100B46
:10D3B000F3F744FCBAF5807FCBF8FC03D3D1BDE88A
:10D3C000F88F00BFAFF300800000000000E06F4066
:10D3D00000000000E0FFEF40D0260220D42E022003
:10D3E0000000E03FCC260220D426022000000000EE
:10D3F000C3685B682DE9F04F2DED028B9FED328BFA
:10D40000CDB004460D4653F821800026DFF8C4B0A5
:10D41000D8F82030B3424ED9D8F824304FF4807178
:10D420002B4A0CA853F8269001364FF47F4A002768
:10D4300033464AF023FB0CABCDF810A029460093ED
:10D44000204604ABCDE90177D9F800208DED068B9D
:10D4500001F0B4FED0B133465A464FF480710CA8A7
:10D460004AF00CFB0CAB019729460093204608AB11
:10D47000CDF820A0CDE90277D9F804208DED0A8BF4
:10D4800001F05AFE50B908A8FEF7BEFD04A8FEF749
:10D49000BBFD4DB0BDEC028BBDE8F08F08AB04AA1C
:10D4A0002946204608F082F808A8FEF7ADFD04A83A
:10D4B000FEF7AAFDACE7294620464DB0BDEC028B35
:10D4C000BDE8F04F08F05DB800000000000000006B
:10D4D000F60C0608280D060830B54FF47F4385B0DA
:10D4E0000D4C00220D4D0093002329682068CDE9E2
:10D4F00002236B46012207F0D9FF6846FEF784FD40
:10D50000002029F0C9F808F0F1FD2968206805B06D
:10D51000BDE8304007F0BEBED4320220D83202202F
:10D52000F0B5104C85B0104D0146266868462F684E
:10D530004FF0FF320D4B0BF049FD39466B46002290
:10D54000304607F0B3FF6846FEF75EFD002029F085
:10D55000A3F808F0CBFD2968206805B0BDE8F040CD
:10D5600007F098BED4320220D8320220E22FD387AF
:10D5700038B50D460446FEF747FD2B7823706B78CF
:10D5800063706A886280AB68A360EB68E360D3076E
:10D5900041BFA26853680133536038BD4FF47F43E5
:10D5A000002210B5036000230446C0E90223FFF700
:10D5B000DFFF204610BD0000C3685B682DE9F0471F
:10D5C00053F82170A4B00024524B4FF47F4A4FF01F
:10D5D00000084FF000090093224604AB0194054671
:10D5E0000E46CDF810A0CDE90244CDE9068901F040
:10D5F00019FE002838D0484B0122314628460093B6
:10D6000008AB0194CDF820A0CDE90244CDE90A8908
:10D6100001F008FE28B3414B022231462846009310
:10D620000CAB0194CDF830A0CDE90244CDE90E89D0
:10D6300001F0F8FD90B13A4B0322314628460093A1
:10D6400010AB0194CDF840A0CDE90244CDE9128998
:10D6500001F0E8FD70B910A8FEF7D6FC0CA8FEF7A3
:10D66000D3FC08A8FEF7D0FC04A8FEF7CDFC24B03C
:10D67000BDE8F0872B4B284631461D602A4B1E60C3
:10D6800007F0FAFD04A80AF005FFA8B103789BB1E2
:10D690004FF60D731CAA04A920A81C93234B1E93BC
:10D6A00003F054FE20A904A8FFF762FF20A8FEF7AC
:10D6B000ABFC1CA8FEF7A8FC1D4B04A914A81C6811
:10D6C000FFF76CFF08A918A8FFF768FF0CA91CA8B2
:10D6D000FFF764FF10A920A8FFF760FF154B1CAAF5
:10D6E00018A9029314A8144B019397F82030003B1B
:10D6F00018BF0123009320ABA04720A8FEF784FCAD
:10D700001CA8FEF781FC18A8FEF77EFC14A8FEF703
:10D710007BFCA0E7570D0608800D0608AF0D060834
:10D72000DB0D0608D4320220D8320220FF1D060885
:10D7300064020020D9D4000821D5000800000000B0
:10D740002DE9F84F524B1A6802F1010ABAF1010FA4
:10D75000C3F800A04BD14F4B002200244E4D9B46F6
:10D760001A80A3F800220FF21819D9E9008950464F
:10D770000AF1010AF2F700FF42464B4606460F4601
:10D78000F3F78EF80BF1020B41EC100BFEF750FC97
:10D790003DA3D3E9002351EC100BF2F757FF2246CB
:10D7A0002B46F2F79DFDF3F729FA2246ABF800006D
:10D7B0002B4630463946F2F791FD42464B46F3F789
:10D7C0006FF841EC100BFEF733FC2FA3D3E90023D5
:10D7D00051EC100BF2F73AFF22462B46F2F780FD90
:10D7E000F3F70CFABAF5807FABF80002BFD12B4AF1
:10D7F000136803F1010ABAF1010FC2F800A03AD18F
:10D80000274B00224FF00008DFF88C9003F5806171
:10D8100003F1040B1A600A6019A7D7E900675046A4
:10D820000AF1010AF2F798FE32463B4604460D46DD
:10D83000F3F736F841EC100BFEF7FAFB51EC100B46
:10D84000F3F7FCF942464BF8040B4B4620462946B9
:10D85000F2F744FD32463B46F3F722F841EC100B59
:10D86000FEF7E6FB51EC100BF3F7E8F9BAF5807F11
:10D87000CBF8FC03D3D1BDE8F88F00BFAFF3008035
:10D880000000000000E06F4000000000E0FFEF40FB
:10D89000D0260220D42E02200000E03FCC26022019
:10D8A000D426022070B50F4C86B00F4D266802A812
:10D8B00029680191FFF7C0FA019902AB01223046B5
:10D8C00007F0F4FD02A8FEF79FFB002028F0E4FE1D
:10D8D00008F00CFC2968206806B0BDE8704007F02D
:10D8E000D9BC00BFDC320220E032022070B52DED41
:10D8F000028B92B00024B0EE408A2D4E06A82D4D2A
:10D90000FFF79AFA2C4B04223168009306AB286883
:10D910000194CDE9024401F085FCB8B1214606A886
:10D920000AF02CFC0AA8F0EE408AFFF785FA234B98
:10D930000522316800930AAB28680194CDE90244BE
:10D9400001F070FC48B90AA8FEF75EFB06A8FEF7D6
:10D950005BFB12B0BDEC028B70BD0AA80AF09AFD09
:10D96000FDF734FDF0EE680AB0EE480A0590FEF7C8
:10D9700075FAB0EE408A0598FDF744FD4FF60B733B
:10D98000C8EE007A3168224628680E930EABCDEDC2
:10D99000107A07F08BFD0EA8FEF736FB204628F024
:10D9A0007BFE08F0A3FB3168286807F073FCCAE728
:10D9B000E0320220DC320220070E0608320E060892
:10D9C00038B50D460446FEF71FFB2B7823706B78A5
:10D9D00063706A886280AB68A360EB68E360D3071A
:10D9E00041BFA26853680133536038BD70B5A8B019
:10D9F000054600240E4604A8FFF71EFA554B2246A2
:10DA000031460093284604AB0194CDE9024401F06D
:10DA100009FC002848D008A8FFF70EFA4E4B012257
:10DA200031460093284608AB0194CDE9024401F049
:10DA3000F9FB002835D00CA8FFF7FEF9474B02226E
:10DA40003146009328460CAB0194CDE9024401F025
:10DA5000E9FB18B310A8FFF7EFF9414B0322314659
:10DA60000093284610AB0194CDE9024401F0DAFBA3
:10DA700088B114A8FFF7E0F93A4B0522314600932C
:10DA8000284614AB0194CDE9024401F0CBFB80B9E8
:10DA900014A8FEF7B9FA10A8FEF7B6FA0CA8FEF71C
:10DAA000B3FA08A8FEF7B0FA04A8FEF7ADFA28B05A
:10DAB00070BD2D4B284631461D602C4B1E6007F073
:10DAC000DBFB04A80AF0E6FCA8B103789BB14FF693
:10DAD0000D7320AA04A924A82093254B229303F0B8
:10DAE00035FC24A904A8FFF76BFF24A8FEF78CFAE5
:10DAF00020A8FEF789FA14A80AF0CCFCFDF766FC12
:10DB00001C4B044604A918A81D68FFF747FD08A987
:10DB10001CA8FFF743FD0CA920A8FFF73FFD10A9A3
:10DB200024A8FFF73BFD144B20AA1CA9029318A8B8
:10DB3000124BCDE9004324ABA84724A8FEF764FAB2
:10DB400020A8FEF761FA1CA8FEF75EFA18A8FEF7F7
:10DB50005BFA9DE7580E06087F0E0608AD0E060814
:10DB6000D20E0608320E0608DC320220E032022015
:10DB7000FF1D060858020020A5D80008EDD80008AF
:10DB80002DE9F84F524B1A6802F1010ABAF1010F60
:10DB9000C3F800A04BD14F4B002200244E4D9B46B2
:10DBA0001A80A3F800220FF21819D9E9008950460B
:10DBB0000AF1010AF2F7E0FC42464B4606460F46E0
:10DBC000F2F76EFE0BF1020B41EC100BFEF730FA90
:10DBD0003DA3D3E9002351EC100BF2F737FD2246A9
:10DBE0002B46F2F77DFBF3F709F82246ABF800006D
:10DBF0002B4630463946F2F771FB42464B46F2F768
:10DC00004FFE41EC100BFEF713FA2FA3D3E90023CC
:10DC100051EC100BF2F71AFD22462B46F2F760FB8F
:10DC2000F2F7ECFFBAF5807FABF80002BFD12B4AC8
:10DC3000136803F1010ABAF1010FC2F800A03AD14A
:10DC4000274B00224FF00008DFF88C9003F580612D
:10DC500003F1040B1A600A6019A7D7E90067504660
:10DC60000AF1010AF2F778FC32463B4604460D46BB
:10DC7000F2F716FE41EC100BFEF7DAF951EC100B3F
:10DC8000F2F7DCFF42464BF8040B4B462046294690
:10DC9000F2F724FB32463B46F2F702FE41EC100B52
:10DCA000FEF7C6F951EC100BF2F7C8FFBAF5807F0A
:10DCB000CBF8FC03D3D1BDE8F88F00BFAFF30080F1
:10DCC0000000000000E06F4000000000E0FFEF40B7
:10DCD000D0260220D42E02200000E03FCC260220D5
:10DCE000D4260220C36800225B6830B553F8215067
:10DCF0008DB04FF47F430024049300230194CDE9B9
:10DD00000623184B2246009304ABCDE9024401F0F0
:10DD100089FA20B904A8FEF777F90DB030BD95F85F
:10DD20002030012B0FD1204628F0B6FC044604A970
:10DD300008A8FFF733FC08A9204608F053FC08A800
:10DD4000FEF762F9E6E7022BE4D1204628F0A4FCB6
:10DD5000044604A908A8FFF721FC08A9204608F0FA
:10DD600054FCECE7F70E06082DE9F84F524B1A6801
:10DD700002F1010ABAF1010FC3F800A04BD14F4BD9
:10DD8000002200244E4D9B461A80A3F800220FF279
:10DD90001819D9E9008950460AF1010AF2F7ECFB9B
:10DDA00042464B4606460F46F2F77AFD0BF1020B50
:10DDB00041EC100BFEF73CF93DA3D3E9002351ECF5
:10DDC000100BF2F743FC22462B46F2F789FAF2F7E2
:10DDD00015FF2246ABF800002B4630463946F2F7D5
:10DDE0007DFA42464B46F2F75BFD41EC100BFEF725
:10DDF0001FF92FA3D3E9002351EC100BF2F726FCF7
:10DE000022462B46F2F76CFAF2F7F8FEBAF5807F5D
:10DE1000ABF80002BFD12B4A136803F1010ABAF133
:10DE2000010FC2F800A03AD1274B00224FF00008A2
:10DE3000DFF88C9003F5806103F1040B1A600A602F
:10DE400019A7D7E9006750460AF1010AF2F784FBE7
:10DE500032463B4604460D46F2F722FD41EC100BDC
:10DE6000FEF7E6F851EC100BF2F7E8FE42464BF8ED
:10DE7000040B4B4620462946F2F730FA32463B4621
:10DE8000F2F70EFD41EC100BFEF7D2F851EC100B3F
:10DE9000F2F7D4FEBAF5807FCBF8FC03D3D1BDE80E
:10DEA000F88F00BFAFF300800000000000E06F407B
:10DEB00000000000E0FFEF40D0260220D42E022018
:10DEC0000000E03FCC260220D426022038B5C368EB
:10DED00004460D465B6853F82120054BB2F920003B
:10DEE0001B68984729462046BDE8384007F049BBE3
:10DEF0006002002007F045BBC3682DE9F0475B686E
:10DF000004460D46002653F82170DFF8C8A02DED19
:10DF1000028BADF50A7D9FED2C8B0DF128083B6A35
:10DF2000B3422CD97B6A52464FF48071404653F875
:10DF300026900136334649F0A1FD4FF47F4309F1A5
:10DF400001022946069300232046CDE90233CDE99C
:10DF5000008306AB8DED088B01F0EEF828B305A920
:10DF600006A80BF04BF9059B9BB938B3204699F8EE
:10DF70000020294607F000FB06A8FEF745F82946D1
:10DF800020460DF50A7DBDEC028BBDE8F04707F099
:10DF9000F8BA0F4A4FF4807133464AA849F06EFD33
:10DFA0004AAA2946204607F0A7F906A8FEF72CF84A
:10DFB0000DF50A7DBDEC028BBDE8F08706A8FEF7E3
:10DFC00023F8ACE7AFF30080000000000000000081
:10DFD000570F0608240F0608044B10B5044640F8F6
:10DFE000083BFEF711F8204610BD00BFC40F06081D
:10DFF00010B50446FFF7F0FF1821204629F063F81A
:10E00000204610BD38B50D460446FDF7FDFF2B78C0
:10E0100023706B7863706A886280AB68A360EB687A
:10E02000E360D30741BFA26853680133536038BD32
:10E03000C36A0022F0B553F8216089B04FF47F43E2
:10E04000044601920D4604930023CDE90623364B86
:10E05000CDE90222009304AB01F0E4F8002855D08A
:10E06000002E38D1E36A53F825301BB129462046EB
:10E0700007F065F82D491820FCF7E0FF2C4B002233
:10E08000064603604FF47F43294683600023C0E9BE
:10E090000423E36A43F82500204600F0E9FC04A9C4
:10E0A00006F10800FFF7AEFF04AB01222946204627
:10E0B00007F0FCF94FF0FF33012229462046CDE955
:10E0C00000321A4607F0C0FC00BB1A4A2946204617
:10E0D00007F012F91AE09DF8102006F10807337ACC
:10E0E000934218D004A93846FFF78CFF04AB0122F5
:10E0F0002946204607F0DAF90021204606F0F1FF14
:10E100000028D7D02946204607F019F804A8FDF7C3
:10E110007BFF09B0F0BD084A394604A852F8233005
:10E1200098470028DED0E7E78C0F0608F43BDC7246
:10E13000C40F0608D408060848040020C3685B68BA
:10E1400053F821301B88B3F57A7F70B505469CB033
:10E150000C460AD96FF47A729E18124A52F8262099
:10E1600092B11CB0BDE8704010470DD00F2B04D108
:10E170001CB0BDE87040FEF78FBD192B10D11CB04C
:10E18000BDE87040FEF7F6BF074A6421009303A87C
:10E19000234649F073FC03AA2146284607F0ACF851
:10E1A0001CB070BDE0010020CC0F060810B50F4C6C
:10E1B000C2B02378834217D00D4B20701B789BB1DF
:10E1C0000C4B1B68984723784FF480710A4A0093E0
:10E1D00002A8002349F052FC02A8F2F773F8074B9B
:10E1E000014602A81B68984742B010BD2D3302209B
:10E1F0002C330220740200200D100608700200204B
:10E20000FF22012180F82C20002281864FF0FF316F
:10E210000263C0F8D82082604262C0E90022C0E9EF
:10E220000311C0E90511C0E907127047044B012032
:10E23000044A187000231370034A1360FFF7B6BF37
:10E240002C3302202E330220303302200020024BD8
:10E250001870FFF7ABBF00BF2C33022038B5144B4A
:10E260001C7814B3134B1B78012B1CD0022B124BC0
:10E2700006D1002201201A70FFF798FF204638BD12
:10E280001D781DB100222C461A70F7E70268096854
:10E29000D268526852F821205288002AEED001201C
:10E2A0001870FFF783FF0024E8E70124E6E700BFCA
:10E2B0002C3302202D3302202E3302202DE9F0438F
:10E2C00089B00346124A202168466C4649F0D6FBC5
:10E2D0006846F1F7F7FF002506460E4FDFF8388055
:10E2E000DFF83890B54210D03B6814F8012B591C68
:10E2F00008F803204029396005D1D9F8003040469C
:10E30000984700233B600135ECE709B0BDE8F08396
:10E310008E56070828330220E432022070020020C3
:10E320002DE9F8433F4C22223F4D07462368591CF4
:10E33000EA544029216005D13C4B28461B68984788
:10E3400000232360013FDFF8E480374E236817F88D
:10E35000019F591C2160B9F1000F40D0B9F1220F83
:10E3600017D15C224029EA5405D1D8F80030304654
:10E3700098470023236023682222591C21604029EA
:10E38000EA54E3D1D8F800303046984700232360A0
:10E39000DCE7B9F1090F0ED15C224029EA5405D11E
:10E3A000D8F8003030469847002323602368742251
:10E3B000591C2160E3E7B9F10A0F0ED15C22402914
:10E3C000EA5405D1D8F8003030469847002323603E
:10E3D00023686E22591C2160D1E73A78CFE72222C8
:10E3E0004029EA5405D1114B0F481B689847C4F8DF
:10E3F000009023680A22591CEA544029216005D163
:10E400000A4B09481B6898470023236021680029AC
:10E4100005DD064B04481B68984700232360BDE8D0
:10E42000F88300BF28330220E4320220700200206B
:10E430002DE9F04389B00346124A202168466C4614
:10E4400049F01CFB6846F1F73DFF002506460E4FDC
:10E45000DFF83880DFF83890B54210D03B6814F808
:10E46000012B591C08F803204029396005D1D9F83F
:10E4700000304046984700233B600135ECE709B087
:10E48000BDE8F083F80F060828330220E4320220AA
:10E49000700200202DE9F0414823054616460C463F
:10E4A00005F8013B01EB02082F46444507F102073E
:10E4B0000ED020780009FDF7F0FC07F8020C14F8E4
:10E4C000010B00F00F00FDF7E8FC07F8010CECE78A
:10E4D000002305F81630BDE8F0810000F0B51F46B6
:10E4E000154BCBB004461B780D4616460BB3134BA9
:10E4F0001B68984709A908A8FCF732FE104B4FF497
:10E500008071104A1B680AA80693089B0593509BCC
:10E51000CDE903732368CDE901560093012349F047
:10E52000ADFA0AA8F1F7CEFE074B01460AA81B6810
:10E5300098474BB0F0BD00BF2C330220740200207E
:10E5400094260220FB0F0608700200200C4B1B785B
:10E5500000B5C1B08BB10B4B1B68984702234FF439
:10E560008071094A684649F089FA6846F1F7AAFEBF
:10E57000064B014668461B68984741B05DF804FBAE
:10E580002C330220740200201010060870020020B4
:10E590000E4B1B7810B50446C2B0ABB10C4B1B68D8
:10E5A000984706230B4A4FF4807102A8009449F063
:10E5B00065FA02A8F1F786FE074B014602A81B6820
:10E5C0009847204600F084F842B010BD2C3302205A
:10E5D0007402002058100608700200202DE9F84F40
:10E5E000384C7B22384E05462368591CF25440298A
:10E5F000216005D1354B30461B68984700232360C6
:10E600002846FFF75BFE23682C22591CF254402950
:10E61000216005D12D4B2C481B68984700232360AF
:10E6200005F108074FF00009DFF8A0A0B846DFF8B1
:10E6300098B06868FFF7FCFE20682B68411C4B45CA
:10E64000216012D94FF02C034029335405D1DAF858
:10E6500000305846984700232360404609F10109DD
:10E6600008F11008FFF72AFEE6E77D23402933541E
:10E6700005D1164B14481B68984700232360236874
:10E680000A22591CF2544029216005D10F4B0E4833
:10E690001B689847002323602168002905DD0B4B88
:10E6A00009481B6898470023236000242B68A34275
:10E6B00005D9384601341037FFF76AFFF6E7BDE8A1
:10E6C000F88F00BF28330220E432022070020020BD
:10E6D00000B5037893B0132B7AD8DFE803F00A1F54
:10E6E00021283033373A3D404A57505C635C636AB7
:10E6F0006E71394A3F2102A8FDF7D4FA374A40210A
:10E7000002A8FDF7E9FA02A8F1F7DCFD344B014657
:10E7100002A81B68984713B05DF804FB314AE9E78B
:10E720008168314A314B002908BF1A46E2E790F967
:10E7300008302F4A3F2102A849F0A0F9DEE7037A0A
:10E740002C4AF7E7B0F908302B4AF3E703892B4A44
:10E75000F0E783682A4AEDE783682A4AEAE7D0E9C6
:10E760000223CDE90023284A3F2102A849F086F977
:10E77000C4E7D0E90223CDE90023244AF4E70822C4
:10E7800081180DEB0200FFF785FEB7E700F10801E5
:10E79000042202A8F7E709F07DFE13B05DF804EB50
:10E7A000FFF7BEBD09F0BCF913B05DF804EBFFF74D
:10E7B00015BF8368164ADB68BCE78368154AB9E76A
:10E7C000212308228DF8083081180DF10900DAE7BD
:10E7D00000238DF8083091E719100608281E060856
:10E7E0007002002024100608141006085A060608B5
:10E7F0002A1006082F1006083410060838100608DC
:10E800003C1006083C08060840100608451006089B
:10E810004A1006084E100608164B1B782DE9F041E9
:10E820000446C2B013B3144BDFF854801B689847FA
:10E83000124FE66B00243369A34217D9736942462D
:10E840004FF4807102A853F824500323CDE900450A
:10E8500049F014F902A8F1F735FD3B68014602A81A
:10E86000984728460134FFF733FFE4E742B0BDE89C
:10E87000F08100BF2C3302207402002070020020BF
:10E8800055100608394B1B782DE9F0430446ADF5C9
:10E89000057D002B66D0364B1B689847E3692268DC
:10E8A000218A002B3AD01B68606A0025314FDFF8BF
:10E8B000CC90CDE90230CDE9002107232E4A4FF458
:10E8C000807104A849F0DAF804A8F1F7FBFC3B6872
:10E8D000014604A89847D4F80C80D8F80820D8F846
:10E8E0001030AA421DD92B44A66A4A464FF48071C3
:10E8F00006EB0316236844A800930423CDE90156D0
:10E9000049F0BCF844A8F1F7DDFC3B68014644A897
:10E91000984730460135FFF7DBFEDEE74FF0FF3367
:10E92000C2E70025DFF85490D8F81030AB4219D96F
:10E93000A66A4A4623684FF4807106EB051644A880
:10E9400000930523CDE9015649F098F844A8F1F762
:10E95000B9FC3B68014644A8984730460135FFF7AB
:10E96000B7FEE1E70DF5057DBDE8F0832C3302200D
:10E9700074020020700200200410060852100608DD
:10E980000D4B1B7810B50446C2B09BB10B4B1B68F6
:10E99000984723684FF48071094A009302A809231D
:10E9A00049F06CF802A8F1F78DFC064B014602A86D
:10E9B0001B68984742B010BD2C330220740200201F
:10E9C0000D10060870020020104B1B7810B504468D
:10E9D000C4B0C3B10E4B1B689847606BF1F7DEFD06
:10E9E00023680C4A00930823CDE902014FF480719B
:10E9F00004A849F043F804A8F1F764FC064B01466B
:10EA000004A81B68984744B010BD00BF2C330220F7
:10EA1000740200205F10060870020020104B1B7863
:10EA200070B50546C2B00E461446BBB10D4B1B680F
:10EA300098472B680C4A4FF48071009302A80A2370
:10EA4000019649F01BF802A8F1F73CFC074B014680
:10EA500002A81B6898472046FFF762FC42B070BDD1
:10EA60002C330220740200206C1006087002002073
:10EA7000124B1B7830B50446C5B00D46DBB1104BC8
:10EA80001B689847E36A4FF480710E4A53F82530AB
:10EA900004A8003B18BF0123CDE90153236800936C
:10EAA0000D2348F0EBFF04A8F1F70CFC064B0146E0
:10EAB00004A81B68984745B030BD00BF2C33022026
:10EAC000740200200710060870020020104B1B780B
:10EAD00030B50446C5B00D46BBB10E4B1B68984718
:10EAE000236B4FF480710C4A5B5D04A8CDE90153A0
:10EAF000236800930E2348F0C1FF04A8F1F7E2FB5E
:10EB0000064B014604A81B68984745B030BD00BFBE
:10EB10002C33022074020020071006087002002027
:10EB2000F8B5461E2A4C2B4D236816F8017F591C58
:10EB3000002F39D0092F17D15C2240292160EA54D7
:10EB400005D1254B28461B6898470023236023687E
:10EB50007422591CEA544029216005D11E4B2846D5
:10EB60001B6898470023236023683278591C0A2ABF
:10EB7000216017D15C224029EA5405D1164B284662
:10EB80001B6898470023236023686E22591C21606C
:10EB90004029EA54C8D1104B28461B6898470023E7
:10EBA0002360C1E73278F3E70A2240292160EA5462
:10EBB00004D1094B07481B68984727602168002942
:10EBC00005DD054B03481B68984700232360F8BD0B
:10EBD00028330220E432022070020020114B1B78FF
:10EBE00070B50546C4B00E461446CBB10E4B1B683B
:10EBF00098472B680D4A4FF480710193042304A8B1
:10EC0000029600930B2348F039FF04A8F1F75AFB52
:10EC1000074B014604A81B6898472046FFF780FF72
:10EC200044B070BD2C330220740200206910060825
:10EC30007002002070B5C2B004460D4600F032FDEF
:10EC400000283DD1AC423BD0661E47F6FE439E42B3
:10EC500038D8284B02A81C68FFF7D2FA02AA31B2B2
:10EC6000204600F025FD10B1012106F0CDFB6C1E01
:10EC700047F6FE439C4231D81E4B02A81E68FFF7A0
:10EC8000BFFA02AA21B2304600F012FD10B10021F5
:10EC900006F0BAFB184B1B7893B1184B1B689847CA
:10ECA0000C234FF48071164A02A8009548F0E6FE46
:10ECB00002A8F1F707FB134B014602A81B6898470F
:10ECC00042B070BD002CD2DA0F4BE44302A81E689C
:10ECD000FFF796FA02AA21B23046C2E7002DD9DA30
:10ECE000094B02A81C68FFF78BFAE94302AA2046E9
:10ECF00009B2C9E7A86302202C3302207402002065
:10ED00000D10060870020020AC6302200000000015
:10ED10002DE9F84F524B1A6802F1010ABAF1010FBE
:10ED2000C3F800A04BD14F4B002200244E4D9B4610
:10ED30001A80A3F800220FF21819D9E90089504669
:10ED40000AF1010AF1F718FC42464B4606460F4607
:10ED5000F1F7A6FD0BF1020B41EC100BFDF768F982
:10ED60003DA3D3E9002351EC100BF1F76FFC2246D1
:10ED70002B46F1F7B5FAF1F741FF2246ABF8000058
:10ED80002B4630463946F1F7A9FA42464B46F1F791
:10ED900087FD41EC100BFDF74BF92FA3D3E90023BE
:10EDA00051EC100BF1F752FC22462B46F1F798FA82
:10EDB000F1F724FFBAF5807FABF80002BFD12B4AF0
:10EDC000136803F1010ABAF1010FC2F800A03AD1A9
:10EDD000274B00224FF00008DFF88C9003F580618C
:10EDE00003F1040B1A600A6019A7D7E900675046BF
:10EDF0000AF1010AF1F7B0FB32463B4604460D46E4
:10EE0000F1F74EFD41EC100BFDF712F951EC100B30
:10EE1000F1F714FF42464BF8040B4B4620462946B7
:10EE2000F1F75CFA32463B46F1F73AFD41EC100B44
:10EE3000FDF7FEF851EC100BF1F700FFBAF5807FFB
:10EE4000CBF8FC03D3D1BDE8F88F00BFAFF300804F
:10EE50000000000000E06F4000000000E0FFEF4015
:10EE6000D0260220D42E02200000E03FCC26022033
:10EE7000D426022038B50D460446FDF7C5F82B7898
:10EE800023706B7863706A886280AB68A360EB68FC
:10EE9000E360D30741BFA26853680133536038BDB4
:10EEA00038B50A780446152A03D18968FEF776FB3F
:10EEB00006E0182A06D1B1F90820094909F068F8D6
:10EEC000204638BD162AF1D18D6805F1080008F0FA
:10EED0002EFEA96900EB011120460831E6E700BFCC
:10EEE000586F022008B5D0F85031132B06D9084AC4
:10EEF000D0E9000106F000FA002008BD0133C0F897
:10EF0000503100EB0310FFF7B5FF0120F5E700BF1C
:10EF1000761006081FB5D0F85031132B12D80133E4
:10EF20004FF6157202916946C0F8503100EB03109C
:10EF30000092FFF79FFF6846FDF766F8012005B0D5
:10EF40005DF804FB0020FAE72DE9F04F054695B087
:10EF5000894690461F460026714CD0E902AB09F164
:10EF600001039A5D19F8063003EB0223C3F30C0189
:10EF700013F460430CD1DAF80C3053F8211020461A
:10EF8000FFF7B0FF002835D1002015B0BDE8F08FA5
:10EF9000B3F5005F03D1AB6A03EB0111EFE7B3F503
:10EFA000804F09D1DBF810301944AB6A03EB011133
:10EFB0002046FFF7AFFFE5E7B3F5C04F1CD1DAF805
:10EFC00010308B4204D9DAF8143053F82110EFE7EF
:10EFD000C3F101034FF618720B441092129310A95B
:10EFE0002046FFF77FFF019010A8FDF70DF8019B69
:10EFF000002BC9D00236B2E7B3F5004F05D14FF66A
:10F000001773ADF848101093E9E7B3F5204F75D1A9
:10F01000D4F8501110A84B1E04EB0111C4F8503164
:10F02000FEF7BCFA10A904A8FFF73AFF10A8FCF7F6
:10F03000EBFFD4F8501110A84B1E04EB0111C4F8DB
:10F040005031FEF7ABFA10A908A8FFF729FF10A866
:10F05000FCF7DAFF9DF82030012B15D84FF47F43E1
:10F0600010A92046109300231293FFF73BFF019055
:10F0700010A8FCF7C9FF019B83B108A8FCF7C4FFE7
:10F0800004A8FCF7C1FFB5E70E2B0ED0102B0CD057
:10F09000244B3A466168284606F0F6FB08A8FCF7C0
:10F0A000B3FF04A8FCF7B0FF6EE708A808F03FFD27
:10F0B00003A9019004A809F0DFF80399019B09B1A5
:10F0C000194BE6E7002802DB1B68834201DC174B83
:10F0D000DFE708A901900CA8FEF760FA144B019A2B
:10F0E0000CA910A808F068FD10A92046FFF7FAFE49
:10F0F000019010A8FCF788FF0CA8BAE7B3F5404FC1
:10F1000005D10C4B204653F8213098473AE7B8F127
:10F11000000F01D1012038E70236C8F80060F9E796
:10F120003833022090100608A6100608D6100608EC
:10F130002F0E2E1380020020F0B589B01E4C1E4603
:10F140000D46109B00271146A360C4F85071DDE9FD
:10F150000E32C4E90005FFF7F7FE0546D8B1D4F832
:10F160005031012B17D104F110016846C4F85071D9
:10F17000FEF714FA694604A8FFF792FE04A9304688
:10F18000FFF778FE04A8FCF73FFF6846FCF73CFF5A
:10F19000284609B0F0BD4FF47F43002204A9304651
:10F1A000049300230025CDE90623FFF763FE04A89E
:10F1B000FCF72AFFECE700BF38330220F0B585B03A
:10F1C000174C1F460D460C9B00261146A360C4F841
:10F1D0005061DDE90A32C4E90005FFF7B5FE0546D6
:10F1E000B0B1D4F85031012B18D104F110016846A8
:10F1F000C4F85061FEF7D2F99DF80030153B032B9F
:10F2000009D838466946FFF735FE6846FCF7FCFE2C
:10F21000284605B0F0BD6846FCF7F6FE3546F7E730
:10F22000383302202DE9F0470C1EC2B00546DDF848
:10F2300030819DF83491DDE94AAE03DBC7683E6852
:10F24000A64212DC2B8A4FF48071174A02A8009361
:10F25000234648F013FC284602AB5246214606F0EE
:10F2600013FB002042B0BDE8F0877F68002A57F802
:10F27000247002DBFE6896420ADC2B8A4FF4807110
:10F2800002A8CDE900431346084A48F0F7FBE2E73D
:10F290003C69CDE94C89CDE94AAE54F8222042B010
:10F2A000BDE8F047FFF748BFF91006082811060827
:10F2B0002DE9F0430C1EC5B00546DDF83881DDE9C7
:10F2C0004C9E03DBC7683E68A64212DC2B8A4FF4D3
:10F2D0008071194A04A80093234648F0CFFB2846C2
:10F2E00004AB4A46214606F0CFFA002045B0BDE8FF
:10F2F000F0837F68002A57F82470D7F80CC001DB30
:10F3000062450CDB2B8A4FF4807104A8CDF800C055
:10F31000CDE901431346094A48F0B0FBDFE73C69F9
:10F32000CDF83091CDE94DE854F8222045B0BDE844
:10F33000F043FFF743BF00BFF91006086C11060841
:10F340007FB5066A1EB90024204604B070BD8368EC
:10F35000F168B3F90230CA69DB4352F82320002A6E
:10F36000F1D0B2F900305D1CEDD0B2F90220541C8E
:10F37000E9D049680024144D103051F82310096970
:10F3800051F822102246A8603046C5F85041C5E920
:10F3900000632346FFF7D8FD0028D4D0D5F85031BC
:10F3A000012BD0D105F110016846C5F85041FEF798
:10F3B000F5F89DF800306846182B08BFBDF90840E5
:10F3C000FCF722FEC0E700BF383302200000000037
:10F3D0005B4900202DE9F84F14230C46FF25002639
:10F3E00000270A46013B087401F110015574508250
:10F3F000C2E90667F5D1534AC4F85031116801F1EA
:10F40000010ABAF1010FC2F800A04AD14E4A002405
:10F410004E4D93461380A2F800320FF21419D9E929
:10F42000008950460AF1010AF1F7A6F842464B4618
:10F4300006460F46F1F734FA0BF1020B41EC100BC4
:10F44000FCF7F6FD3CA3D3E9002351EC100BF1F7D8
:10F45000FDF822462B46F0F743FFF1F7CFFB22469B
:10F46000ABF800002B4630463946F0F737FF4246EE
:10F470004B46F1F715FA41EC100BFCF7D9FD2EA322
:10F48000D3E9002351EC100BF1F7E0F822462B46AC
:10F49000F0F726FFF1F7B2FBBAF5807FABF8000278
:10F4A000BFD12B4A136803F1010ABAF1010FC2F868
:10F4B00000A03AD1274B00224FF00008DFF88C90D3
:10F4C00003F5806103F1040B1A600A6018A7D7E9FD
:10F4D000006750460AF1010AF1F73EF832463B4612
:10F4E00004460D46F1F7DCF941EC100BFCF7A0FDEA
:10F4F00051EC100BF1F7A2FB42464BF8040B4B46C4
:10F5000020462946F0F7EAFE32463B46F1F7C8F9B5
:10F5100041EC100BFCF78CFD51EC100BF1F78EFB5E
:10F52000BAF5807FCBF8FC03D3D1BDE8F88F00BFDC
:10F530000000000000E06F4000000000E0FFEF402E
:10F5400038330220D0260220D42E02200000E03FD3
:10F55000CC260220D426022038B51424034D05EB16
:10F560000410FCF751FD013CF9D138BD38330220BD
:10F5700038B50D460446FCF747FD2B7823706B78B1
:10F5800063706A886280AB68A360EB68E360D3074E
:10F5900041BFA26853680133536038BDC36B10B5D7
:10F5A0000446186858B10022054B1A7006F03EFA5E
:10F5B000044B1B6898472046FFF72EF9012010BD29
:10F5C000540200206C020020334B2DE9F04F1B68E1
:10F5D00089B0984700285CD0FBF7D8FE2F4F06462D
:10F5E0004FF0000A4FF0000B0DF1070203A902A82B
:10F5F00006F068FA50B19DF807306BB106F082FA58
:10F60000DDE90201FEF79AFD3C7864B1244B1B68EA
:10F6100009B0BDE8F04F184703A902A8FEF71EFE87
:10F620000028EBD1F2E7029B4FF47F49039ADB6895
:10F630005B6853F82280D8F804300298A3421BD9A3
:10F64000D8F80830C26833F814305269D25CD20757
:10F6500010D5856A04A9CDF8109005EB031528464E
:10F66000CDE906ABFFF784FF04A8FCF7CDFC2846E4
:10F67000FEF78EFF0134DEE7012105F032FD10B107
:10F68000029805F071FDFBF781FE831B042BABD9BB
:10F69000BCE709B0BDE8F08F6802002054020020EA
:10F6A00078020020014B1878704700BF54020020F8
:10F6B000C36B70B505460C461646F3B1144B1B6878
:10F6C0009847D0B1B36853B11A880F2A07D1306A6E
:10F6D00098B12246198CBDE87040FDF7D3BAEB68AB
:10F6E00053F824309B8C5B0707D40A4B1B683BB153
:10F6F0001A8AA24202D05B6CF9E70023184670BD5B
:10F70000214628461A46BDE8704006F0B6B800BF4C
:10F710006802002094340220008A7047564B2DE97D
:10F72000F0431B688DB006460C469146984700286A
:10F7300000F09E80E44361D4376AFB68B3F920206F
:10F7400094425BDA5B6A53F82450B5F90030013318
:10F7500054D0B5F90230013350D0B36806F110042B
:10F760001B881C2B53D11722444B0321684608F0F9
:10F77000E1F9029833694FF6077808A910300A9327
:10F780001026CDF82080FFF7F3FE08A8FCF73CFC1C
:10F790003B4B1A22042104A808F0CCF9069808A9CA
:10F7A00054F8043B304410360A93CDF82080FFF71C
:10F7B000DFFE08A8FCF728FC502EEFD1029804A920
:10F7C0002030FFF7D5FE0298D9F8003008A9303074
:10F7D000CDF820800A93FFF7CBFE08A8FCF714FCB5
:10F7E0006B46B5F90220B5F90010384605F05EFE0B
:10F7F00004A8FCF709FC6846FCF706FCFFF7E4FEEA
:10F80000FFF7E2FE0DB0BDE8F043FFF7DDBE1422C6
:10F810001C4B0221684608F08DF9029833694FF6B7
:10F82000077808A910300A931026CDF82080FFF73A
:10F830009FFE08A8FCF7E8FB114B1A22042104A83C
:10F8400008F078F9069808A954F8043B30441036BB
:10F850000A93CDF82080FFF78BFE08A8FCF7D4FBB5
:10F86000502EEFD1029804A92030FFF781FEB7E7B0
:10F870000DB0BDE8F08300BF680200200BB3E35376
:10F88000F88EF6B1BB4059282DE9F0411D46814B59
:10F8900080460E461B6814462DED028B8CB09847AF
:10F8A000002853D07FEA080000F1EB80236ADB6870
:10F8B000B3F91820824240F3E480DA695B6852F8B9
:10F8C0002020B2F9002053F82270C6B92B462246F8
:10F8D000314680B205F0A8FC3B88182B36D1A368CE
:10F8E000B3F90230434531D12A46214608A814F025
:10F8F0007BFC284608A9FFF73BFE08A824E0162E4B
:10F900002ED14FF47F430022314680B2049300236E
:10F91000CDE9062304AB224605F086FC9DF81030A5
:10F920000E2B01D0102B16D104A808F000F94FF6C9
:10F9300007720368089208A928460A93FFF718FE81
:10F9400008A8FCF761FB04A8FCF75EFB0CB0BDEC5B
:10F95000028BBDE8F0814FF6077308930023EAE7B6
:10F96000402E0BD126F0EAFF0028EFD003685B6E33
:10F9700098474FF607730A900893BAE7042E07D109
:10F980003B88182BE2D1214608A814F0EFFAB0E723
:10F99000052E07D13B88182BD8D1214608A814F092
:10F9A0003FFBA6E7072E07D13B88182BCED1214677
:10F9B00008A814F08FFB9CE70A2E08D13B88182B6F
:10F9C000C4D1204614F0E0FBFBF714FDD1E7252E4F
:10F9D000BCD13B8886B2182B49D1A768BB8B9B074B
:10F9E00003D52B78073B012B05D82A462146304604
:10F9F00005F03CFE30E0214604A814F06BFB00212A
:10FA000004A808F0BBFB002128468DED030A08F08E
:10FA1000B5FB20468DED020A14F0B6FBDDED030ABE
:10FA20009DED020A0190FCF719FAB0EE408A0198A8
:10FA3000FBF7E8FC4FF60B7308AA2146C8EE007AE4
:10FA400030460893CDED0A7A05F010FE08A8FCF7C1
:10FA5000DBFA04A8FCF7D8FA0022B7F90610204612
:10FA60000CB0BDEC028BBDE8F041FFF757BE2A4653
:10FA7000214630460CB0BDEC028BBDE8F04105F0EC
:10FA8000F5BD4FF47F43002208930023CDE90A23FC
:10FA90002FE700BF680200202DE9F84F524B1A688B
:10FAA00002F1010ABAF1010FC3F800A04BD14F4B8C
:10FAB000002200244E4D9B461A80A3F800220FF22C
:10FAC0001819D9E9008950460AF1010AF0F754FDE6
:10FAD00042464B4606460F46F0F7E2FE0BF1020B9C
:10FAE00041EC100BFCF7A4FA3DA3D3E9002351EC41
:10FAF000100BF0F7ABFD22462B46F0F7F1FBF1F7C8
:10FB00007DF82246ABF800002B4630463946F0F728
:10FB1000E5FB42464B46F0F7C3FE41EC100BFCF709
:10FB200087FA2FA3D3E9002351EC100BF0F78EFDD9
:10FB300022462B46F0F7D4FBF1F760F8BAF5807F48
:10FB4000ABF80002BFD12B4A136803F1010ABAF1E6
:10FB5000010FC2F800A03AD1274B00224FF0000855
:10FB6000DFF88C9003F5806103F1040B1A600A60E2
:10FB700019A7D7E9006750460AF1010AF0F7ECFC33
:10FB800032463B4604460D46F0F78AFE41EC100B28
:10FB9000FCF74EFA51EC100BF1F750F842464BF8D7
:10FBA000040B4B4620462946F0F798FB32463B466D
:10FBB000F0F776FE41EC100BFCF73AFA51EC100B23
:10FBC000F1F73CF8BAF5807FCBF8FC03D3D1BDE860
:10FBD000F88F00BFAFF300800000000000E06F402E
:10FBE00000000000E0FFEF40D0260220D42E0220CB
:10FBF0000000E03FCC260220D426022001207047DE
:10FC0000704770477047704707B50190002026F095
:10FC100043FD0022019903B05DF804EB06F01BBA26
:10FC200008B5034A2A21034B034845F0C3FF00BF30
:10FC3000BD1106085A060608DA1106087047704713
:10FC400070470000000000002DE9F84F524B1A6881
:10FC500002F1010ABAF1010FC3F800A04BD14F4BDA
:10FC6000002200244E4D9B461A80A3F800220FF27A
:10FC70001819D9E9008950460AF1010AF0F77CFC0D
:10FC800042464B4606460F46F0F70AFE0BF1020BC2
:10FC900041EC100BFCF7CCF93DA3D3E9002351EC68
:10FCA000100BF0F7D3FC22462B46F0F719FBF0F7C8
:10FCB000A5FF2246ABF800002B4630463946F0F748
:10FCC0000DFB42464B46F0F7EBFD41EC100BFCF709
:10FCD000AFF92FA3D3E9002351EC100BF0F7B6FCDA
:10FCE00022462B46F0F7FCFAF0F788FFBAF5807F42
:10FCF000ABF80002BFD12B4A136803F1010ABAF135
:10FD0000010FC2F800A03AD1274B00224FF00008A3
:10FD1000DFF88C9003F5806103F1040B1A600A6030
:10FD200019A7D7E9006750460AF1010AF0F714FC59
:10FD300032463B4604460D46F0F7B2FD41EC100B4F
:10FD4000FCF776F951EC100BF0F778FF42464BF8D0
:10FD5000040B4B4620462946F0F7C0FA32463B4694
:10FD6000F0F79EFD41EC100BFCF762F951EC100B23
:10FD7000F0F764FFBAF5807FCBF8FC03D3D1BDE880
:10FD8000F88F00BFAFF300800000000000E06F407C
:10FD900000000000E0FFEF40D0260220D42E022019
:10FDA0000000E03FCC260220D4260220002070472D
:10FDB000F8B50B460C460546006853F8081B626808
:10FDC00099420CD10AB139F063FE636800212A68B8
:10FDD0006B60D1540023226863601370F8BD05F195
:10FDE0000807B842C5E9001208BF0020A26818BF82
:10FDF000AE68AA6010B12060A660EBE72360E9E777
:10FE000073B5044616460D4619B912B10D4832F0C5
:10FE100001FF731B0F2B019307D9002201A9204674
:10FE200039F0E6FD019B2060A36032462946206838
:10FE300039F076FE019B226800216360D15402B044
:10FE400070BD00BFFC11060800F0FD00A0F10D031D
:10FE500058425841704782B0ADF8000000208DF83C
:10FE600003208DF80210009B9AB21B0C62F30F0066
:10FE700063F31F4002B07047401A4FF007034ABFB8
:10FE8000821F90FBF3F392FBF3F3A3EBC30318443D
:10FE900070470B681A1D4FF00702A8BF0433B3FB6D
:10FEA000F2F2C2EBC2029B1ADBB203707047000091
:10FEB0001FB5164A044601AB1068516803C3906829
:10FEC000A2781860022A1AD1B4F9003099070ED12D
:10FED000642093FBF0F100FB113109B291B94FF4AA
:10FEE000C87193FBF1F001FB10331BB253B102F167
:10FEF00010030DEB030212F80D0C04B010BD531EDD
:10FF00000B2BF4D94FF01D00F7E700BF90EA05086E
:10FF100030B5B0F900208578C3784FF4C870022D51
:10FF200098BF013A1849002ABBBF6FF4C77C02EBA7
:10FF30000C0492FBF0F494FBF0F4022D01FB04217D
:10FF400005EBC5024FF0050088BF6FF4E47502EBC6
:10FF500002128CBF521902F26352B2FBF0F2581E29
:10FF600040F26D1303FB0100642300EB9100B1FB31
:10FF7000F3F1401A054B104403FB0400A0F52F20B9
:10FF8000A0F66C2030BD00BF70FEFFFFB13A02004A
:10FF900008B5FFF7BDFF08BD13B5B0F90010044662
:10FFA00011F5004F14D08278531E0B2B10D8C07857
:10FFB00060B101A8ADF804108DF80620FFF778FFB6
:10FFC000C3B2E078834234BF0020012002B010BDEC
:10FFD0000020FBE700F52F2303F66C23002BB8BFAE
:10FFE00000F50B2273B5B8BF02F6BC72264927484C
:10FFF00040F2B45640F26D15B4BF92FBF1F193FBA1
:020000040801F1
:10000000F1F148F6AC6200FB0130B0FBF2F2B0FB5C
:10001000F6F30244D21A1E4BB0FBF3F3D21A4FF49C
:10002000C873B2FBF5F403FB014148F69463B2FBDD
:10003000F3F3B2FBF6F203449B1A992205FB143347
:10004000052503EB830401330234B4FBF2F0424391
:100050000232B2FBF5F29B1A40F2F95294428DF84B
:10006000073094BFC21CA0F109020020022A98BFE9
:1000700001318DF80620BDF8063089B261F30F001A
:1000800063F31F4002B070BDB13A02004FC5FDFFDF
:10009000B03A020037B583780446028801A88DF88B
:1000A00006300123ADF804208DF80730FFF770FF0C
:1000B000E5786946009001A805F00F05072D08BFF7
:1000C0000025FFF7E6FE9DF804102846FFF7D4FE52
:1000D000E37807221B0902FB0300009B0738184442
:1000E00003B030BD73B5B0F900600446857868464A
:1000F000ADF800608DF80250FFF7DAFE8DF80700CA
:1001000001A8ADF804608DF80650FFF741FF01A982
:1001100001906846FFF7BDFEE1789DF80000FFF70B
:10012000ABFE019B181A02B070BD38B50D460446EF
:10013000FBF76AFF2B7823706B7863706A886280A4
:10014000AB68A360EB68E360D30741BFA268536864
:100150000133536038BDD0F8501110B54B1E8CB030
:10016000044600EB0111C0F8503108A8FDF716FA5B
:1001700008A96846FEF794FE08A8FBF745FFD4F8E7
:10018000501108A84B1E04EB0111C4F85031FDF7C3
:1001900005FA08A904A8FEF783FE08A8FBF734FFB8
:1001A000002104A809F02AF818B10021684609F0D6
:1001B00025F84FF6027308A90A9020460893FEF727
:1001C00091FE044608A8FBF71FFF04A8FBF71CFFDD
:1001D0006846FBF719FF20460CB010BDD0F850114F
:1001E00010B54B1E8CB0044600EB0111C0F8503125
:1001F00008A8FDF7D3F908A96846FEF751FE08A83C
:10020000FBF702FFD4F8501108A84B1E04EB0111B4
:10021000C4F85031FDF7C2F908A904A8FEF740FE62
:1002200008A8FBF7F1FE002104A808F0E7FF18B9C1
:100230000146684608F0E2FF4FF6027308A90A90EB
:1002400020460893FEF74EFE044608A8FBF7DCFEA6
:1002500004A8FBF7D9FE6846FBF7D6FE20460CB093
:1002600010BDD0F8501110B54B1E88B000EB011135
:100270000446C0F8503104A8FDF790F904A9684677
:10028000FEF70EFE04A8FBF7BFFE9DF800300C2B16
:1002900014D14FF60C730493DDE90223CDE9062354
:1002A000204604A9FEF71EFE044604A8FBF7ACFE98
:1002B0006846FBF7A9FE204608B010BD0B2B09D1FC
:1002C0000021684607F05AFF4FF60B738DED060AC2
:1002D0000493E5E7A3F10902012A07D84FF6097351
:1002E0000493DDE90223CDE90623D9E7DA1F012AC9
:1002F00005D84FF607730493029B0693D0E75A1F65
:10030000012A07D8BDF908304FF60572ADF818304C
:100310000492C5E7033B012B07D89DF908304FF63F
:1003200003728DF818300492BAE70024C0E7D0F8C1
:10033000501110B54B1E88B000EB01110446C0F8F7
:10034000503104A8FDF72AF904A96846FEF7A8FD74
:1003500004A8FBF759FE9DF800300C2B16D1DDE9FF
:10036000022101F100434FF60C71CDE906230491FF
:10037000204604A9FEF7B6FD044604A8FBF744FE98
:100380006846FBF741FE204608B010BD0B2B0BD191
:100390000021684607F0F2FEB1EE400A4FF60B73FB
:1003A0008DED060A0493E3E7A3F10902012A0AD8B6
:1003B000029B4FF60971039A5B42049162EB420281
:1003C000CDE90632D4E7DA1F012A06D8029B4FF6A0
:1003D00007725B4204920693CAE75A1F012A08D8A3
:1003E000BDF808304FF605725B420492ADF8183044
:1003F000BEE7033B012B08D89DF808304FF6037287
:100400005B4204928DF81830B2E70024B8E7D0F8C8
:10041000501110B54B1E88B000EB01110446C0F816
:10042000503104A8FDF7BAF804A96846FEF738FD74
:1004300004A8FBF7E9FD9DF80030A3F10902012AA9
:1004400016D8029B4FF60A71DA43039B0491DB43F3
:10045000CDE90623204604A9FEF744FD044604A87E
:10046000FBF7D2FD6846FBF7CFFD204608B010BD74
:10047000DA1F012A06D8029B4FF60872DB4304926A
:100480000693E7E75A1F012A05D8BDF808304FF652
:100490000672DB43F3E7033B012B05D89DF80830D8
:1004A0004FF60472DB43EAE70024DBE7D0F8501193
:1004B00010B54B1E8AB000EB01110446C0F8503154
:1004C00002A8FDF76BF801A902A808F097FE019AAF
:1004D000A2B980F001034FF60272204606A9DBB2F2
:1004E00006920893FEF7FEFC044606A8FBF78CFD77
:1004F00002A8FBF789FD20460AB010BD0024F7E7EB
:1005000070B5D0F850118EB004464B1E02AD00EB12
:10051000011106AEC0F850312846FDF73FF8D4F877
:10052000501130464B1E04EB0111C4F85031FDF759
:1005300035F8D4F850110AA84B1E04EB0111C4F889
:100540005031FDF72BF801A90AA808F057FE019BCE
:100550009BB9002814BF314629462046FEF7C2FC4D
:1005600004460AA8FBF750FD3046FBF74DFD284630
:10057000FBF74AFD20460EB070BD0024F1E71FB521
:100580000446FAF703FF4FF60873694602902046C7
:100590000093FEF7A7FC04466846FBF735FD2046AE
:1005A00004B010BD30B584688BB005461CB3D0F8DC
:1005B00050114B1E00EB0111C0F8503102A8FCF79E
:1005C000EDFF01A902A807F057FE019CB4B903286A
:1005D0000ED8AB684FF6077206A953F820302846AC
:1005E00006920893FEF77EFC044606A8FBF70CFD76
:1005F00002A8FBF709FD20460BB030BD0024F7E749
:100600007FB505460068FFF787F8011E24DB2B68DD
:1006100089B200265A68114B1B689A4214BF0131F7
:10062000C94389B20CB230B226F036F8A0B12146E7
:10063000013605F0DFFD0028F5D04FF6027369465C
:10064000029028460093FEF74DFC04466846FBF7EF
:10065000DBFC204604B070BD0020EEE7AC63022056
:100660001FB503684FF60B7269465B6B00920293ED
:10067000FEF738FC04466846FBF7C6FC204604B08B
:1006800010BD0000D0F85011F0B54B1E95B00446D7
:1006900000EB0111C0F850316846FCF77FFFD4F839
:1006A000501104A800264B1E04EB0111C4F8503170
:1006B000FCF774FF9DF8003008A81B2B9DF8103044
:1006C0000CBFBDF80820029A1B2B1D4B0CBFBDF8B8
:1006D0001870069F394607F02DFA08A807F027FA88
:1006E00000F10805BE421ADAD4F850110CA8013600
:1006F0004B1E04EB0111C4F85031FCF74FFF0CA95D
:1007000010A8FEF7CDFB10A928461035FFF70DFD08
:1007100010A8FBF779FC0CA8FBF776FCE2E708A928
:100720002046FEF7DFFB044608A8FBF76DFC04A893
:10073000FBF76AFC6846FBF767FC204615B0F0BD86
:10074000D4607283D0F8501110B54B1E8AB000EB04
:1007500001110446C0F8503102A8FCF71FFF01A99F
:1007600002A807F089FD019B8BB94FF6077308902B
:1007700006A920460693FEF7B5FB044606A8FBF73C
:1007800043FC02A8FBF740FC20460AB010BD002441
:10079000F7E7D0F8501110B54B1E8AB000EB0111ED
:1007A0000446C0F8503102A8FCF7F8FE01A902A8DF
:1007B00007F0E4FC019B93B94FF60B73204606A9A2
:1007C0008DED080A0693FEF78DFB044606A8FBF79D
:1007D0001BFC02A8FBF718FC20460AB010BD002441
:1007E000F7E7D0F8501110B54B1E8AB000EB01119D
:1007F0000446C0F8503102A8FCF7D0FE01A902A8B7
:1008000007F03AFC019B93B94FF60C73204606A9FA
:1008100006938DED080BFEF765FB044606A8FBF773
:10082000F3FB02A8FBF7F0FB20460AB010BD002442
:10083000F7E7D0F8501110B54B1E88B000EB01114E
:100840000446C0F8503104A8FCF7A8FE04A9684685
:10085000FEF726FB04A8FBF7D7FB9DF800300C2B16
:1008600016D1DDE9022121F000434FF60C71CDE9EC
:1008700006230491204604A9FEF734FB044604A88D
:10088000FBF7C2FB6846FBF7BFFB204608B010BD74
:100890000B2B0BD10021684607F070FCB0EEC00AAC
:1008A0004FF60B738DED060A0493E3E7A3F10902FB
:1008B000012A0CD8DDE90232002A02DA5B4262EB3F
:1008C00042024FF60971CDE906320491D2E7DA1FF0
:1008D000012A08D8029B4FF60772002BB8BF5B4273
:1008E00004920693C6E75A1F012A08D8BDF90830BA
:1008F0004FF60572002BB8BF5B429BB2F0E7033B9B
:10090000012B08D89DF908304FF60372002BB8BFB1
:100910005B42DBB2E4E70024B4E7D0F8501110B535
:100920004B1E88B000EB01110446C0F8503104A8FA
:10093000FCF734FE04A96846FEF7B2FA04A8FBF7F8
:1009400063FB9DF800300C2B16D19DED020B40F09F
:10095000B3FF4FF60C738DED060B0493204604A9EC
:10096000FEF7C0FA044604A8FBF74EFB6846FBF707
:100970004BFB204608B010BD0B2B0BD10021684665
:1009800007F0FCFB4FF60B73BBFE400A8DED060A29
:100990000493E3E70024E9E7D0F8501110B54B1EAB
:1009A00088B000EB01110446C0F8503104A8FCF7F0
:1009B000F5FD04A96846FEF773FA04A8FBF724FBCB
:1009C0009DF800300C2B16D19DED020B40F090FEEF
:1009D0004FF60C738DED060B0493204604A9FEF729
:1009E00081FA044604A8FBF70FFB6846FBF70CFBF3
:1009F000204608B010BD0B2B0BD10021684607F034
:100A0000BDFB4FF60B73BAFE400A8DED060A049348
:100A1000E3E70024E9E70000D0F850112DE9F047A2
:100A20004B1E88B000EB01110446C0F8503104A8F9
:100A3000FCF7B4FD9DF8103000254FF000081B2B8B
:100A4000DFF8809004A80CBFBDF818A0DDF818A04E
:100A5000FBF7DAFA554524DAD4F8501168464B1EF4
:100A600004EB0111C4F85031FCF798FD694604A865
:100A7000FEF716FA002104A807F0FEFA04A857ECC6
:100A8000106BFBF7C1FA6846FBF7BEFA32463B46ED
:100A900040464946F0F76AF808B1B046B946013514
:100AA000D8E74FF60C7304A920460493CDE90689D4
:100AB000FEF718FA044604A8FBF7A6FA204608B089
:100AC000BDE8F0870000F07FD0F850112DE9F04725
:100AD0004B1E88B000EB01110446C0F8503104A849
:100AE000FCF75CFD9DF8103000254FF000081B2B33
:100AF000DFF8809004A80CBFBDF818A0DDF818A09E
:100B0000FBF782FA554524DAD4F8501168464B1E9B
:100B100004EB0111C4F85031FCF740FD694604A80C
:100B2000FEF7BEF9002104A807F0A6FA04A857ECC6
:100B3000106BFBF769FA6846FBF766FA32463B46EC
:100B400040464946EFF7F4FF08B1B046B9460135D3
:100B5000D8E74FF60C7304A920460493CDE9068923
:100B6000FEF7C0F9044604A8FBF74EFA204608B089
:100B7000BDE8F0870000F0FFD0F8501130B54B1EF3
:100B800095B0044600EB0111C0F8503110A8FCF7F5
:100B900005FD10A96846FEF783F910A8FBF734FAA3
:100BA000D4F8501110A84B1E04EB0111C4F85031B9
:100BB000FCF7F4FC10A904A8FEF772F910A8FBF7E3
:100BC00023FA234A04A908A808F046FA0CA8214AE7
:100BD000694608F041FA08A807F05CFC30B94FF606
:100BE000077310934FF0FF33129318E00CA807F02F
:100BF00051FC0028F3D008A807F04CFC05460CA8CF
:100C000007F048FC014628464FF6077547F056FFA7
:100C1000E0B908A807F03EFC40421095129010A9D8
:100C20002046FEF75FF9044610A8FBF7EDF90CA883
:100C3000FBF7EAF908A8FBF7E7F904A8FBF7E4F9E2
:100C40006846FBF7E1F9204615B030BD1095C9E7BD
:100C50004DBF16F633912281D0F850112DE9F0479F
:100C60004B1E9AB0044600EB0111C0F8503116A893
:100C7000FCF794FC16A902A8FEF712F916A8FBF7D8
:100C8000C3F9D4F8501116A84B1E04EB0111C4F897
:100C90005031FCF783FC16A906A8FEF701F916A847
:100CA000FBF7B2F9D4F8501116A84B1E04EB011152
:100CB000C4F85031FCF772FC16A90AA8FEF7F0F848
:100CC00016A8FBF7A1F90EA8374A02A908F0C4F943
:100CD0000EA807F0DFFB80B900260EA8FBF794F9F9
:100CE0000AA8FBF791F906A8FBF78EF902A8FBF713
:100CF0008BF930461AB0BDE8F0870EA807F0CAFBA2
:100D0000EFF7E0FA01A9074606A807F0B5FA019E39
:100D10000546002EE0D112A8244A0AA908F09CF941
:100D200012A807F0B7FB00283BD0BD4212A8B8BFFD
:100D30003D4607F0AFFBEFF7C5FA1D4B81462A464B
:100D40001C4916A808F042F99DF85830012B21D013
:100D5000ED1B16A807F09EFB804600EB050A0EA8C7
:100D600007F098FB791C02465046FAF79BFFAE420B
:100D70000BDA12A807F08EFBB6FBF9F309FB13633D
:100D8000C35C08F806300136F1E716A92046FEF7E5
:100D9000A9F8064616A8FBF737F912A8FBF734F9AD
:100DA0009BE70646F9E700BFE6AB6ACFD73B358144
:100DB000DD143BF475100608D0F850112DE9F0430E
:100DC0004B1E91B0044600EB0111C0F850310CA845
:100DD000FCF7E4FB0CA96846FEF762F80CA8FBF7E9
:100DE00013F9D4F850110CA84B1E04EB0111C4F8F0
:100DF0005031FCF7D3FB0CA904A8FEF751F80CA85E
:100E0000FBF702F9684607F045FB804650B900241D
:100E100004A8FBF7F9F86846FBF7F6F8204611B08E
:100E2000BDE8F08304A807F035FB06460028EED0A5
:100E300040464FF00009EFF745FA451C294928467E
:100E4000FAF7FCF8074642462946FAF72BFF3146E7
:100E5000384648F0D3FC30B13146002009F1010991
:100E600048F0CCFCF7E73846FAF722F91E49284645
:100E7000FAF7E4F8424629460746FAF713FF1B4BF8
:100E80000D22494608A8DFF8688006F053FE08A83E
:100E900006F04DFE05463146384648F0AFFC0835B1
:100EA000014699B143464FF0FF320CA808F08EF886
:100EB0000CA928461035FFF738F90CA8FBF7A4F861
:100EC0003146002048F09AFC0146EAE73846FAF736
:100ED000EFF808A92046FEF705F8044608A8FBF736
:100EE00093F895E7C00B9DEAC10B9DEAD47526E8FF
:100EF000C09E2045D0F8501110B54B1E88B000EBB5
:100F000001110446C0F8503104A8FCF747FB04A9BE
:100F10006846FDF7C5FF04A8FBF776F89DF800309A
:100F20000E2B01D0102B15D1684606F000FE4FF6AF
:100F30000872036804A9204604920693FDF7D2FFC5
:100F4000044604A8FBF760F86846FBF75DF8204606
:100F500008B010BD0024F7E710B586B00446684617
:100F600027F090FD0B4A0023DDE90001EFF7C4FFF5
:100F70004FF613730293EFF73BFBCDE9040102A98F
:100F80002046FDF7AFFF044602A8FBF73DF82046D8
:100F900006B010BD40420F00D0F8501110B54B1EE6
:100FA00088B000EB01110446C0F8503104A8FCF7EA
:100FB000F5FA04A96846FDF773FF04A8FBF724F8C7
:100FC0009DF800300C2B16D19DED020B40F0C4FDB6
:100FD0004FF60C7304938DED060B204604A9FDF724
:100FE00081FF044604A8FBF70FF86846FBF70CF8EE
:100FF000204608B010BD0B2B0BD10021684607F02E
:10100000BDF840F045FE4FF60B738DED060A0493D4
:10101000E3E7A3F10902012A0CD80021684607F092
:101020008DF9EFF7E5FA41EC100B40F095FD4FF626
:101030000B73CFE7023B062B04D8DDED027AB8EE46
:10104000E70ADEE70024D0E7D0F8501110B54B1EB8
:1010500088B000EB01110446C0F8503104A8FCF739
:101060009DFA04A96846FDF71BFF04A8FAF7CCFF18
:101070009DF800300C2B16D19DED020B40F0BCFB0F
:101080004FF60C7304938DED060B204604A9FDF773
:1010900029FF044604A8FAF7B7FF6846FAF7B4FF39
:1010A000204608B010BD0B2B0BD10021684607F07D
:1010B00065F840F0A9FD4FF60B738DED060A049319
:1010C000E3E7A3F10902012A0CD80021684607F0E2
:1010D00035F9EFF78DFA41EC100B40F08DFB4FF630
:1010E0000B73CFE7023B062B04D8DDED027AB8EE96
:1010F000E70ADEE70024D0E7D0F8501110B54B1E08
:1011000088B000EB01110446C0F8503104A8FCF788
:1011100045FA04A96846FDF7C3FE04A8FAF774FF70
:101120009DF800300C2B16D19DED020B40F05CFEBB
:101130004FF60C7304938DED060B204604A9FDF7C2
:10114000D1FE044604A8FAF75FFF6846FAF75CFF91
:10115000204608B010BD0B2B0BD10021684607F0CC
:101160000DF840F05BFF4FF60B738DED060A04930C
:10117000E3E7A3F10902012A0CD80021684607F031
:10118000DDF8EFF735FA41EC100B40F02DFE4FF68D
:101190000B73CFE7023B062B04D8DDED027AB8EEE5
:1011A000E70ADEE70024D0E7D0F8501110B54B1E57
:1011B00088B000EB01110446C0F8503104A8FCF7D8
:1011C000EDF904A96846FDF76BFE04A8FAF71CFFC9
:1011D0009DF800300C2B16D19DED020B40F044FE23
:1011E0004FF60C7304938DED060B204604A9FDF712
:1011F00079FE044604A8FAF707FF6846FAF704FFE9
:10120000204608B010BD0B2B0BD10021684606F01C
:10121000B5FF40F031FF4FF60B738DED060A0493D6
:10122000E3E7A3F10902012A0CD80021684607F080
:1012300085F8EFF7DDF941EC100B40F015FE4FF6A5
:101240000B73CFE7023B062B04D8DDED027AB8EE34
:10125000E70ADEE70024D0E703680D225B682DE98A
:10126000F043D3E9107989B0154B394605466846F5
:10127000002606F05FFC684606F059FC4FF60D7834
:1012800000F10804BE420FD059F82630204604A9C8
:1012900001361B681034CDF810800693FEF745FF29
:1012A00004A8FAF7B1FEEDE769462846FDF71AFEF5
:1012B00004466846FAF7A8FE204609B0BDE8F08368
:1012C000FC8747FFD0F8501110B54B1E88B000EBDB
:1012D00001110446C0F850316846FCF75FF99DF8EB
:1012E0000030184A1B2B12680CBFBDF80830029B57
:1012F000002A21DB21684968086C90421CDD002B24
:101300001ADB496C51F822205168994214DD926829
:1013100052F823304FF60D72049204A9204606932A
:10132000FDF7E0FD044604A8FAF76EFE6846FAF7FA
:101330006BFE204608B010BD4FF60D730493024BB0
:10134000EBE700BF9834022075100608F0B52DEDCC
:10135000028BB5B0154604466846FDF7A1FD294647
:1013600004A8FDF79DFD9DF800100846FEF76CFDF2
:1013700030B99DF810201046FEF766FD002832D0E7
:10138000494A694608A807F067FE484A04A90CA81C
:1013900007F062FE0CAA08A910A807F0B9FF002305
:1013A0009DF8402014A98DF8503010A8404B53F8F8
:1013B00022308022984710A92046FCF7EFF810A8A9
:1013C000FAF722FE0CA8FAF71FFE08A8FAF71CFE8F
:1013D00004A8FAF719FE6846FAF716FE204635B05B
:1013E000BDEC028BF0BD0C2915D00C2A13D00B29B3
:1013F00027D10021684606F0C1FEB0EE408A0021E8
:1014000004A806F0BBFE4FF60B7338EE000A23600B
:1014100084ED020ADCE70021684606F02DFE00217B
:1014200004A857EC106B06F027FE4FF60C713046FF
:101430002160394653EC102BEEF752FFC4E902014C
:10144000C6E70B2AD5D0A1F10903012B12D8002140
:10145000684606F073FF05460E4604A8002106F014
:101460006DFF28184FF6097346EB01012360C4E9AC
:101470000201ADE7A2F10903012BE8D902390629DF
:1014800007D94FF47F43002223600023C4E90223DD
:101490009EE7023A062AF4D8069A029B13444FF6B6
:1014A0000772A360226093E7A8FAEA84B6CA73D2EF
:1014B000CC030020D0F8501110B54B1E8CB0044660
:1014C00000EB0111C0F850316846FCF767F8D4F81A
:1014D000501104A84B1E04EB0111C4F85031FCF765
:1014E0005DF808A86A4604A9FFF730FF9DF82000C0
:1014F00018B108A92046FDF7F5FC044608A8FAF73C
:1015000083FD04A8FAF780FD6846FAF77DFD2046C2
:101510000CB010BDF0B52DED028B89B01546044618
:101520006846FDF7BDFC294604A8FDF7B9FC9DF807
:1015300000200C2A03D09DF810300C2B1FD1002165
:10154000684606F099FD002104A857EC106B06F0E0
:1015500093FD4FF60C7130462160394653EC102B49
:10156000EEF7BCFEC4E9020104A8FAF74DFD684697
:10157000FAF74AFD204609B0BDEC028BF0BD0B2AFC
:1015800018D00B2B16D0A2F10901012924D8002173
:10159000684606F0D3FE05460E4604A8002106F074
:1015A000CDFE281A4FF6097366EB01062360C4E9E5
:1015B0000206D9E70021684606F0E0FDB0EE408A59
:1015C000002104A806F0DAFD4FF60B7338EE400A4E
:1015D000236084ED020AC7E7A3F109010129D6D9E6
:1015E000023A062A07D94FF47F43002223600023E2
:1015F000C4E90223B8E7023B062BF4D8069A029B03
:101600009B1A4FF60772A3602260ADE7D0F8501125
:1016100010B54B1E8CB0044600EB0111C0F85031E0
:101620006846FBF7BBFFD4F8501104A84B1E04EB2F
:101630000111C4F85031FBF7B1FF08A86A4604A9AC
:10164000FFF768FF9DF8200018B108A92046FDF7B4
:1016500049FC044608A8FAF7D7FC04A8FAF7D4FC1A
:101660006846FAF7D1FC20460CB010BDF0B52DED60
:10167000028B89B0154604466846FDF711FC2946E1
:1016800004A8FDF70DFC9DF800200C2A03D09DF85E
:1016900010300C2B1FD10021684606F0EDFC002114
:1016A00004A857EC106B06F0E7FC4FF60C713046BF
:1016B0002160394653EC102BEEF7C8FFC4E9020154
:1016C00004A8FAF7A1FC6846FAF79EFC204609B088
:1016D000BDEC028BF0BD0B2A1CD00B2B1AD0A2F153
:1016E0000901012928D80021684606F027FE054691
:1016F0000E4604A8002106F021FE4FF6097305FBF3
:1017000001F2236000FB0623A5FB00500344C4E95B
:101710000253D5E70021684606F030FDB0EE408A5E
:10172000002104A806F02AFD4FF60B7328EE000AEC
:10173000236084ED020AC3E7A3F109010129D2D98C
:10174000023A062A07D94FF47F4300222360002380
:10175000C4E90223B4E7023B062BF4D8069A029BA5
:1017600053434FF60772A3602260A9E7D0F85011E7
:1017700010B54B1E8CB0044600EB0111C0F850317F
:101780006846FBF70BFFD4F8501104A84B1E04EB7E
:101790000111C4F85031FBF701FF08A86A4604A9FB
:1017A000FFF764FF9DF8200018B108A92046FDF757
:1017B00099FB044608A8FAF727FC04A8FAF724FCCA
:1017C0006846FAF721FC20460CB010BD2DE9F04127
:1017D0002DED028B88B0154604466846FDF760FB88
:1017E000294604A8FDF75CFB9DF800200C2A03D0D5
:1017F0009DF810300C2B15D10021684606F03CFCFA
:10180000002104A857EC106B06F036FC4FF60C7163
:1018100053EC102B216030463946EFF741F8C4E90C
:10182000020134E00B2A21D00B2B1FD0A2F10901B9
:10183000012938D80021684606F080FD07460E468B
:1018400004A8002106F07AFD4FF60C7380460D4681
:10185000236038463146EEF7CBFE06460F4640463B
:101860002946EEF7C5FE02460B46D4E7002168463E
:1018700006F084FCB0EE408A002104A806F07EFC4D
:101880004FF60B73C8EE007A2360C4ED027A04A809
:10189000FAF7BAFB6846FAF7B7FB204608B0BDEC8A
:1018A000028BBDE8F081A3F109010129C2D9023AF6
:1018B000062A07D94FF47F43002223600023C4E99E
:1018C0000223E4E7023B062BF4D80298EEF754FE1D
:1018D00006460F460698EEF74FFE0B46024639467F
:1018E0003046EEF7DDFF4FF60C73236097E7D0F834
:1018F000501110B54B1E8CB0044600EB0111C0F81E
:1019000050316846FBF74AFED4F8501104A84B1E2C
:1019100004EB0111C4F85031FBF740FE08A86A46F9
:1019200004A9FFF753FF9DF8200018B108A920462D
:10193000FDF7D8FA044608A8FAF766FB04A8FAF7F8
:1019400063FB6846FAF760FB20460CB010BD2DE93A
:10195000F04389B0154604466846FDF7A1FA2946CA
:1019600004A8FDF79DFA6846002106F085FB68464D
:10197000002157EC106B06F07FFB04A8002159EC06
:10198000108B06F079FB4046494653EC102BEEF7DE
:1019900087FF41EC100B3FF08FFF04A8002159ECAA
:1019A000108B06F069FB4FF60C71404621604946EA
:1019B00053EC102BEEF74AFE02460B4630463946F2
:1019C000EEF78CFCC4E9020104A8FAF71DFB684697
:1019D000FAF71AFB204609B0BDE8F083D0F85011A1
:1019E00010B54B1E8CB0044600EB0111C0F850310D
:1019F0006846FBF7D3FDD4F8501104A84B1E04EB46
:101A00000111C4F85031FBF7C9FD08A86A4604A9C2
:101A1000FFF79DFF9DF8200018B108A92046FDF7AB
:101A200061FA044608A8FAF7EFFA04A8FAF7ECFA04
:101A30006846FAF7E9FA20460CB010BD30B589B017
:101A4000154604466846FDF72BFA294604A8FDF71B
:101A500027FA0021684606F00FFC0546002104A87D
:101A600006F00AFC4FF6077305FA00F02360A06049
:101A700004A8FAF7C9FA6846FAF7C6FA204609B088
:101A800030BDD0F8501110B54B1E8CB0044600EBA1
:101A90000111C0F850316846FBF780FDD4F85011B1
:101AA00004A84B1E04EB0111C4F85031FBF776FD7E
:101AB00008A86A4604A9FFF7C1FF9DF8200018B1E5
:101AC00008A92046FDF70EFA044608A8FAF79CFA82
:101AD00004A8FAF799FA6846FAF796FA20460CB085
:101AE00010BD30B589B0154604466846FDF7D8F9F3
:101AF000294604A8FDF7D4F90021684606F0BCFB8E
:101B00000546002104A806F0B7FB4FF6077345FA17
:101B100000F02360A06004A8FAF776FA6846FAF7A6
:101B200073FA204609B030BDD0F8501110B54B1EE5
:101B30008CB0044600EB0111C0F850316846FBF749
:101B40002DFDD4F8501104A84B1E04EB0111C4F86C
:101B50005031FBF723FD08A86A4604A9FFF7C1FF2F
:101B60009DF8200018B108A92046FDF7BBF90446EE
:101B700008A8FAF749FA04A8FAF746FA6846FAF705
:101B800043FA20460CB010BD30B589B01446054666
:101B90006846FDF785F9214604A8FDF781F9002183
:101BA000684607F02BFB0446002104A807F026FB3B
:101BB00004404FF6077304A8E4B22B60AC60FAF758
:101BC00023FA6846FAF720FA284609B030BDD0F863
:101BD000501110B54B1E8CB0044600EB0111C0F83B
:101BE00050316846FBF7DAFCD4F8501104A84B1EBC
:101BF00004EB0111C4F85031FBF7D0FC08A86A4689
:101C000004A9FFF7C1FF9DF8200018B108A92046DC
